:020000040000FA
:1000000008480400010000000CFB00000CFB00008D
:100010000CFB00000CFB00000CFB00000CFB0000C4
:100020000CFB00000CFB00000CFB00000CFB0000B4
:100030000CFB00003EF200000CFB00000CFB00007B
:100040000CFB000064F200008AF200000CFB0000D0
:100050000CFB000038F000008AF00000F8230000DC
:100060000CFB00000CFB0000C6E400004AE10000AD
:100070000CFB00009CFA00001EF800000CFB0000C6
:100080000CFB000088F900000CFB00000CFB0000DA
:100090000CFB0000C0F20000E6F200005EF8000079
:1000A000C2F0000014F100000CFB00000CFB00008B
:1000B0000CFB00000CFB00000CFB00000CFB000024
:1000C0000CFB00000CFB00000CFB00000CFB000014
:1000D0000CFB00000CFB0000E2FA00000CFB00002F
:1000E0000CFB00000CFB00000CFB000052E50000C4
:1000F000E0E100000CFB00000CFB000074FA0000C3
:100100009AF800000CFB00000CFB00000CFB000048
:100110000CFB00000CFB00000CFB00000CFB0000C3
:100120000CFB00000CFB00000CFB00000CFB0000B3
:100130000CFB00000CFB00000CFB00000CFB0000A3
:100140000CFB00000CFB000060FA00000CFB000040
:100150000CFB00000CFB00000CFB00000CFB000083
:100160000CFB00000CFB00000CFB00000CFB000073
:100170000CFB00000CFB0000DAE5000076E200005A
:1001800024EF00000CFB00000CFB00000CFB000047
:100190000CFB00000CFB00000CFB0000F0F3000067
:1001A0000CFB00000CFB00000CFB00000CFB000033
:1001B0000CFB00000CFB00000CFB00000CFB000023
:1001C0000CFB00000CFB00000CFB00000CFB000013
:1001D0000CFB00000CFB00000CFB00000CFB000003
:1001E0000CFB00000CFB00000CFB00000CFB0000F3
:1001F0000CFB00000CFB00000CFB00000CFB0000E3
:1002000000000000000000000CFB00000CFB0000E0
:100210000CFB00000CFB00000CFB00000CFB0000C2
:100220000CFB00000CFB00000CFB00000CFB0000B2
:100230000CFB00003EF200000CFB00000CFB000079
:100240000CFB000064F200008AF200000CFB0000CE
:100250000CFB000038F000008AF00000F8230000DA
:100260000CFB00000CFB0000C6E400004AE10000AB
:100270000CFB00009CFA00001EF800000CFB0000C4
:100280000CFB000088F900000CFB00000CFB0000D8
:100290000CFB0000C0F20000E6F200005EF8000077
:1002A000C2F0000014F100000CFB00000CFB000089
:1002B0000CFB00000CFB00000CFB00000CFB000022
:1002C0000CFB00000CFB00000CFB00000CFB000012
:1002D0000CFB00000CFB0000E2FA00000CFB00002D
:1002E0000CFB00000CFB00000CFB000052E50000C2
:1002F000E0E100000CFB00000CFB000074FA0000C1
:100300009AF800000CFB00000CFB00000CFB000046
:100310000CFB00000CFB00000CFB00000CFB0000C1
:100320000CFB00000CFB00000CFB00000CFB0000B1
:100330000CFB00000CFB00000CFB00000CFB0000A1
:100340000CFB00000CFB000060FA00000CFB00003E
:100350000CFB00000CFB00000CFB00000CFB000081
:100360000CFB00000CFB00000CFB00000CFB000071
:100370000CFB00000CFB0000DAE5000076E2000058
:100380009E4801000CFB00000CFB00000CFB000071
:100390000CFB00000CFB00000CFB0000F0F3000065
:1003A0000CFB00000CFB00000CFB00000CFB000031
:1003B0000CFB00000CFB00000CFB00000CFB000021
:1003C0000CFB00000CFB00000CFB00000CFB000011
:1003D0000CFB00000CFB00000CFB00000CFB000001
:1003E0000CFB00000CFB00000CFB00000CFB0000F1
:1003F0000CFB00000CFB00000CFB00000CFB0000E1
:1004000000480400010000004F472300607D2400E5
:1004100000018800000000000B000700E05D2B00D9
:100420000100200010000700000020000000E00094
:100430000200320000000200000000007ABF02004B
:10044000000000000000FE004440A900E0AE2100D2
:100450000000E0000300320000002000A00188003E
:100460004440A80000000600F8FF2000591C2100AD
:1004700091018800800078000000EB001A0037002E
:100480008180E80032A0B4009101BA00E28040000F
:1004900032A0B4009102BA00E280400032A0B40061
:1004A0000002EB00472BDE00F507B200602CE100F4
:1004B00009003A00330007000700E00002003200A4
:1004C0000059EB00010037000201E8008301E90058
:1004D000F8FF3E00040037006128E100010032000F
:1004E0000082EB00040007001101BA000200E000E6
:1004F000E3FF3A0000000600220007000700E000CA
:10050000020032003159BA00020037008100E800D1
:100510000201E8008301E90017003200190007001A
:100520000700E000020032002159BA000200370043
:100530008100E9000201E8008301E9000D003200BA
:100540000400E00003003A00E280400032A0B40062
:10055000E9FF37000B0007000700E000020032004F
:1005600011D9BA00010037000201E8008301E90057
:10057000F5FF3A008100E800E180400032A0B400BD
:10058000000006000810E600020037000910E6002F
:10059000020037008083EB00000006008003EB00C0
:1005A000000006008A1F78008B1F780000000600FC
:1005B00091018800800478000000EB001A003700E9
:1005C000E284440032A0B4009905BA00E2844400F9
:1005D00032A0B4009906BA00E284440032A0B4000C
:1005E0000006EB00476FDE00FD07B200636CE10020
:1005F00003003A00EBFF07000000EB000A003700A1
:10060000606CE10004003A00005DEB008B05E9003E
:10061000FDFF3E00040037006168E1000100320088
:100620000086EB000B00070019C7BA001905BA00D5
:100630000E04E00003003A000A00E000E0FF3A0088
:1006400000000600FE07B2009E0188008A047800C0
:10065000F5FF3700395DBA008B05E9000C00320068
:10066000295DBA008B05E900080032000C00E000AB
:1006700003003A00E284440032A0B400F5FF3700E2
:1006800019DDBA008B05E900FAFF3A008904E80099
:10069000E184440032A0B40000000600FEFA040029
:1006A0000000000060D7040000000000D4CD04006A
:1006B00000000000BCBE040000000000F2BD040009
:1006C000000000000CBE0400000000005ABE040040
:1006D0000000000040E90400000000007EE004008B
:1006E00000000000DAF3040000000000F8C104007C
:1006F00000000000D0B104000000000008BA0400AF
:100700000000000004BA0400000000003EBA04002B
:10071000000000000CBA04000000000070BA0400E1
:1007200000000000A664040000000000D86404007B
:100730000000000008650400000000004A65040095
:10074000000000009265040000000000DA6504006B
:10075000000000002066040000000000986604000D
:1007600000000000E46604000000000030670400A0
:10077000000000009067040000000000FE67040015
:10078000000000007C68040000000000CC68040049
:1007900000000000E8680400000000007069040028
:1007A00000000000C869040000000000046A0400A2
:1007B00000000000406A040000000000A66A040077
:1007C00000000000DE6B040000000000106C04005C
:1007D00000000000346C040000000000826C040083
:1007E00000000000006D0400000000004E6D0400D9
:1007F00000000000986D040000000000C66D0400B9
:1008000000000000F86D0400000000003A6E0400D3
:1008100000000000569C040000000000C49C04007E
:10082000000000008A9C040000000000FE9C040000
:10083000000000007E9D040000000000BC9D04003C
:1008400000000000549E040000000000B89E040058
:1008500000000000869E04000000000084A0040048
:1008600000000000EA9E040000000000489F040011
:1008700000000000E09F04000000000016A004003B
:100880000000000032A00400000000004EA00400A0
:1008900000000000B4A0040000000000EAA0040072
:1008A0000000000006A10400000000006EA104008A
:1008B000000000009EA1040000000000CEA1040082
:1008C00000000000FAA1040000000000389D0400B0
:1008D0000000000036BF0400000000000E9A040073
:1008E000000000001CC10400000000002C9B04005C
:1008F000000000006022B800060220000000D000C6
:100900008180D2000482D2008582D2000000A00043
:100910000202520083825A000300310002024200A8
:1009200083824A000000A1000603E900F3FF3A00B9
:1009300000000600020AB900001BB9000200B8005E
:10094000810042008100430000000600889FBE0035
:100950008A9FBE008C1F78000006EB00E00F50005D
:10096000E08F5800E00F5900E08F590007003D006C
:100970006044B8006055B8000000540081805C00FD
:1009800002015D0083815D001C002000E00F520029
:10099000E08F5A00E00F5B00E08F5B0007003D0036
:1009A0006044B8006055B8000402540085825C00C1
:1009B00006035D0087835D000C00A200170107009D
:1009C0000C00E000060032006022B8006033B8007E
:1009D0000000520081805A0002015B0083815B00AD
:1009E0004F0678004F05BE004F04BE000000060011
:1009F000889FBE008A9FBE0030044200B0844A0037
:100A000030054B0090854B006000B1000898BE0097
:100A10000A90BE00C10007000200310068004000DB
:100A20001008E8004F05BE004F04BE00000006009D
:100A3000889FBE008A9FBE003004BE002005BE0015
:100A40000418540005985C0006185D0007985D00C6
:100A500011002000B1000700010039008000EB0008
:100A6000108810004F05BE004F04BE0000000600B5
:100A70001200FA00889FBE008A9FBE008C9FBE00B5
:100A8000E0B79F00F1B79F0082BF9F0093BF9F0018
:100A90000605BE000404BE000000EB00D0B79F00B6
:100AA000C0B79F00B0B79F00A0B79F0090B79F004E
:100AB0000006EB005FB19700CFB0970082014100C4
:100AC0003FB097000200E00004003D0098000700DE
:100AD0007E805700C6FF0700030037009400070020
:100AE0007E805700D2FF0700DFB697000D00E000C0
:100AF0000C0035006FB29700FFB297000FBB970054
:100B00009FBB970010002000010020006011B8007A
:100B100000027200818272000203730083837300FB
:100B2000580007000C06E80001042000810F560061
:100B3000E0FF3A000D00E00004003D000802BE00A6
:100B40000A03BE007E805700A9FF07005FA8970038
:100B50000000E00005003A001FB29700AFB2970016
:100B60003FB39700CFB39700460007006FB09700E0
:100B7000FFB097000FB997009FB997004F06BE00CE
:100B80004F05BE004F04BE000080FA0000000600C2
:100B9000881F780018002000881F7800B4FF070025
:100BA0008F87E9004F04780000000600801FEB00EB
:100BB000AFFF07008F87E90000000600889FBE0096
:100BC0008A9FBE003D00070007003D00400007006F
:100BD000180020004500070008003D002B0007001A
:100BE0000004EB00050037000004EB003F000700A5
:100BF00002003D002500070018002000E4FF070068
:100C00000800E000010032003D0007004F05BE0073
:100C10004F04BE0000000600889FBE008A9FBE00F1
:100C20008C1F78002500070008003D002800070001
:100C30001C0020000820E10009A8E1000AB0E10042
:100C40000BB8E10007003D00050037000006EB008F
:100C50002600070003003D006044B8006055B8005E
:100C60000C000700D1FF07000C00E000010032007B
:100C7000230007004F0678004F05BE004F04BE005A
:100C80000000060008000700000006006044B800ED
:100C90006055B8000402540085825C0006035D00C4
:100CA00087835D0000000600A4B79F00B5B79F00D2
:100CB000C6B79F00D7B79F0000000600E00F5000A6
:100CC000E08F5800E00F5900E08F59000000060047
:100CD0006044B8006055B8000000540081805C009A
:100CE00002015D0083815D0000000600E00F5200FC
:100CF000E08F5A00E00F5B00E08F5B000000060011
:100D00006022B8006033B8000000520081805A00B1
:100D100002015B0083815B00000006000440E100EB
:100D200005C8E10006D0E10007D8E1000000060098
:100D30004F09DE0082817100B3B79F004F01DE00D2
:100D40008180400082807000A1B79F008FB0970023
:100D50004F09DE00000040000200700090B79F00C5
:100D60007FA897004F01DE008180400082807000E4
:100D700081B79F000D0007004F3ADE0000004000E1
:100D800004007000F0AF9F0008000700040242005A
:100D900085824A0006034B0087834B00C2FF070091
:100DA0000802BE000A03BE00000006002FB2970032
:100DB000BFB297004FB39700DFB397000000060063
:100DC00080017800110009008280D8008001FD00B8
:100DD000110009004288D800830078000000060056
:100DE000839F68000100E00002003D0060001000E9
:100DF000E08018000300E00002003D0060011100E7
:100E0000E0811900BBFE07004F00E00002003B003C
:100E100060001000E080180000000600889FBE00FF
:100E20008A9FBE008C9FBE000404B8000506B8006F
:100E30008904460060854E000606B8000A05460093
:100E4000E0854E000706B8008B054600040EB8008A
:100E5000890446000A854E00E0854D00050EB80065
:100E60000A0546008B854E00060EB8008B0546002D
:100E70000416B8000A0546008B854E000516B8001A
:100E80008B054600041EB8008B0546000800BE0016
:100E90000A01BE004F06BE004F05BE004F04BE0053
:100EA000000006008001780002003700B159780088
:100EB0000201E9000200E000FCFF3A000000060029
:100EC000800078003104E000FEFF3A000080EA0074
:100ED000008040000000060080017800020037001A
:100EE000815978000201E9000200E000FCFF3A00AD
:100EF00000000600E68747008E1F7800D0BF9F00E5
:100F0000E1BF9F000E0037005FBA970014407800E1
:100F1000EFB99700934078000201E900814F50003B
:100F2000040032000080FB008180FB0001005000C3
:100F30000600370066875700041FE800030FE8002B
:100F40000200E000F0FF3A000000EB004F077800DD
:100F50006F00B100000006004E65000067610000F0
:100F60007469000076650000206900006E70000062
:100F700075740000207400006F2000007371000081
:100F800072740000006D000061740000682E0000A3
:100F9000636F000070790000006300006F70000054
:100FA0006965000073200000737200006320000078
:100FB000746F00002064000065730000742000005E
:100FC000656C0000656D0000656E00007420000017
:100FD00062790000206500006C6500006D6500000E
:100FE0006E7400000064000065730000740000006F
:100FF0007372000063000000C3870000CD8700000B
:10100000FFFF0000F3870000FFFF0000F8870000EB
:1010100000000000000000006D6100007468000026
:101020002E660000696C00006C000000666900001C
:101030006C6C000073200000646500007374000095
:10104000207700006974000068200000636F0000D2
:101050006E730000746100006E7400002076000062
:10106000616C00007565000000760000616C000096
:1010700075650000000000000C8800001688000064
:10108000FFFF0000F387000001000000358800002A
:1010900000000000000000006D61000074680000A6
:1010A0002E6100006464000073630000616C000046
:1010B00061720000006100006464000020730000A1
:1010C000636100006C61000072200000746F00001A
:1010D000206500006163000068200000656C00006E
:1010E000656D0000656E0000742000006F660000F2
:1010F0002073000072630000206100006E64000035
:1011000020730000746F0000726500002072000000
:1011100065730000756C000074200000746F00009F
:101120002064000065730000740000007363000019
:10113000616C000061720000000000004C8800003B
:101140005B880000FFFF0000F3870000FFFF000046
:10115000F8870000010000009688000000000000F1
:10116000000000006D610000746800002E61000046
:1011700064640000006100006464000073200000EB
:101180007372000063310000206100006E64000093
:101190002073000072630000322C000020770000F2
:1011A0007269000074650000207400006F20000068
:1011B00064650000737400002C200000656C000062
:1011C000656D0000656E000074200000627900000B
:1011D000206500006C6500006D6500006E74000005
:1011E00000730000726300003100000073720000A1
:1011F0006332000000000000B2880000BB880000DD
:10120000FFFF0000F3870000FFFF0000F1880000EF
:10121000FFFF0000F6880000000000000000000052
:101220006D610000746800002E730000756200009C
:1012300000730000756200007374000072610000AA
:1012400063740000732000007372000063320000BA
:1012500020660000726F00006D20000073720000B5
:1012600063310000207400006F20000064650000FE
:10127000737400002C200000656C0000656D000098
:10128000656E000074200000627900002065000097
:101290006C6500006D6500006E74000000000000C9
:1012A0001089000019890000FFFF0000F38700008B
:1012B000FFFF0000F1880000FFFF0000F68800003B
:1012C00000000000000000006D6100007468000074
:1012D0002E6D0000756C0000006D0000756C000044
:1012E00074690000706C00006965000073200000E4
:1012F0007372000063310000206100006E64000022
:10130000207300007263000032200000746F000040
:101310002064000065730000742C0000206500004C
:101320006C6500006D6500006E74000020620000B6
:1013300079200000656C0000656D0000656E00009E
:1013400074000000648900006D890000FFFF000048
:10135000F3870000FFFF0000F1880000FFFF00009E
:10136000F688000000000000000000006D61000031
:10137000746800002E6400006976000000640000BC
:101380006976000069640000657300002073000046
:1013900072630000312000006279000020730000B9
:1013A0007263000032200000746F000020640000AF
:1013B00065730000742C0000206500006C6500005F
:1013C0006D6500006E74000020620000792000004E
:1013D000656C0000656D0000656E00007400000023
:1013E000B6890000BF890000FFFF0000F3870000FE
:1013F000FFFF0000F1880000FFFF0000F6880000FA
:1014000000000000000000006D6100007468000032
:101410002E6D0000696E0000007700007269000008
:1014200074650000732000007468000065200000EF
:101430006D6900006E6900006D7500006D20000090
:101440006F6600002073000072630000312000000E
:10145000616E0000642000007372000063320000BF
:10146000207400006F2000006465000073740000A9
:101470002C200000656C0000656D0000656E0000AA
:101480007420000062790000206500006C65000097
:101490006D6500006E74000000000000048A00000A
:1014A0000D8A0000FFFF0000F3870000FFFF00002F
:1014B000F1880000FFFF0000F68800000000000037
:1014C000000000006D610000746800002E6D0000D7
:1014D0006178000000770000726900007465000008
:1014E0007320000074680000652000006D6100003A
:1014F000786900006D7500006D2000006F660000C7
:10150000207300007263000031200000616E000053
:101510006420000073720000633200002074000039
:101520006F20000064650000737400002C20000030
:10153000656C0000656D0000656E000074200000A1
:1015400062790000206500006C6500006D65000098
:101550006E74000000000000628A00006B8A0000C8
:10156000FFFF0000F3870000FFFF0000F18800008C
:10157000FFFF0000F68800000000000000000000EF
:101580006D610000746800002E6300006C61000053
:101590006D700000006300006C6100006D70000061
:1015A0002073000072630000207400006F200000B0
:1015B0006C6F0000772F000068690000676800000A
:1015C000206200006F7500006E6400007320000050
:1015D000696E0000746F00002064000065730000F5
:1015E000742C0000206500006C6500006D65000033
:1015F0006E7400002062000079200000656C00001D
:10160000656D0000656E0000740000006C6F0000E6
:1016100077000000686900006768000000000000B3
:10162000C08A0000CB8A0000FFFF0000F3870000A3
:10163000FFFF0000F8870000FFFF0000068B00009E
:10164000FFFF00000A8B0000000000000000000007
:101650006D610000746800002E6400006F7400006B
:1016600000770000726900007465000073200000BC
:101670007468000065200000646F000074200000A2
:10168000707200006F640000756300007420000039
:101690006F660000207300007263000031200000BC
:1016A000616E00006420000073720000633200006D
:1016B000207400006F200000646500007374000057
:1016C0002C2000006166000074650000722000009C
:1016D000612000007368000069660000740000006B
:1016E000736800006966000074000000288B000029
:1016F000318B000001000000F3870000FFFF0000B5
:10170000F1880000FFFF0000F688000001000000E3
:10171000708B000000000000000000006D61000000
:10172000746800002E7300007461000074000000F3
:1017300070650000726600006F7200006D7300003B
:10174000207300007461000074690000737400006D
:1017500069630000732000006F6E000020730000BA
:1017600072630000006D0000696E0000006D0000F3
:1017700061780000006D0000656100006E000000EF
:101780008E8B0000988B0000FFFF0000F8870000A0
:1017900001000000B38B000001000000B78B0000C7
:1017A00001000000BB8B00000000000000000000F2
:1017B0006D610000746800002E6100007267000017
:1017C000626F0000756E0000647300000067000027
:1017D0006574000020740000686500002069000046
:1017E0006E6400006963000065730000202800003B
:1017F00061720000676D0000696E00002C2000001F
:1018000061720000676D000061780000292000000F
:101810006F6600002074000068650000206C000006
:10182000696D00006974000020760000616C0000A2
:1018300075650000732000006F66000020730000D3
:101840007263000000610000726700006D690000B3
:101850006E00000061720000676D0000617800009A
:1018600000000000D88B0000E78B0000FFFF0000A5
:10187000F887000001000000238C00000100000038
:101880002A8C000000000000000000006D610000D4
:10189000746800002E7300006F7200007400000076
:1018A000736F00007274000020610000727200000B
:1018B00061790000206900006E200000706C00005B
:1018C0006163000065000000617200007261000049
:1018D00079000000468C0000508C0000FFFF0000E3
:1018E000648C000000000000000000006D6100003A
:1018F000746800002E6D0000756C000064690000C3
:101900007600000070650000726600006F720000D3
:101910006D730000206400006573000074200000F7
:101920003D200000286100002A620000292F0000ED
:1019300063200000696E00002033000032200000A8
:101940006269000074730000206500006C6500008F
:101950006D6500006E7400002062000079200000B8
:10196000656C0000656D0000656E0000740000008D
:10197000610000006200000063000000768C00003F
:10198000828C0000FFFF0000F3870000FFFF0000D3
:10199000B88C0000FFFF0000BA8C0000FFFF0000C1
:1019A000BC8C000000000000000000006D61000021
:1019B000746800002E610000746100006E32000047
:1019C0000070000065720000666F0000726D00001C
:1019D000732000006465000073740000203D000067
:1019E00020610000746100006E3200002879000060
:1019F0002C78000029200000656C0000656D000057
:101A0000656E00007420000062790000206500000F
:101A10006C6500006D6500006E74000000790000C8
:101A20000078000000000000D68C0000E18C00006F
:101A3000FFFF0000F3870000FFFF00000F8D000094
:101A4000FFFF0000118D00000000000000000000FA
:101A50006D610000746800002E730000696E000064
:101A60000070000065720000666F0000726D00007B
:101A7000732000006465000073740000203D0000C6
:101A800020730000696E0000287800002920000003
:101A9000656C0000656D0000656E0000742000003C
:101AA00062790000206500006C6500006D65000033
:101AB0006E74000000000000288D0000318D0000D1
:101AC000FFFF0000F3870000FFFF0000118D000002
:101AD00000000000000000006D610000746800005C
:101AE0002E6300006F73000000700000657200003C
:101AF000666F0000726D00007320000064650000D6
:101B000073740000203D0000206300006F7300002C
:101B10002878000029200000656C0000656D000039
:101B2000656E0000742000006279000020650000EE
:101B30006C6500006D6500006E7400000000000020
:101B40006C8D0000758D0000FFFF0000F387000022
:101B5000FFFF0000118D00000000000000000000E9
:101B60006D610000746800002E7200006F74000048
:101B700032000000726F00007461000074650000A4
:101B800073200000762000006F66000020610000D6
:101B90006E6700006C65000020610000207400008A
:101BA0006F20000064650000737400000076000080
:101BB00000000000B08D0000BA8D0000020000009F
:101BC000F387000002000000D78D00000100000034
:101BD000B88C000000000000000000006D610000F3
:101BE000746800002E730000717200007400000021
:101BF00070650000726600006F7200006D73000077
:101C00002064000065730000742000003D20000087
:101C10007371000072740000287800002920000011
:101C2000656C0000656D0000656E000074200000AA
:101C300062790000206500006C6500006D650000A1
:101C40006E74000000000000EE8D0000F88D0000B2
:101C5000FFFF0000F3870000FFFF0000118D000070
:101C600000000000000000006D61000074680000CA
:101C70002E6E00007A73000065710000007700008E
:101C80007269000074650000207400006F2000007D
:101C90006465000073740000207400006865000033
:101CA000206D000069640000646C00006520000085
:101CB000696E000064650000782000006F66000017
:101CC0002074000068650000206C00006172000054
:101CD00067650000737400002073000065710000E8
:101CE000756500006E630000652000006F660000EF
:101CF000206E00006F6E00002D7A000065720000FB
:101D00006F200000656C0000656D0000656E0000CE
:101D10007473000020660000726F00006D200000E8
:101D200073720000632C0000202D000031200000A1
:101D300069660000206E00006F74000020660000DD
:101D40006F7500006E640000206F000072200000BC
:101D500069660000207300006D6100006C6C00007B
:101D60006572000020740000686100006E200000B1
:101D70006D6900006E4C0000656E00006774000025
:101D8000680000006D6900006E4C0000656E000088
:101D90006774000068000000348E00003F8E000071
:101DA00001000000F3870000FFFF0000F88700003B
:101DB00001000000C28E00000000000000000000D2
:101DC0006D610000746800002E720000616E0000FA
:101DD00064000000666900006C6C00002061000077
:101DE00072720000617900002077000069740000C1
:101DF00068200000726100006E6400006F6D0000DA
:101E000020760000616C0000756500007300000022
:101E1000E08E0000EA8E0000FFFF0000F387000064
:101E20000000000000000000646500007175000003
:101E3000652E0000736900007A65000000720000E2
:101E4000657000006F72000074200000736900006C
:101E50007A650000206F00006620000064650000C5
:101E60007374000000640000657100007565000077
:101E700000730000697A000065000000148F000004
:101E80001F8F0000FFFF0000338F000001000000E3
:101E9000398F0000000000000000000064650000B1
:101EA00071750000652E0000676500007400000079
:101EB000666900006C6C000020640000657300001F
:101EC00074200000667200006F6D00002064000046
:101ED000657100007565000020610000742000003D
:101EE000696E00006465000078000000696E000003
:101EF00064650000780000004E8F0000588F0000DD
:101F0000FFFF0000338F0000FEFF0000F38700009A
:101F100001000000768F00000000000000000000BB
:101F20006465000071750000652E00007365000097
:101F300074000000636F00007069000065730000AA
:101F40002073000072630000207400006F20000006
:101F50006465000071750000652000006174000078
:101F6000206900006E640000657800000000000039
:101F7000908F00009A8F0000FFFF0000338F000059
:101F8000FEFF0000F887000001000000768F0000CF
:101F90000000000000000000646500007175000092
:101FA000652E0000696E0000736500007274000009
:101FB000007300006869000066740000206400007F
:101FC000657100007565000020610000742000004C
:101FD000696E0000646500007820000062790000EE
:101FE000206C0000656E0000287300007263000022
:101FF00029200000616E000064200000696E00006E
:1020000073650000727400002073000072630000AA
:1020100000000000CC8F0000D98F0000FFFF0000FF
:10202000338F0000FEFF0000F88700000100000071
:10203000768F0000000000000000000064650000D2
:1020400071750000652E000065720000617300006C
:1020500065000000736800006966000074200000DD
:102060006465000071750000652000006174000067
:10207000206900006E6400006578000020620000A6
:10208000792000006C6500006E200000746F000075
:10209000206500007261000073650000006C0000A4
:1020A000656E0000000000001E9000002A900000F5
:1020B000FFFF0000338F000001000000768F00005A
:1020C000010000004F900000000000000000000030
:1020D0006465000071750000652E000070750000D9
:1020E000736800005F660000726F00006E7400008D
:1020F000006900006E73000065720000742000002B
:10210000737200006320000062650000666F0000CB
:102110007265000020740000686500002066000001
:10212000726F00006E740000206F000066200000D7
:102130006465000071750000650000006890000093
:1021400079900000FFFF0000338F0000FEFF0000C9
:10215000F887000000000000000000006465000037
:1021600071750000652E0000707500007368000036
:102170005F620000616300006B000000696E000098
:102180007365000072740000207300007263000029
:102190002061000066740000657200002074000079
:1021A0006865000020620000616300006B20000091
:1021B0006F66000020640000657100007565000016
:1021C00000000000AE900000BE900000FFFF000085
:1021D000338F0000FEFF0000F887000000000000C1
:1021E000000000006465000071750000652E0000AD
:1021F000706F0000705F0000667200006F6E00007C
:1022000074000000666900006C6C0000206400002F
:102210006573000074200000667200006F6D00009E
:1022200020660000726F00006E740000206F0000D6
:1022300066200000646500007175000065200000E4
:1022400074680000656E0000206500007261000087
:1022500073650000206500006C6500006D6500007E
:102260006E74000073000000F29000000291000004
:10227000FFFF0000338F0000FEFF0000F387000027
:10228000000000000000000064650000717500009F
:10229000652E0000706F0000705F0000626100003A
:1022A000636B000000660000696C00006C20000099
:1022B000646500007374000020660000726F000007
:1022C0006D20000062610000636B0000206F000061
:1022D0006620000064650000717500006520000044
:1022E00074680000656E00002065000072610000E7
:1022F00073650000206500006C6500006D650000DE
:102300006E740000730000004491000053910000BF
:10231000FFFF0000338F0000FEFF0000F387000086
:102320000000000000000000000000009301000019
:1023300024030000B704000048060000DA0700008C
:102340006B090000FC0A00008C0C00001C0E000051
:10235000AB0F00003B110000C81200005614000033
:10236000E31500006E170000F9180000831A000042
:102370000C1C0000941D00001A1F0000A02000008B
:1023800024220000A723000029250000A826000021
:1023900027280000A4290000202B0000992C000011
:1023A000122E0000872F0000FC3000006F3200006A
:1023B000DF3300004E350000BA360000253800003B
:1023C0008D390000F33A0000573C0000B93D000091
:1023D000173F000074400000CE410000264300007B
:1023E0007B440000CD4500001D4700006A48000006
:1023F000B4490000FC4A0000404C0000824D00003F
:10240000C04E0000FC4F0000345100006952000033
:102410009B530000CA540000F65500001E570000F0
:102420004358000064590000835A00009D5B00007F
:10243000B45C0000C85D0000D75E0000E45F0000EF
:10244000EC600000F1610000F2620000EF63000048
:10245000E9640000DE650000D0660000BD67000092
:10246000A76800008C6900006E6A00004B6B0000DA
:10247000246C0000F96C0000CA6D0000976E00002B
:102480005F6F000023700000E37000009E71000089
:102490005572000008730000B673000060740000FD
:1024A00005750000A575000042760000D976000091
:1024B0006C770000FB770000847800000979000049
:1024C0008A790000067A00007D7A0000EF7A000029
:1024D0005D7B0000C67B00002A7C0000897C000038
:1024E000E47C0000397D00008A7D0000D77D00007B
:1024F0001D7E0000607E00009D7E0000D67E0000F4
:10250000097F0000397F0000627F0000877F0000A4
:10251000A77F0000C27F0000D87F0000EA7F000094
:10252000F67F0000FE7F0000FF7F00008C020000AD
:10253000DF0200003003000080030000D103000030
:102540002204000073040000C2040000140500000F
:10255000B305000054060000F10600008F070000DC
:102560002D080000CA08000063090000FC090000F3
:10257000340B00005C0C0000820D0000A40E000073
:10258000BD0F0000D3100000E2110000E7120000B0
:10259000EF140000CC16000092180000401A000052
:1025A000D61B0000531D0000B51E00000B200000CC
:1025B000792200008D2400006F26000014280000FE
:1025C00090290000E02A0000112C0000252D0000B9
:1025D000052F000089300000D3310000EC320000EC
:1025E000DD330000AE340000673500000D3600001A
:1025F00020370000FB370000B23800004A390000E5
:10260000CC3900003B3A00009B3A0000F33A00004E
:10261000833B0000F43B0000513C00009F3C000065
:10262000E13C00001A3D00004B3D0000783D0000F9
:10263000C03D0000F93D0000283E00004F3E000074
:10264000703E00008D3E0000A53E0000BC3E000034
:10265000E03E0000FD3E0000143F0000283F000067
:10266000383F0000473F0000533F00005E3F00003E
:10267000703F00007F3F00008A3F0000943F000051
:102680009C3F0000A43F0000AA3F0000AF3F0000B5
:10269000B83F0000C03F0000C53F0000CB3F000036
:1026A000CE3F0000D23F0000D53F0000D83F0000E1
:1026B000DC3F0000E03F0000E33F0000E53F00009A
:1026C000E83F0000E93F0000EB3F0000EC3F000066
:1026D000EE3F0000F13F0000F13F0000F33F00003B
:1026E000F43F0000F53F0000F53F0000F73F000019
:1026F000F73F0000F93F0000F83F0000FA3F0000FC
:10270000FA3F0000FA3F0000FB3F0000FB3F0000E3
:10271000FC3F0000FC3F0000FC3F0000FE3F0000CB
:10272000FD3F0000FD3F0000FD3F0000FE3F0000B8
:10273000FE3F0000FE3F0000FE3F0000FE3F0000A5
:10274000FE3F000000400000FF3F0000FF3F000090
:10275000FF3F0000FF3F0000FF3F0000FF3F000081
:10276000FF3F0000FF3F0000FF3F0000FF3F000071
:10277000FF3F00000040000000400000004000005B
:102780000040000000400000004000000040000049
:102790000040000000400000004000000040000039
:1027A0000040000000400000004000000040000029
:1027B0004164000064720000657300007320000033
:1027C0006F750000742000006F6600002073000029
:1027D00065740000746900006E67000073000000FB
:1027E000536C000065650000702000006D6F0000F4
:1027F00064650000206E00006F740000207300000C
:1028000075700000706F0000727400006564000055
:1028100000450000727200006F7200003A20000054
:102820006D6900006E2000003D3D0000203000007A
:102830007846000046460000464600004646000036
:10284000462000002100000045720000726F000069
:10285000723A0000205500006E610000626C0000BA
:1028600065200000746F0000206600006C610000AD
:102870007368000020620000797400006563000046
:102880006F6400006520000028310000292000004E
:102890002100000045720000726F0000723A0000D3
:1028A000205500006E610000626C00006520000091
:1028B000746F0000206600006C6100007368000007
:1028C0002062000079740000656300006F640000FE
:1028D00065200000283200002920000021000000AF
:1028E00045720000726F0000723A0000205500002F
:1028F0006E610000626C000065200000746F0000D3
:10290000206600006C610000736800002062000017
:1029100079740000656300006F64000065200000AA
:10292000283300002920000021000000466C000030
:1029300061730000686900006E670000204F0000AE
:102940004B000000564D0000204100005353000092
:10295000455200005420000021000000746800006F
:10296000796D0000696F00002D49000049000000EA
:102970005F6900006400000065760000656E00007D
:10298000742E0000736F0000757200006365000014
:1029900000650000766500006E7400002E61000086
:1029A00072670000730000005F6600007776000029
:1029B00065720000736900006F6E0000005F000028
:1029C000707200006F6400007563000074490000BD
:1029D0006400000062750000747400006F6E0000F7
:1029E000732E00005F72000061770000006200003B
:1029F00075740000746F00006E2E000062610000AC
:102A0000636B0000776100007264000000620000E8
:102A100075740000746F00006E2E00006C6500007D
:102A2000667400000062000075740000746F00009E
:102A30006E2E0000636500006E7400006572000079
:102A40000062000075740000746F00006E2E0000BC
:102A5000666F000072770000617200006400000081
:102A600062750000747400006F6E00002E7200002A
:102A7000696700006874000000620000757400005F
:102A8000746F00006E7300002E5F00006D65000023
:102A9000616E00000062000075740000746F000039
:102AA0006E7300002E5F00006E6F000069730000FF
:102AB00065000000707200006F7800002E68000052
:102AC0006F720000697A00006F6E00007461000090
:102AD0006C000000707200006F7800002E63000030
:102AE0006F6D00006D2E0000727800002E5F0000F8
:102AF00070610000796C00006F6100006473000079
:102B000000700000726F0000782E0000636F0000FC
:102B10006D6D00002E720000782E00005F690000CD
:102B20006E740000656E0000736900007469000037
:102B30006573000000700000726F0000782E0000C6
:102B4000636F00006D6D00002E72000078000000C1
:102B5000707200006F7800002E6300006F6D00003F
:102B60006D2E00007478000000700000726F00008D
:102B7000782E0000677200006F7500006E64000020
:102B80002E6100006D620000696100006E7400003B
:102B900000700000726F0000782E00006772000065
:102BA0006F7500006E6400002E7200006566000004
:102BB0006C65000063740000656400000070000034
:102BC000726F0000782E0000677200006F750000C1
:102BD0006E6400002E640000656C000074610000EB
:102BE000006D00006F7400006F7200002E6C00001A
:102BF00065660000742E00007461000072670000BA
:102C000065740000006D00006F7400006F720000BA
:102C10002E72000069670000687400002E740000C6
:102C20006172000067650000740000005F760000BC
:102C300062610000740000005F6900006D6F0000B9
:102C4000740000006D6F0000746F0000722E0000B1
:102C50006C650000667400002E7300007065000053
:102C600065640000006D00006F7400006F7200006A
:102C70002E72000069670000687400002E73000067
:102C80007065000065640000006D00006F74000056
:102C90006F7200002E6C000065660000742E00004C
:102CA000707700006D0000006D6F0000746F000011
:102CB000722E00007269000067680000742E000028
:102CC000707700006D000000616300006300000089
:102CD000746500006D700000657200006174000092
:102CE000757200006500000072630000352E000060
:102CF00061640000647200006573000073000000EE
:102D000072630000352E0000636F00006D6D0000DF
:102D1000616E0000640000006D690000632E000019
:102D2000696E0000746500006E7300006974000035
:102D3000790000006D690000632E000074680000D7
:102D400072650000736800006F6C00006400000092
:102D50006D690000632E00005F6D0000656100007A
:102D60006E000000746900006D650000722E0000A6
:102D700070650000726900006F640000006100006F
:102D8000636300002E5F00007461000070000000AB
:102D9000736400002E70000072650000736500000F
:102DA0006E74000000000000AE94000001000000FE
:102DB000B894000001000000BC9400002000000056
:102DC000C994000002000000D4940000010000003B
:102DD000DF94000005000000EA94000001000000FC
:102DE000F7940000010000000795000001000000BA
:102DF0001395000001000000219500000100000073
:102E000030950000050000003D9500000500000021
:102E10004B950000070000005A95000007000000D5
:102E20006A95000007000000819500000100000085
:102E30009B95000001000000A89500000200000022
:102E4000B595000002000000C995000002000000D6
:102E5000DF95000001000000F19500000100000076
:102E60000396000002000000169600000200000019
:102E70001C960000010000002296000001000000E6
:102E8000339600000100000045960000010000009C
:102E9000549600000300000064960000010000004A
:102EA0006896000001000000749600000100000018
:102EB00080960000010000008C96000001000000D8
:102EC0009A96000001000000A89600000200000091
:102ED000B296000001000000BF9600000100000053
:102EE000C89600000000000000000000DE000000A6
:102EF000AD000000CA000000FE000000BE0000009F
:102F0000EF000000040000000200000004BA00000E
:102F10003EBA00000CBA000070BA0000A6640000BF
:102F2000D8640000086500004A6500009265000052
:102F3000DA6500002066000098660000E466000084
:102F40003067000090670000FE6700007C680000AA
:102F5000CC680000E868000070690000C8690000E3
:102F6000046A0000406A0000A66A0000DE6B0000F0
:102F7000106C0000346C0000826C0000006D0000DA
:102F80004E6D0000986D0000C66D0000F86D0000E9
:102F90003A6E0000569C0000C49C00008A9C000011
:102FA000FE9C00007E9D0000BC9D0000549E000021
:102FB000B89E0000869E000084A00000EA9E0000EB
:102FC000489F0000E09F000016A0000032A0000013
:102FD0004EA00000B4A00000EAA0000006A100007E
:102FE0006EA100009EA10000CEA10000FAA1000089
:102FF000389D000036BF000042610000636B000096
:1030000077610000726400002062000075740000A7
:10301000746F00006E200000737400006174000083
:103020007573000020630000686100006E67000097
:1030300065640000004C000065660000742000001C
:1030400062750000747400006F6E00002073000051
:103050007461000074750000732000006368000054
:10306000616E0000676500006400000043650000B9
:103070006E7400006572000020620000757400002C
:10308000746F00006E200000737400006174000013
:103090007573000020630000686100006E67000027
:1030A00065640000004600006F7200007761000058
:1030B000726400002062000075740000746F0000EC
:1030C0006E200000737400006174000075730000CE
:1030D00020630000686100006E6700006564000006
:1030E0000052000069670000687400002062000060
:1030F00075740000746F00006E200000737400008F
:1031000061740000757300002063000068610000B6
:103110006E670000656400000062000075740000C6
:10312000746F00006E7300000042000075740000B0
:10313000746F00006E73000020760000616C000068
:103140007565000073200000757000006461000068
:103150007465000064000000707200006F78000069
:1031600000500000726F0000786900006D69000077
:103170007479000020760000616C00007565000025
:103180007320000075700000646100007465000029
:1031900064000000707200006F7800002E63000071
:1031A0006F6D00006D00000044610000746100005C
:1031B000207200006563000065690000766500000C
:1031C000642000006F6E000020740000686500003D
:1031D00020700000726F0000786900006D690000C7
:1031E00074790000206300006F6D00006D750000B1
:1031F0006E69000063610000746900006F6E00007A
:1032000000740000617000000041000020740000A4
:1032100061700000206900007320000064650000F8
:1032200074650000637400006564000000410000E4
:1032300063630000656C0000657200006F6D000044
:10324000657400006572000020760000616C00006B
:103250007565000073200000757000006461000057
:1032600074650000640000006D69000063000000E8
:103270004669000072650000642000007768000065
:10328000656E0000206D000069630000726F000031
:10329000706800006F6E000065200000696E00001D
:1032A000746500006E7300006974000079200000EE
:1032B0006973000020610000626F00007665000005
:1032C000207400006872000065730000686F0000E1
:1032D0006C640000007300006F7500006E640000F5
:1032E0002E660000696E00006973000068650000CA
:1032F0006400000046690000726500006420000060
:1033000077680000656E00002074000068650000AA
:10331000207000006C6100007962000061630000B1
:103320006B2000006F660000206100002075000027
:103330007365000072200000696E0000697400006F
:10334000696100007465000064200000736F000074
:10335000756E0000642000006973000020660000A4
:10336000696E000069730000686500006400000079
:10337000546500006D70000065720000617400000B
:103380007572000065200000766100006C75000019
:103390006520000075700000646100007465000025
:1033A000640000007263000035000000524300001A
:1033B000352000006D650000737300006167000038
:1033C00065200000726500006365000069760000FA
:1033D00065640000006D00006F7400006F720000F3
:1033E000004D00006F7400006F7200002074000038
:1033F000696D00006572000000740000696D0000D6
:103400006572000030000000546900006D65000026
:103410007220000030000000746900006D6500003B
:103420007231000000540000696D000065720000F8
:103430002031000000000000F7940000FC9700001D
:10344000079500001B9800001395000036980000B7
:1034500021950000539800003095000071980000FD
:103460008D98000095980000AC980000B19800007D
:10347000CA980000D4980000019900000599000046
:1034800064960000179900003499000038990000F4
:103490006B9900007A99000068960000B8990000C6
:1034A000D2990000D6990000EB990000F199000034
:1034B000FD990000049A00000C9A0000139A000085
:1034C00000000000000000005F730000797300003E
:1034D000746500006D2E000072650000626F0000D0
:1034E0006F74000000520000656200006F6F000002
:1034F0007420000074680000652000006D69000001
:10350000637200006F6300006F6E00007472000051
:103510006F6C00006C650000720000005F730000BB
:1035200079730000746500006D2E00007365000063
:1035300074740000696E0000677300002E72000052
:1035400065610000640000005265000061640000D5
:1035500020610000207300006574000074690000A1
:103560006E67000000610000646400007265000086
:103570007373000000760000616C00007565000048
:10358000005F00007379000073740000656D000037
:103590002E73000065740000746900006E670000FF
:1035A000732E00007772000069740000650000004F
:1035B000577200006974000065200000612000005F
:1035C0007365000074740000696E000067000000FD
:1035D0005F73000079730000746500006D2E0000B9
:1035E0007365000074740000696E0000677300006A
:1035F0002E6600006C610000736800000057000038
:1036000072690000746500002074000068650000A5
:103610002073000065740000746900006E6700008C
:1036200073200000696E0000746F000020660000C7
:103630006C6100007368000000000000457200002B
:10364000726F0000723A000020730000616D00008C
:10365000706C000065730000206D00007573000041
:103660007420000062650000206900006E200000E8
:103670005B2D000031320000382C00003132000098
:10368000375D000020720000616E00006765000079
:10369000005F00006C650000647300002E73000082
:1036A0006574000000530000657400002074000081
:1036B00068650000206C000065640000006C00007C
:1036C0006564000000620000726900006768000025
:1036D000746E00006573000073000000736F0000DB
:1036E000756E0000642E000072650000636F0000BC
:1036F00072640000005300007461000072740000E6
:1037000020720000656300006F72000064690000B1
:103710006E670000206F000066200000724E0000FF
:103720002E77000061760000004E0000007300005C
:103730006F7500006E6400002E7000006C61000068
:1037400079000000537400006172000074200000D2
:10375000706C00006179000062610000636B000022
:10376000206F000066200000704E00002E770000E1
:1037700061760000007300006F7500006E64000049
:103780002E720000657000006C610000790000007E
:10379000537400006172000074200000706C00001F
:1037A0006179000062610000636B0000206F00001F
:1037B00066200000724E00002E7700006176000047
:1037C000007300006F7500006E6400002E6400003E
:1037D0007572000061740000696F00006E000000E7
:1037E00047690000766500002064000075720000E3
:1037F00061740000696F00006E200000696E0000B7
:10380000203100002F31000030730000206F0000D5
:1038100066200000724E00002E77000061760000E6
:10382000006400007572000061740000696F0000A0
:103830006E000000736F0000756E0000642E0000C3
:103840007379000073740000656D00000053000080
:103850007461000072740000207000006C61000050
:1038600079620000616300006B2000006F66000059
:103870002073000079730000746500006D20000063
:10388000736F0000756E0000642000004E000000A1
:103890006C650000647300002E6300006972000014
:1038A000636C000065000000536500007420000098
:1038B0006369000072630000756C000061720000B3
:1038C00020720000696E0000672000006C65000037
:1038D00064730000006C0000300000006C310000D8
:1038E000006C0000320000006C330000006C00002F
:1038F000340000006C350000006C00003600000051
:103900006C370000006C000065640000732E00003E
:10391000746F000070000000536500007420000008
:103920005247000042200000746F00007020000029
:103930006C65000064000000726500006400000017
:1039400067720000656500006E000000626C000098
:1039500075650000006C000065640000732E0000B7
:10396000626F0000747400006F6D00002E72000022
:10397000696700006874000000530000657400006F
:103980002052000047420000206200006F740000D7
:103990006F6D00002072000069670000687400000D
:1039A000206C000065640000006C0000656400008D
:1039B000732E0000626F0000747400006F6D0000D1
:1039C0002E6C000065660000740000005365000066
:1039D000742000005247000042200000626F000087
:1039E000746F00006D2000006C65000066740000BC
:1039F000206C000065640000006C0000656400003D
:103A0000732E000062750000747400006F6E000079
:103A10007300000053650000742000006275000010
:103A2000747400006F6E0000732000006C6500006D
:103A300064730000006C000065640000732E0000D9
:103A4000707200006F7800002E68000000530000C4
:103A500065740000206800006F720000697A000041
:103A60006F6E0000746100006C2000007072000036
:103A70006F780000696D0000697400007920000013
:103A80006C65000064730000006C00006564000059
:103A9000732E0000707200006F7800002E76000018
:103AA000005300006574000020760000657200007D
:103AB00074690000636100006C20000070720000F7
:103AC0006F780000696D00006974000079200000C3
:103AD0006C65000064730000006C00006564000009
:103AE000732E000072630000005300006574000034
:103AF00020720000632000006C650000640000007C
:103B00006C650000647300002E7300006F75000088
:103B10006E64000000530000657400002073000014
:103B20006F7500006E640000206C0000656400008A
:103B3000006C000065640000732E000074650000D6
:103B40006D70000065720000617400007572000005
:103B50006500000053650000742000006E740000D2
:103B6000632000006C65000064000000736F0000BB
:103B7000756E0000642E0000667200006571000022
:103B8000005000006C6100007920000066720000A7
:103B900065710000756500006E630000790000002B
:103BA000487A00000064000073000000736F00009A
:103BB000756E0000642E00007761000076650000DD
:103BC0000053000065740000207400006865000068
:103BD00020700000726900006D61000072790000C1
:103BE0002077000061760000652000006F6600000D
:103BF0002074000068650000207400006F6E0000F3
:103C000065200000676500006E65000072610000BD
:103C1000746F00007200000077610000766500009C
:103C200000700000726F0000782E0000636F0000CB
:103C30006D6D00002E6500006E610000626C00007A
:103C400065000000456E0000616200006C650000C8
:103C5000206F0000722000006469000073610000A2
:103C6000626C0000652000007468000065200000A0
:103C7000707200006F780000696D000069740000C8
:103C800079200000636F00006D6D0000756E00000C
:103C90006963000061740000696F00006E0000003D
:103CA000737400006174000065000000736400001C
:103CB0002E6F0000706500006E0000004F70000065
:103CC000656E00002061000020660000696C000045
:103CD000652000006F6E0000207400006865000021
:103CE0002053000044200000636100007264000063
:103CF000006E0000756D000062650000720000003B
:103D0000737400006174000075730000007300009C
:103D1000642E0000777200006974000065000000E6
:103D200057720000697400006520000064610000A3
:103D300074610000207400006F20000074680000AF
:103D4000652000006F700000656E00006564000073
:103D500020660000696C00006500000064610000DE
:103D60007461000000770000726900007474000044
:103D7000656E000000730000642E00007265000094
:103D800061640000005200006561000064200000D2
:103D9000646100007461000020660000726F000022
:103DA0006D20000074680000652000006F70000046
:103DB000656E00006564000020660000696C00000C
:103DC000650000007265000061640000007300007F
:103DD000642E000073650000656B00000053000056
:103DE000656500006B20000074680000652000001D
:103DF0006F700000656E00006564000020660000C2
:103E0000696C000065000000706F000073690000BD
:103E1000746900006F6E0000005F000072660000B1
:103E20002E6E00006F6400006569000064000000F1
:103E3000536500007420000057690000726500009F
:103E40006C65000073730000204E00006F6400007A
:103E50006520000049440000006E00006F6400000F
:103E60006549000044000000733000002E77000018
:103E70006176000000730000322E000077610000C0
:103E800076000000733300002E770000617600009A
:103E900000730000342E00007761000076000000FF
:103EA000733500002E77000061760000007300007B
:103EB000362E0000776100007600000073370000A6
:103EC0002E7700006176000000000000480D000021
:103ED0000D0000003011000007000000EC1300008E
:103EE000070000000019000007000000781E000015
:103EF000070000000000000000000000781E000025
:103F00000D0000000019000007000000EC13000085
:103F1000070000003011000007000000480D0000FD
:103F20000700000000000000000000004C0400003A
:103F300007000000980800000700000000000000D3
:103F400000000000E40C0000070000003011000039
:103F50000D000000C819000007000000000000006C
:103F6000000000009C27000002000000AB220000BF
:103F7000010000009D1C000002000000FB18000072
:103F8000020000002D32000001000000322D000070
:103F9000010000004628000002000000E8260000A2
:103FA00001000000BF22000002000000FB1800001A
:103FB00002000000FF32000001000000C6200000E7
:103FC00001000000762F0000020000002C2E0000EF
:103FD00001000000CE2C000001000000FD390000AF
:103FE000020000000000000000000000C8190000EE
:103FF00005000000BE0A00000400000000000000F0
:104000000000000030110000070000007C150000D7
:104010000700000000000000000000003011000058
:10402000070000007C15000007000000C819000010
:10403000070000000000000000000000222A00002D
:104040002B2C00003A3B00003C3D00003E3F0000AE
:104050005B5D00007C7F0000008000009A90000003
:10406000418E0000418F0000804500004545000062
:1040700049490000498E00008F9000009292000094
:104080004F9900004F55000055590000999A0000C3
:104090009B9C00009D9E00009F410000494F000036
:1040A00055A50000A5A60000A7A80000A9AA000029
:1040B000ABAC000021AE0000AFB00000B1B2000018
:1040C000B3B40000B5B60000B7B80000B9BA00003C
:1040D000BBBC0000BDBE0000BFC00000C1C20000EC
:1040E000C3C40000C5C60000C7C80000C9CA00009C
:1040F000CBCC0000CDCE0000CFD00000D1D200004C
:10410000D3D40000D5D60000D7D80000D9DA0000FB
:10411000DBDC0000DDDE0000DFE00000E1E20000AB
:10412000E3E40000E5E60000E7E80000E9EA00005B
:10413000EBEC0000EDEE0000EFF00000F1F200000B
:10414000F3F40000F5F60000F7F80000F9FA0000BB
:10415000FBFC0000FDFE0000FF0000002E2E000012
:104160002F2E00002E2F00006D6F00006C6F0000DE
:104170006C6500002F690000326300002F690000A9
:10418000326300005F70000072690000762E00004C
:10419000680000002E2E00002F2E00002E2F0000A1
:1041A0006D6F00006C6F00006C6500002F690000EF
:1041B000326300002F6D0000617300007465000021
:1041C000725F0000707200006F7400006F63000087
:1041D0006F6C00002E630000000000002E2E000017
:1041E0002F2E00002E2F00006D6F00006C6F00005E
:1041F0006C6500002F690000326300002F69000029
:10420000326300005F70000072690000762E0000CB
:10421000680000002E2E00002F2E00002E2F000020
:104220006D6F00006C6F00006C6500002F6900006E
:10423000326300002F6D00006173000074650000A0
:10424000722E0000630000002E2E00002F2E0000B2
:104250002E2F00006D6F00006C6F00006C65000079
:104260002F690000326300002F69000032630000F4
:104270005F70000072690000762E00006800000088
:104280002E2E00002F2E00002E2F00006D6F00003C
:104290006C6F00006C6500002F6900003263000045
:1042A0002F7300006C610000766500002E63000033
:1042B000000000002E2E00002F2E00002E2F0000E8
:1042C0006D6F00006C6F00006C6500002F740000C3
:1042D000696D0000657200002F740000696D0000B8
:1042E000657200002E630000000000000100000065
:1042F0000000000008000000000000004000000076
:104300000000000000010000000000005249000011
:104310004646000000000000000000005741000079
:1043200056450000666D000074200000100000007B
:10433000000000000100000001000000841E0000D9
:1043400000000000841E00000000000001000000CA
:1043500008000000646100007461000000000000BB
:104360000000000041720000677500006D650000EC
:104370006E7400002061000072720000617900001C
:1043800020730000697A0000652000006973000056
:10439000207400006F6F0000206C0000617200004C
:1043A00067650000202800003E330000322900002D
:1043B000000000005F4C00004F4700004455000023
:1043C0004D5000002E23000040210000005F00003F
:1043D00054450000535400004D4F0000442E00008F
:1043E0002340000021000000564D0000434F000014
:1043F000444500002E410000424F00000000000034
:104400002E2E00002F2E00002E2F00006D6F0000BA
:104410006C6F00006C6500002F6600006C6100008E
:10442000736800002F6600006C6100007368000074
:104430002E630000000000002E2E00002F2E000032
:104440002E2F00006D6F00006C6F00006C65000087
:104450002F690000326300002F6900003263000002
:104460005F70000072690000762E00006800000096
:104470005F54000045530000545300004400000006
:104480005F7000006F770000657200006F660000CB
:1044900066000000506F000077650000726F00003A
:1044A00066660000000000002E2E00002F2E000087
:1044B0002E2F00006D6F00006C6F00006C65000017
:1044C0002F75000061720000742F000075610000FC
:1044D000727400002E630000000000002E2E000009
:1044E0002F6D00006D61000037360000363000008F
:1044F0002E630000000000005F4200004C570000E7
:10450000484C0000564C00002E440000415400006E
:104510000000000010110000141200001300000041
:104520000116000017000000038000000F0F0000BC
:104530000F00000001017800833E2000830F50002F
:1045400003003C0083C12F00830F500001003D0099
:10455000030078000281B900481ADD004810DE002F
:104560000000720000000600EA874700889FBE0036
:104570008A9FBE008C9FBE008E1F780000057800C9
:104580002B87200081BF9F00A28720006D8620001E
:10459000AE8620000006EB000FB8970030027800CE
:1045A00080BF9F001BA2B900133220001100090038
:1045B000432AD800000278006A007E000002420010
:1045C0006087200060007E00F60320000683B900AB
:1045D0004FA0DE00060242008702480002003B00B6
:1045E000F403B0000580B000CA28DD004624DE00D8
:1045F00008847000080078006387200088317E00FE
:10460000631C210083014600A89998008802780065
:1046100005F0A7008502EA0084252000848F52005F
:10462000010034001209E800B012B0006425200037
:10463000840F500001003E000009EB00E0862000DE
:1046400060007E006A027E00000252001D034200EC
:10465000860E7800652C2100850F53000100340080
:10466000850E7800A5D32E009D8F120001003D001D
:10467000850E78000000E00008003A001E00E80007
:10468000000F780075022000850F500004003400F0
:1046900080022000000F780001003700000FEB00BF
:1046A000800220009E0F100004003A00800EEB00F4
:1046B000800DEB000002EB00060037006522B90018
:1046C0001D00780036002000110009000600D80007
:1046D000040240001B0242002500200011000900D6
:1046E0000502D80000027800840D78001032200006
:1046F000800F520001003400800D7800F0CD2F00B3
:104700009B0F100001003D00800D7800200020006C
:10471000920F10000E00340060C1B300D2B79F00AA
:10472000E3B79F00F898020000000000300020006E
:104730005FB19700000978001B007800240020007A
:10474000110009000400D800800D7800EFB1970037
:104750003B007800E09998000C86E8000281E800B0
:104760008D86E8000E87E800E40F56008AFF3A00C5
:104770009043800098D6020000000000A043800013
:10478000BED60200000000004F0778004F06BE00B2
:104790004F05BE004F04BE00AF00B1000000060090
:1047A000881F780000047800D18681001800780006
:1047B00060FF070070438800E186810018009000C8
:1047C0005CFF0700804388004F047800000006006B
:1047D0006628EF006828EF00800220005043880020
:1047E000604388006E28EF007028EF00000006008C
:1047F00021E3A90085A0A9000040060000000000F8
:1048000000000000000000000000000000000000A8
:104810000000000000000000000000000000000098
:104820000000000000000000000000000000000088
:104830000000000000000000000000000000000078
:1078000002003700315878000201E9000200E00070
:10781000FCFF3A0000000600020037000158780023
:107820000201E9000200E000FCFF3A00000006004F
:10783000889FBE008A9FBE008C9FBE008E1F78006E
:10784000000478000206BE0058159000E81590006C
:107850008000EB00820F5500838F5D0038003200FE
:10786000484090000004E00024003200EE022000B6
:107870000807470014C0B3000A01BE008E0078005C
:1078800018409000E6AA020000000000110020004D
:107890000000E0002A003A00404498005809900097
:1078A000E8099000780890008810900002004000DD
:1078B00083804800800F5500818F5D000F003100EC
:1078C000B84490000B00370058089000E80890007A
:1078D0000A0540008B85480014C0B3000A01BE00B1
:1078E0008E00780018409000E6AA02000000000018
:1078F0008944E900E1CF5400F3FF3E008000EB0033
:10790000E00F5600E08F5E000D003200E102200023
:107910008880400014C0B3000C01BE0018409000E5
:1079200076AA020000000000110020000000E00024
:1079300003003A005C1498006D1498008000EB007E
:10794000010078004F0778004F06BE004F05BE00CB
:107950004F04BE0000000600881F78000004780075
:10796000E10220008880400014C0B300184090005D
:1079700076AA0200000000008000780030C0B3004A
:107980000100E00045003A00D0222000080040003D
:107990001081FB004811DD00C022200008004000DB
:1079A0001080FB000201700020C0B30051A52A0026
:1079B000810F510039003A0078E29000C822DD00C2
:1079C0000400200068E090008080FB0000002000A0
:1079D000000272008182720048E090000080FB008B
:1079E0008000EB00000272008182720058E090007B
:1079F0004800DD008000EB0000027200818272000E
:107A00000580FB0080007800040078000001BE00C3
:107A100064142400450520000040EB00840F510051
:107A2000858F59001D00320038439100C833DD00B6
:107A300006002000284091008080FB00000020000C
:107A40000003730081837300084091000080FB00F5
:107A50008000EB00000373008183730018409100E5
:107A60004800DD008000EB00000373008183730099
:107A70000781FB0082017800060178000200BE0049
:107A800004006800858068000080700000F0A70096
:107A90000000EA000000EA004F00DE004F0478001A
:107AA00000000600920020000000E0000C00320000
:107AB0001004E0000A003200B0019000818F5100F4
:107AC00007003A00104090006AAA0200000000007F
:107AD0000001EB000008A30001003200320020008A
:107AE0000200780000000600889FBE008A1F780010
:107AF000000478006011B800080078004CFF07000F
:107B0000800478000900E00060003A0030C0B30053
:107B1000984F100054003A00584090000004E000D4
:107B2000510032006000B8005014980061149800B1
:107B3000EA02200008054500022020008000EB003A
:107B40000A00780034FF0700C0222000080040002F
:107B500051C5B30001487800D02220000800400041
:107B6000A1CAB3000148780020C5B300606C98003A
:107B7000706C98006F4040000074980011C4B3000E
:107B800011749800232120008881410022C7B3008E
:107B900082497800332120008881410082497800A1
:107BA00042212000080141000149780051212000B4
:107BB0008880400080487800780090008808900015
:107BC0006221200008014100004978007221200054
:107BD00008014100C801DE0003497800822120002D
:107BE00008014100400ADE00050020000449780039
:107BF00092212000080141004808DE000049780079
:107C000058009000E8009000A221200008014100E7
:107C100000497800B221200008014100C801DE00BF
:107C200003497800C221200008014100400ADE001B
:107C30000500200004497800D221200008014100FD
:107C40004808DE000049780014C0B300180990000D
:107C5000A80990008A00780018409000E6AA020067
:107C600000000000594498000001EB008040EB0048
:107C70001840900080AB02000000000000F0A70058
:107C80000000EA008004EA00CF4CDE000900780022
:107C90004F0578004F04BE0000000600F88747003B
:107CA000889FBE008A9FBE008C9FBE008E1F7800FA
:107CB00002447800100178009201FB000303B10038
:107CC000E98F510008003E0092429000A4C3B30027
:107CD00084CF520004003A000288E800B40020007B
:107CE0000300E000DA013A00BE4A80008E08780006
:107CF000C40020000E00E000D50132001E04E000A8
:107D00000D0032001E4090006AAA02000000000030
:107D10000080FB000008A30007003A000002EB000F
:107D20000804E000CA0132000028A300C8013200A4
:107D3000A4002000C6013700004FEB000040EB001C
:107D40001047980066A90200000000000080FB00B8
:107D5000340020000008A300BD013A000804E00040
:107D600003003200A40020000028A300B8013A005C
:107D70006011B8000E007800F7FE07006011B8002F
:107D8000C2B79F00D3B79F00E14F50001B003A00DD
:107D90000EF09300D40020000004E000AC0132009B
:107DA0007EF19300C811DD00020020006EF0930008
:107DB0008080FB00000020000001710081817100C3
:107DC0004EF093000080FB008000EB00000171008A
:107DD000818171005EF093004800DD008000EB00BF
:107DE0000002710081827100C4B79F00D5B79F0067
:107DF0000401BE000E007800D7FE0700140020002A
:107E0000E34F500092013200D40020000004E00053
:107E10008F013A00AE789000C808DD001E7890000F
:107E20000080FB008100700000202000808F500047
:107E300087013A005EC490004844DD004EC09000C7
:107E40000080FB00080470008004EB00E00F540089
:107E5000E08F5C0012003A005ED49000C844DD0060
:107E6000080020004ED090008080FB000000200021
:107E700000047400818474002ED090000080FB0008
:107E80008000EB0000047400818474003ED09000F8
:107E90004800DD008000EB00000474008184740061
:107EA000580F9800690F9800EE78900031479800BD
:107EB0000140E900D4002000E14F500064013E0081
:107EC000BE7B9000274798000704E0006001320065
:107ED0000780FB000001E900000061005C013A003E
:107EE0000EC390004833DD007E7890000080FB00D8
:107EF00006037000460798006F00630054013A00C3
:107F00002EC190004811DD001EC090000080FB00D3
:107F1000020070006105B800AAB79F00BBB79F00C0
:107F2000E00F5500E08F5D0014003A001ED0900075
:107F3000C802DD00040020000ED190008281FB0009
:107F40000200200002027200838272006EC990005B
:107F50000281FB008001EB0002027200838272004A
:107F60007EC990004811DD008001EB00020672001E
:107F700083867200ACB79F00BDB79F00DE7D900086
:107F8000C85DDD004E7890000080FB008B0570001E
:107F9000D40020002E0132000181FB008001EB00A3
:107FA0000800BE00F4B79F0086BF9F00E7B79F00A0
:107FB0009A040200000000000006BE006158B800EC
:107FC000E0AF9F00F1AF9F000FBB97004430DE0091
:107FD0006FA99700FFA9970002004000E0804900C8
:107FE0000005460081854E008AB79F009BB79F0021
:107FF0007FB29700EFB397002FB09700BFB0970004
:108000008A0F50008B8F5800110139000A00500070
:108010008B8058000781FB008001EB007A0402008E
:10802000000000007FB297000FBB9700E00F5000E8
:10803000E08F58000601320015C0B30053FF200046
:10804000830F5000E08F58000500360035C0B300A4
:10805000EB0F4000E08F580001003E0025C0B30048
:1080600062054000E08548003A0F98004B0F9800E9
:108070000FB097009FB097004FB19700DFB1970006
:108080000000410081804900301798004117980096
:108090006FA89700FFA89700020040008380480067
:1080A000A0B79F00B1B79F00700F9800011798000C
:1080B000E3CF52001C003A00D40020000600E0008C
:1080C000E3003A005ED99000C811DD0002002000F4
:1080D0004ED890008080FB0000002000000071005E
:1080E000818071002ED990000281FB008001EB009D
:1080F00002007000838070003ED990004811DD00BE
:108100008001EB000200700083807000101798005F
:10811000211798004258DD00CE50DE00810070002B
:108120004250DD001A003700D40020000600E000B5
:10813000C70032002FB19700BFB197000C0041007B
:108140008D8049001017980021179800E2CF520047
:1081500003003A000A0045008B804D000C003700F8
:1081600032002000030020000A00BE00E5B79F0097
:108170009A040200000000008100D1000080D300BA
:108180006105650000004500E0804800EFB29700FF
:10819000F01FB0000180B000C709DD004900DE001B
:1081A00000807100C908DE00D4002000800F540058
:1081B000818F5C00A60039000080EB008080EB001E
:1081C00070079800010F98006000B80050079800F1
:1081D00061079800E3CF520093003A000040EB00A3
:1081E000504798007ED990004811DD006ED890006D
:1081F0000080FB00020170004FB59700DFB59700CB
:108200000A014100E0814D00120F9800230F9800F1
:10821000E10220008E80400014C0B3001E40900098
:10822000E5B79F0076AA020000000000EFB29700B9
:108230000000E0007C003A00D02220000E00400048
:108240009080FB00C808DD00C02220000E00400026
:108250001080FB008100700050A52A00808F500024
:1082600071003A001E719000C811DD00020020006C
:108270000E7090008080FB00000020000001710063
:10828000818171006E6890000080FB008000EB002F
:1082900000017100818171007E6890004800DD005E
:1082A0008000EB0000017100818171002025250014
:1082B00011162400800F5100818F59005A003A0096
:1082C000502120000E0040001081FB008001EB00D7
:1082D000C811DD0002002000402120000E004000F7
:1082E0001080FB008000EB00C000DD0000002000DB
:1082F0000001710081817100202120000E004000EA
:108300001080FB008000EB00000171008181710092
:10831000302120000E0040001080FB004800DD00EE
:108320008000EB000001710081817100202727008F
:1083300011142600800F5100818F59003A003A0035
:10834000D02120000E0040001081FB008001EB00D6
:10835000C811DD0002002000C02120000E004000F6
:108360001080FB008000EB00C000DD00000020005A
:108370000000710081807100A22120000E014100E7
:108380001281FB008001EB0002007000838070000E
:10839000B22120000E0141001281FB004811DD00D6
:1083A0008001EB000200700083807000500798008D
:1083B00061079800902120000E0040001081FB0012
:1083C0008001EB00C811DD000200200080212000A8
:1083D0000E0040001080FB008000EB00C000DD00BC
:1083E00000002000000071008180710062212000E7
:1083F0000E0141001281FB008001EB0002007000C1
:1084000083807000722120000E0141001281FB0068
:108410004811DD008001EB000200700083807000D5
:1084200070079800010F9800054F78005809EC007C
:10843000C04A8800300798006000B80050179800C4
:10844000611798000040EB00404798000002EB00E5
:10845000040078004F0778004F06BE004F05BE00AD
:108460004F04BE008F01B10000000600000178003B
:10847000EB014100830F5100050032003282FB0006
:108480003180FB0000005200FAFF320000000600BD
:108490000000050080017800D1012A0051417800D8
:1084A0000200FB000204E00002003200830F5000D3
:1084B000FAFF3A0000000600E6874700889FBE00EA
:1084C0008A9FBE008C9FBE008E1F78000105780039
:1084D0009A007800810478008900780031417800A2
:1084E000F3C2B300834F5100FAFF3200C3C5B3009B
:1084F000834F5100F7FF320010047800B2002000D3
:108500000102200008007800C3FC07000901780080
:108510008006EB008000EB008E0020000046EB00A0
:1085200032407800804578008100E80003C2B30043
:10853000834F500034003600EFC14100834F50009C
:1085400031003200C3C5B300834F50002E0032000B
:10855000E3C2B300834F5000020032008E8F5600FA
:108560000A003900E80F570045003A00E3C2B300A3
:10857000834F500042003A00200020000066DD00DA
:108580008E067800BE002000E5FF37000004E00002
:1085900005003D003C40B3008085FB000B08B100A6
:1085A000D0022A00E0C57D000B80FB00F1B79F00E0
:1085B00082BF9F00B7FF0700FFB097000FB9970079
:1085C0000000E0002E003A00F0CBB30000C04500F0
:1085D000F94F500002003E000C14A00007003700C5
:1085E000F0C9B30000C04500F94F500003003E0041
:1085F0000C04A00000CEB30080C545000BF47E0043
:108600008D06E800C6FF3700018D44008040EB0076
:1086100002C2B300824F500001003E0041C0B300CF
:10862000600020000D00E0001600320050CEB300C4
:10863000984F100002003A0050C0B300004C780080
:10864000E80F570002003A00200020000066DD001D
:108650000C86FB0063006600E10F500001003A0049
:108660000144A0006C066600E40F560001003A00C9
:108670000134A000314C98000000EB0001003700ED
:10868000600020004F0778004F06BE004F05BE0077
:108690004F04BE006F00B10000000600881F780084
:1086A0000004780062005100E0805900380A900010
:1086B000C80A900062025200E0825A006011B800BD
:1086C000840F5000858F5800090031002841900028
:1086D0000281FB008001EB009A0402000000000010
:1086E00038119000C81190000001410081814900BB
:1086F0000200BE004F04780000000600889FBE0004
:108700008A9FBE008C9FBE008E1F780000047800F8
:108710000206BE001A0020000B002000E10F5100ED
:10872000E08F59007A00360038089000C8089000A1
:10873000800F5100818F590075003100184078007A
:10874000E24F50002F003200E34F5000450032004E
:108750000085EB008085EB00E14F50006C003A0093
:108760008204D100828444004949DE0078089000E8
:108770008810900000014100E08148000800780066
:108780002BFC07000085EB008085EB000000E0007B
:108790005F003A0009007800F01FB200E002B0006C
:1087A000684778008904E8004949DE0078089000AD
:1087B0008810900000014100E08148000800780026
:1087C0001BFC07000000E00051003A000E87FB0090
:1087D000F91FB200E902B00068C57C004855DD0011
:1087E0000A0577000C08A300020032004455DE00A1
:1087F00002003700FEFF20000E0565008005EB003B
:10880000430037004818DD004811DE000201700007
:10881000C819DE007808900088109000020140001E
:10882000838148000800780001FC07000085EB0008
:108830008085EB000000E00035003A000C064600A1
:10884000FC1FB200EC02B00068457E000A85FB0008
:108850000C0644001C4090004800DD000A05700032
:10886000E6FF37004918DD004711DE000201700005
:10887000C719DE00780890008810900002014000BF
:108880008381480008007800E9FB07000085EB00C1
:108890008085EB000000E0001D003A004266DD002C
:1088A000FC1FB200EC02B0000C004400204190001C
:1088B0000281FB008001EB00C012DD0004002000FB
:1088C00030419000C811DD0002002000020172005A
:1088D00083817200104090004800DD008000EB00B2
:1088E000000171008181710068407E000080FB0002
:1088F0008000EB000001710081817100F0FF200019
:108900000300600080007800020078000005BE00CF
:108910000A00BE004F0778004F06BE004F05BE009C
:108920004F04BE0000000600881F78000004780095
:108930000000EB002004980038019000C80190006E
:1089400020002000E10F5100E08F59003E0032006E
:1089500098007800310A9000C10A9000840F5100FD
:10896000858F590038003100E00F5100E08F590029
:1089700014003A0030C0B300914F100005003A00D7
:1089800011119000A1119000E00F5100E08F5900EB
:108990000C003A006011B80052049800630498007B
:1089A00041019000200020000200E000260032007B
:1089B00011119000A111900072049800030C98000E
:1089C00019003700214090000004E00010003A0038
:1089D0001800780049FF07000001BE00E10F4000C9
:1089E000E08F480015003200E10F5000E08F580082
:1089F0001400360018007800C0089000300890007D
:108A0000800F5100818F5900F1FF39000D003700B0
:108A10005204980063049800010078001FFF0700CB
:108A200070049800010C9800E302200018804100B7
:108A3000100C98000000EB0003003700100020002D
:108A400001003700200020004F04780000000600DD
:108A50000800FA00889FBE008A9FBE008C9FBE005F
:108A6000000478000205BE000406BE0020002000BD
:108A7000E10F5100E08F5900A50036003809900041
:108A8000C8099000820F5500838F5D00A00031005F
:108A900098407800E2CF500040003200E3CF500011
:108AA00052003200E1CF500097003A008A04D10012
:108AB0008A8444004949DE007808900088109000BC
:108AC00000014100E08148000800780058FB0700E1
:108AD0000000E0008C003A0089007800F11FB2002D
:108AE0006105650008003200E0022000010040003E
:108AF000684178006F4161000C80FB004400DD009C
:108B000000407100010037000C40780081004400F3
:108B1000E06898008904E80010C0B3004044980061
:108B20004949DE007808900088109000000141005B
:108B3000E0814800080078003DFB07000000E000ED
:108B400071003A00F91FB2000A00E000050032008F
:108B5000CC68DD004466DE000C867000C46EDE006A
:108B60000B003700E10220008980400068C17800D6
:108B700001CFB300814061004869DD004866DE0036
:108B80000C067100C86EDE006F4666000CC67000F1
:108B900089044400EC6C98005B003700485BDD0002
:108BA0004851DE0002017300C859DE0078089000C9
:108BB000881090000201400083814800080078007E
:108BC0001BFB07000000E0004F003A000A054500CB
:108BD000FA1FB2008A004400EC6898000105780092
:108BE0004866DE007C6D980047003700C95BDD00F9
:108BF0004751DE0002817300C759DE0078089000FB
:108C0000881090000201400083814800080078002D
:108C100007FB07000000E0003B003A004255DD0082
:108C2000FA1FB200E90220008A844400890044004F
:108C3000638240008182E8001581FB008001EB0027
:108C4000C013DD0006002000E6B79F00F7B79F00C5
:108C50001481FB008001EB00C813DD00060020003A
:108C600086BF9F0097BF9F006FB19700FFB197002D
:108C70000601710087817100E2B79F00F3B79F0082
:108C80005183FB004833DD006131B80082BF9F0093
:108C900093BF9F006FB39700FFB397000203730069
:108CA00083837300E6B79F00F7B79F0068C17C001D
:108CB0000283FB008003EB006FB19700FFB19700C8
:108CC000060371008783710002002F000701610015
:108CD0008001EB00C011DD00020020000C067100D5
:108CE0008D8671000A0544006C6D98004861DE00B5
:108CF000824878004069DE0003002000824A780044
:108D0000486EDE000C4A780011C0B3004144980060
:108D10004F06BE004F05BE004F04BE000080FA00A3
:108D2000000006000400FA00889FBE008A9FBE0073
:108D30008C1F7800000678000204BE00E00F51008E
:108D4000E08F59000B003A005C029000EC029000AA
:108D5000E00F5200E08F5A00120032003C089000F1
:108D6000CC089000800F5200818F5A000D00310016
:108D70000E0037000C00780060FE0700E10F500085
:108D8000E08F5800510036003C099000CC0990005B
:108D9000820F5000838F5800520039000802BE0035
:108DA0000200370014002000050020000405BE006A
:108DB00061054500E0854D003C089000CC0890001E
:108DC000800F5500818F5D0005003900E10F5200D2
:108DD000E08F5A00400036002A0020000B002000DF
:108DE0000A01BE000C00780094BF9F00A5BF9F0041
:108DF00042FE07001FBA9700AFBA9700E00F50007D
:108E0000E08F58000A003200E10F4000E08F480078
:108E100034003200E10F5000E08F58003100320082
:108E2000840F5500858F5D00E1FF3A002A0037006E
:108E3000F4FF2F00F5FF20000A01BE000C007800AF
:108E400003FF0700000178000200E00018003A006C
:108E5000E00F5400E08F5C00070032000A02BE0001
:108E60000801BE000C007800F9FE07000001780040
:108E70000200E0000E003A005A0698006B069800C7
:108E80007C0090008C089000E10F4000E08F4800CB
:108E90001300320061005000E08058007006980016
:108EA000010E980010C0B300504698000C00370027
:108EB0001000200001002000E10F510009003A00DD
:108EC0000080EB008080EB000600370010002000DF
:108ED00001002000030037006000B80001003700E7
:108EE0000A00BE004F0678004F05BE004F04BE00CA
:108EF0000080FA0000000600889FBE008A9FBE0026
:108F00008C9FBE008E1F78000004780081067800D8
:108F1000A80490008904E8004E0020007B00320085
:108F20007800900088089000E00F5000E08F580013
:108F3000760032006F8664006B003A0061004000EA
:108F4000E080480070049800010C980058019000DF
:108F5000E801900018007800E00F5100E08F590000
:108F600004003A0040009000808F54005E003900F9
:108F700066003700A04090008180FB008100E9007E
:108F8000444ADE008480600057003A00DBFD0700A1
:108F90000005BE002E002000E10F5000E08F5800B9
:108FA0005A0036001E002000E10F4000E08F48000C
:108FB000560032001800780030099000C009900077
:108FC000820F5500838F5D00400039004E00200065
:108FD0000D00E0004D00320058019000E8019000C3
:108FE00050FF07000005BE007E002000E00F50008B
:108FF000E08F5800450032002E002000E10F5000A5
:10900000E08F5800410032001E002000E10F4000B8
:10901000E08F48003D0032006011B8001800780071
:1090200003FA07000000E00038003A00E1022000E7
:1090300018804000022020008000EB00F6F90700B5
:10904000980678000A01BE000D00780093FD070025
:10905000D0169800E11698008046EB000F0037000C
:1090600011C0B300414098006011B80018007800AA
:10907000EFF907000000E00023003A001800780034
:1090800050119000E011900061014100E081490021
:1090900052109800631098008D46E8001800780080
:1090A000A040900081CF5600EDFF39000D81FB00FC
:1090B0008001EB0050129000E0129000020152007B
:1090C00083815A0052109800631098005A04980047
:1090D0006B0498000A01BE00180078006FFD0700BD
:1090E00070049800010C980029049800E102200007
:1090F000188040004566DD000C0640001C0C9800FE
:109100000007EB00010037001E0020000E00780071
:109110004F0778004F06BE004F05BE004F04BE004B
:1091200000000600889FBE00000478000800780058
:10913000FDFD0700800478000900E00016003A00F9
:10914000780190008809900018007800B8F90700AD
:10915000800478000900E0000F003A001808900031
:109160001004E0000B003200B04890000138A3006A
:1091700004003A00A8089000BCFC07000000E000D2
:10918000050032008000EB00080078005AFF07005D
:10919000E8FF370049002000090078004F04BE00B6
:1091A000000006000200FA00881F78000004780022
:1091B000E1BF9F0011407800F2C2B300824F50001F
:1091C00003003200C2C5B300824F500002003A00D3
:1091D0008100E800E1BF9F006000B8003004980003
:1091E000410498006FB89700F1C1B30090CF100010
:1091F00005003E0008007800CBFD07008000EB0072
:10920000110C98002A00370074004400E4805700D5
:10921000A9FC07000000E00025003A0008007800E3
:10922000C0FF0700A8089000B14890000000E000CF
:1092300005003200E40F50001D003A000128A30091
:109240001A0032001A0037000128A30018003A0063
:1092500018089000B04890000148A30013003200A5
:10926000505290004822DD00C05090008180FB00E9
:10927000048270008002EB00C022DD0004002000A8
:10928000305990004811DD00205890000080FB000C
:10929000020170008001EB00020072008380720006
:1092A0003004980041049800D7FF37005000200098
:1092B0004F0478000080FA0000000600889FBE007E
:1092C0008A1F7800000478000800780096FD0700E7
:1092D000800478000900E0001D003A007801900049
:1092E000880990001800780051F907008004780080
:1092F0000900E00016003A001808900010407800BD
:10930000FB4F4000160032000004E0001400320061
:109310001100200008007800F7FE0700ECFF37007E
:10932000180D9000020220008000EB000A00780077
:1093300039F90700B2002000A80890000A00780060
:109340002FF907001800780011C0B30041409800C1
:10935000090078004F0578004F04BE0000000600A9
:1093600078019000880990001800780030F9070013
:10937000800478000900E000F5FF3A00E8FF3700BC
:10938000881F78008A9FBE008C9FBE000004780072
:109390000205BE0020002000E10F5100E08F5900BF
:1093A0002F00360038099000C8099000820F550040
:1093B000838F5D0020003900290037000A01BE00BC
:1093C00008007800CDFC07000006BE00E00F50004A
:1093D000E08F58001D003200E10F5000E08F580070
:1093E0001C003200E10F4000E08F48001B003200FB
:1093F0006022B8000A01BE000800780094FD070052
:109400000000E00016003A00780090008808900004
:10941000E10F4000E08F480006003200610040008C
:10942000E080480070049800010C980010C0B30060
:10943000504498000C05BE0038089000C808900001
:10944000800F5500818F5D00DCFF39000000EB00CC
:10945000030037002000200001003700100020002A
:109460004F06BE004F05BE004F0478000000060006
:10947000B20020000004E00009003A00B04A800079
:109480000000E000010032000048EB000100E000B5
:10949000010032008048EB00B14A88000001EB0077
:1094A00002007800000006002800FA00889FBE0035
:1094B0008A1F78008C9FBE008004780081BF9F00C7
:1094C000800CEB007F4561007E416100A1FD2F0013
:1094D0008F80400070805700F0F90700E1FC2F00FA
:1094E0008F804000F1B79F000000E00004003A00C8
:1094F0008FB89700A0FD2F000F00400029FF070044
:109500006FB497000000E00003003A000800E0009C
:1095100001003A00600020008A80FB007C8160002E
:10952000550032000000E0000A003200E40F500055
:1095300003003A00A0FD2F000F0040005FFF07006E
:109540006FB497000000E00092003A000A34A000D7
:109550000700370038499000710161007000200059
:109560008C003A00800020000128A30089003A0006
:109570000A38A3004C0032001CB2020000000000B8
:10958000604C98004801DE00724C98004009DE00F3
:1095900003002000025498004808DE001054980090
:1095A0000040EB00304C9800405C9800505C980004
:1095B000605C9800705C980075004400F400440002
:1095C0007B014400FA0144001086FB004866DD0080
:1095D0001182FB000C0672008006EB00C066DD0005
:1095E0000C0020001282FB004822DD009382FB0069
:1095F000048272008002EB00040676008586760005
:109600008049EB000049EB008048EB000048EB008C
:109610005FA8970011C0B30041409800E00F5600CA
:10962000E08F5E002000320050129000E0129000A7
:109630000C01BE0094BF9F00A5BF9F0050FF070014
:109640001FBA9700AFBA97000000E00051003A003F
:109650005FA8970061065600E0865E005C009800F7
:109660006D0098000401BE0071F807000000E000E2
:109670000D003200470037000000E00045003A00CE
:10968000384990000281FB00400020000248A300FE
:1096900040003A000118A3000300320070002000CF
:1096A0000208A3003B003A000A38A3000100320080
:1096B0000A54A0005FA8970050119000E01190009C
:1096C000D20C9800E30C9800F80C9800CA4498005B
:1096D000585190004811DD00C85090008180FB0077
:1096E000028170008001EB00C011DD00020020004B
:1096F000385A90004822DD00A85890008180FB0075
:10970000048270008002EB00040171008581710009
:10971000F2049800830C9800785990000281FB00B5
:109720008001EB00C812DD000400200068599000A1
:109730008281FB000200200002017200838172001E
:10974000485A90000482FB008002EB000401710083
:1097500085817100585A90004822DD008002EB009C
:109760000401710085817100D2049800E30498001F
:109770006011B800B2049800C3049800B20C9800BD
:10978000C30C9800800C7800300090009004980082
:109790000000EB004F06BE004F0578004F04BE00EE
:1097A0000080FA0000000600E6874700889FBE00A0
:1097B0008A9FBE008C9FBE008E1F78000004780038
:1097C0000107780082047800F3B79F000300780057
:1097D0000008EB009800900018007800B1F807002E
:1097E0000000E000AF003A00C840900020002000D8
:1097F0000104E000AB003500700020000108A30068
:10980000A800320058019000E80190003800900054
:10981000C800900000005100818059006149B800E3
:10982000800F5100818F59009B0036008004780022
:109830009900370038019000C801900002007800BC
:10984000F01FB2007A003A0018007800C91BDE0051
:10985000C718DD004913DE00068370002042900027
:109860000442E9000642620013003A00E00F510092
:10987000E08F590003003A007800900088089000BB
:109880000500370018099000A809900084BF9F00C8
:109890009AFB07000FBA9700E10F5000E08F5800C5
:1098A0000F003600E10F4000E08F48005900320001
:1098B000100C9800210C9800980578001809900069
:1098C000A80990000B00780084BF9F0073FB07007D
:1098D0000FBA9700E00F5000E08F580005003A00E3
:1098E000484090000074A0004044980020002000F0
:1098F0006C0037000486FB008006EB000006460083
:1099000081864E00494DDE00220032002B4090003F
:109910000482FB00840045000080FB00808F500023
:1099200001003600040550000A4278000C01BE0018
:109930008E0078001B40900076AA02000000000014
:10994000C84090000000E00023003A000168A30036
:109950000E00320038089000C80890000C06500035
:109960008D8658006150B800800F5600818F5E00D0
:109970000600310001022000888040004960DD00BF
:1099800000004700022020009DF707004955DD0038
:109990003700370038099000C80990008C0F51003B
:1099A0008D8F590020003200484090000068A300CD
:1099B0000E003200010220008880400014C0B30075
:1099C0001B409000E6AA020000000000C840900082
:1099D0000000E000030032000174A0004144980040
:1099E0000F0037000164A1004144980001022000EB
:1099F000888040001800780014C0B3000C01BE003D
:109A00001040900076AA0200000000000000E00074
:109A100005003200484090000074A00040449800C7
:109A2000100020001F0037003C0C98004D0C9800DF
:109A300038009000C800900080007800F11FB2004C
:109A4000002020000100500009057800808F54009C
:109A500001003600000578000002200008004000E8
:109A6000810040000A0178000E00780064F70700CA
:109A70000A07470038009000C80090000000450029
:109A8000E080480030049800410498007FB09700BF
:109A9000100845008A8454000900E00065FF3A0080
:109AA0000000EB004F0778004F06BE004F05BE00D8
:109AB0004F04BE006F00B10000000600E6874700BB
:109AC000889FBE008A9FBE008C9FBE008E1F7800BC
:109AD000000478000107780082047800F3B79F0043
:109AE000030078000008EB00980090001800780050
:109AF000ECF707000000E000D0003A00C8409000FA
:109B0000200020000104E000CC003500700020009F
:109B10000118A300C900320058009000E80090002E
:109B200000814400E0814800800F5100818F59007E
:109B3000B30031008004EB00B10037003801900021
:109B4000C801900002007800F01FB20090003A00B7
:109B500098007800C91ADE004718DD004912DE00BF
:109B600004027000214090000040E90004406000C1
:109B700080F79F0020003A00E00F5100E08F59006D
:109B80000C003A007801900088099000E00F510025
:109B9000E08F59000F003A006011B8000100780012
:109BA00060FC07000001BE0070049800010C9800E2
:109BB0000500370018099000A809900001007800FE
:109BC00058FC07000001BE00E00F5100E08F590073
:109BD0008D00320048409000E10F5100E08F5900A5
:109BE00022003200E10F4100E08F490062003200A4
:109BF000120C9800230C9800484090000068A300C5
:109C00001100320001022000888040001800780016
:109C100014C0B30038099000C809900010409000AB
:109C2000E6AA020000000000C84090000000E0002A
:109C3000030032000174A000414498005000370036
:109C40000164A1004144980098057800180990002B
:109C5000A80990000B00780090FA0700E00F500070
:109C6000E08F580005003A00484090000074A000C2
:109C70004044980020002000700037000FF197004A
:109C80000286FB008006EB000006460081864E003F
:109C9000494DDE0022003200AB4090000280FB0004
:109CA000000145008180FB00810F5100010036005A
:109CB000008550000A4278000C01BE008E0078003A
:109CC0001B409000E6AA0200000000000000E00037
:109CD00028003A0038089000C80890000C06500090
:109CE0008D8658006150B800800F5600818F5E004D
:109CF00009003100C960DD0081004700000220003A
:109D00000800400002202000BDF6070048409000F7
:109D10000064A100404498004955DD002E00370042
:109D200038089000C80890008C0F50008D8F5800A4
:109D30001500320038019000C801900058009000D2
:109D4000E8009000800F5100818F59000E00310013
:109D5000010220008880400014C0B3000C01BE0046
:109D60001B40900076AA0200000000000000E00006
:109D700005003200484090000074A0004044980064
:109D8000100020002D0037003C0C98004D0C98006E
:109D900038009000C8009000F01FB20001202000A1
:109DA0008080500009057800818F54000100360042
:109DB00001057800010220008880400000804000FA
:109DC0000A0178008E0078008DF607004840900068
:109DD0000064A000404498000A0747003800900043
:109DE000C800900000004500E08048003004980062
:109DF000410498007FB09700100845008A84540001
:109E00000900E0004DFF3A0038009000C8009000C3
:109E100058019000E8019000820F5000838F580095
:109E200002003600500498006104980048409000F9
:109E30000054A000404498000000EB004F07780059
:109E40004F06BE004F05BE004F04BE006F00B100BC
:109E500000000600889FBE00000478009800900073
:109E6000180078000FF707000000E00041003A00FA
:109E7000C84090008180FB000158A3003D003200E3
:109E80000168A30010003200010220008880400019
:109E90001800780014C0B30038099000C809900079
:109EA00010409000E6AA0200000000008000780048
:109EB000100020000100E0002E003A004840900011
:109EC0000064A1004044980058099000E8099000FF
:109ED0001800780056F607000000E00025003A0060
:109EE000F80C90006B8044001054A00028489000AB
:109EF000C05C980038489000D05C980048489000BA
:109F0000E05C980058489000F05C98006848900029
:109F1000A05C980078489000B05C980008509000D1
:109F2000C054980018509000D05498001CB2020001
:109F300000000000E05498004801DE00F254980050
:109F40004009DE0003002000825C98004808DE0023
:109F5000905C9800484090000054A1004044980054
:109F60001800780011C0B300414098001800780034
:109F7000DDF607004F04BE0000000600881F7800D1
:109F80000004780008007800B2FF07000000E0003D
:109F900001003A00000C78004F0478000000060031
:109FA000EA874700889FBE008A9FBE008C9FBE0044
:109FB0008E1F7800000778000202BE009E0090000D
:109FC0001E007800F2B79F0085BF9F00B5F607001E
:109FD000D0B79F007FB297008FBA97000000E000D3
:109FE000F0003A004E4190000204E000EB00350022
:109FF0005E009000EE009000800F5200818F5A00AA
:10A00000030036000218A30001003A000002BE005F
:10A010003E009000CE0090006011B800320798001A
:10A02000430798006044B800E00F5200E08F5A00E8
:10A03000A00032001E037800264190000281FB0040
:10A040008001EB00491DDD00C715DE008B057500A2
:10A050004915DD00E00F5000E08F5800230032006A
:10A0600061045000E084580061005200E0805A0012
:10A070000A01BE00F4B79F0085BF9F00E6B79F00AE
:10A080007A040200000000000006BE000A01BE00C3
:10A090000800BE007A040200000000007FB29700B2
:10A0A0008FBA97006FB39700800F5600818F5E00C4
:10A0B0000E00390060001500E0801D000003640000
:10A0C0000181640082017800060178000200BE0070
:10A0D00030079800410798000002520081825A0020
:10A0E0001E099000AE099000170037007E01900015
:10A0F0008E099000E00F5100E08F590010003A00E7
:10A100006011B80006007800F4B79F0085BF9F007B
:10A1100004FB07000001BE007FB297008FBA9700D2
:10A12000E10F5000E08F580058003200E10F40006E
:10A13000E08F48008400320070079800010F9800FB
:10A14000120F9800230F98006044B800E00F5100F0
:10A15000E08F590057003200340037004E40900025
:10A160000018A3000B0032001E007800F4B79F0017
:10A1700085BF9F00EBFA07000001BE007FB2970089
:10A180008FBA9700E00F5000E08F580008003A00A7
:10A190002A0037001E007800F4B79F0085BF9F009B
:10A1A00056F907000001BE008FBA97007FB29700F2
:10A1B000E10F4100E08F490004003A004E4090005A
:10A1C0000074A0004047980051003700E10F510093
:10A1D000E08F5900060036001E007800C00890008D
:10A1E00030089000800F5100818F59000500390020
:10A1F0004E4090000074A0004047980022002000CC
:10A2000055003700120F9800230F98003E00900071
:10A21000CE0090000000450081804D00300798007E
:10A22000410798000A0252008B825A008A0F52009E
:10A230008B8F5A00C9FF3E00010037000A02BE00A2
:10A240003E009000CE0090000000420081804A0055
:10A25000300798004107980004007800F01FB20012
:10A260006044B800130032001E007800F4B79F006D
:10A2700085BF9F0009F907007FB297008FBA97004A
:10A28000E00F5000E08F580004003A004E4090006C
:10A290000074A0004047980040003700C92CDE0041
:10A2A0004729DD004924DE00080471000004440051
:10A2B00081844C003E009000F01FB2002A00320062
:10A2C0003E099000CE099000820F5400838F5C00FD
:10A2D000250032004E4090000068A30010003200BC
:10A2E000010220008E8040001E00780014C0B300E0
:10A2F00010409000E6AA020000000000CE4090004E
:10A300000000E000040032000174A0004147980002
:10A3100010002000220037000164A100414798008E
:10A32000010220008E8040001E00780014C0B3009F
:10A330000801BE001040900076AA02000000000054
:10A340000000E000060032004E4090000074A000C3
:10A350004047980012002000D2B79F00110037003C
:10A36000380F9800490F98003E009000CE009000F2
:10A370005E019000EE019000820F5000838F580024
:10A380000800360050079800610798004E40900082
:10A390000054A00040479800020037002000200031
:10A3A000D0B79F005FB097004F0778004F06BE0000
:10A3B0004F05BE004F04BE00AF00B1000000060014
:10A3C000FF4F500002003E0080407800060037003A
:10A3D0008040EB00F2C3B300824F500002003E0009
:10A3E00001C4B30080C050000140780000000600A6
:10A3F000889FBE008A1F7800800478005A48EC00CD
:10A400005AE8B70001C6B300814F50000100360082
:10A410005A68EF005AC8BF00804C780009047800E1
:10A4200002C2B30082404000016C780002C6B30053
:10A4300082CF50000100360002CC50000985E800B0
:10A440000044B000004D780001C6B300814F5000B9
:10A4500001003600014D500019407800D8FF070078
:10A46000804C780018407800D5FF0700004C780039
:10A470001A407800D2FF0700004D78004F057800A1
:10A480004F04BE0000000600800078000000EB00D2
:10A49000E48F50000A003200E88F500008003200BC
:10A4A000100020000100E00005003A00704280002A
:10A4B00000F0A7000000EA000000EA004F00DE0004
:10A4C00000000600889FBE000004BE00090444008E
:10A4D0000100370069045400E80F5400FDFF3C0000
:10A4E00001003700690444000800E000FDFF35006A
:10A4F00008007800E4FF07000000E000F3FF3200EE
:10A50000080078004F04BE00000006008000EB0049
:10A51000E80F5000E08F58002B003E000060010063
:10A5200008003700090037000B0037000E00370025
:10A5300011003700130037001500370018003700EE
:10A540001C0037000041EB000C0037000041EB001D
:10A5500001C2B300140037000041EB0001C2B30098
:10A5600001407800110037000041EB008240780084
:10A5700000C2B3000D00370002C2B3008240780071
:10A58000F7FF370002C2B3008040EB00F4FF370052
:10A5900002C2B300824078000040EB0003003700A5
:10A5A00002C2B3008040EB000240780018C70400EC
:10A5B0000000000052C0B300F1C0B30000C2B300FD
:10A5C00018C702000000000000000600889FBE00BF
:10A5D0000004780008007800CCFF07008004EB003E
:10A5E000E80F5400E08F5C003D003E000860010071
:10A5F0000800370009003700360037000D0037002B
:10A6000034003700170037001F0037002F003700D5
:10A6100030003700000021002F00370040002000EC
:10A620007A740200000000008CB1020000000000FB
:10A630002B003700001020007A7402000000000098
:10A64000400020007A740200000000000041EB008E
:10A6500082407800F0C0B30018C70200000000007C
:10A660001F003700400020007A7402000000000044
:10A67000000120007A74020000000000600F20003A
:10A68000A094880016003700C0272A00C4B4020036
:10A69000000000000000E0000E003A002100200051
:10A6A000408D200052B50200000000002100200073
:10A6B000608D200052B50200000000000000EB0099
:10A6C000C4B4020000000000020037005228EF006E
:10A6D0005428EF00400020007A74020000000000BF
:10A6E0004F04BE00000006000400FA00889FBE0070
:10A6F000000478000001EB006000B800BCC7020055
:10A70000000000008043EB00074378008742780098
:10A710000742780087417800074178008740780039
:10A7200007407800C8C60200000000008040EB002F
:10A7300000C1B300E8C50200000000008040EB004B
:10A7400010C1B300E8C50200000000008040EB002B
:10A7500040C1B300E8C50200000000008040EB00EB
:10A7600050C1B300E8C50200000000008040EB00CB
:10A7700020C1B300E8C50200000000008040EB00EB
:10A7800030C1B300E8C50200000000008040EB00CB
:10A7900060C1B300E8C50200000000008040EB008B
:10A7A00070C1B300E8C50200000000008040EB006B
:10A7B00001407800E8C50200000000008040EB0086
:10A7C00010C0B300E8C50200000000008004EB00E8
:10A7D000E80F5400E08F5C0054003E000860010068
:10A7E00008003700090037000E0037000A00370064
:10A7F0004B0037000F0037002200370044003700BD
:10A8000047003700000021004600370096B10200E3
:10A8100000000000030037000010200092740200C6
:10A8200000000000400020009274020000000000C0
:10A830000F0037004000200092740200000000006A
:10A840000001200092740200000000008040EB0034
:10A85000E0C1B300E8C5020000000000402921006B
:10A860000008EB00F1BF2F0020932000108860004B
:10A87000202721000008EB000080E8000008EB0022
:10A880002A003700C0272A00C4B4020000000000DC
:10A890000000E0001E003A00C0BF9F00D0BF9F0034
:10A8A000210020006880570052B50200000000001F
:10A8B000210020006680570052B502000000000011
:10A8C0004FB89700D408E30003003A005FB8970040
:10A8D000D608E3000B0032006000B80012B5020099
:10A8E0000000000021002000408D200098B50200EB
:10A8F0000000000021002000608D200098B50200BB
:10A90000000000000000EB00C4B4020000000000E2
:10A91000202721000008EB000080E8000008EB0081
:10A920004000200092740200000000004F04BE00AE
:10A930000080FA00000006006448EC0080407800C7
:10A9400042862000014978000100FB000104E0007C
:10A950000700340082C2B30082CF500008003400E8
:10A9600001C8B300428620000149780000000600BB
:10A9700042002000110009000200D8000000EA0097
:10A98000000006000400FA00889FBE008A9FBE00F7
:10A99000C8918000812321000005EB0010002000F9
:10A9A00051017800880F5100020034000005780042
:10A9B000020478000000E800E50F5000F8FF3A00BC
:10A9C000C446800062051500220020001100090025
:10A9D0000202D8008000FD0001D5B900C9DA2000CC
:10A9E000890F54000A00340001FA2000810F54003E
:10A9F00005003C0088845400110009008204D8003E
:10AA0000800478000F0037008404EA000D0037004E
:10AA100071BB2000810F540000013C00813EB10059
:10AA2000810F54000900340089C12F00888444003C
:10AA300092FF2F00110009008204D80080047800E2
:10AA4000C912B000848F54000100340084047800DF
:10AA50008400EA00818F540001003D0081047800E9
:10AA6000311F2000810F54000A003C005848E200CA
:10AA70000300320094938800A493880009003700F3
:10AA8000202721000008EB000080E8000008EB0010
:10AA900004003700402721000A8844000080E900B4
:10AAA0000A8854005848E200140034005948E20073
:10AAB000120032006C8057004DFE07006FF19700C6
:10AAC000DFF097004FF0970018C702000000000069
:10AAD0005FF19700CFF097006FF0970050C702002A
:10AAE000000000004FF19700EFF097005FF0970033
:10AAF00034C7020000000000060037008EFF070088
:10AB00000001EB00800078000000EB00BCC70200F1
:10AB1000000000005848E2001600320057C8BF008D
:10AB2000DA48B40057E8B700FE4F50000200360084
:10AB3000DAE8EF00040037000004E00002003A0009
:10AB400010C0B300DAE8B7007585200095427800A0
:10AB50008580FB004309DE00C408DE0081437800E5
:10AB60000243780004C2B300854178000040EB0046
:10AB7000080037008043EB000743780005C2B300AC
:10AB800005427800854178000741780087407800C9
:10AB900007407800C8C602000000000030FC220018
:10ABA0009080FB008100EA00CF08DE000000EB008F
:10ABB0000104E000040032009AC8BF000080FB00DE
:10ABC0000000E9004F00DE00A28920000149780062
:10ABD0000000E00007003200C14680002103B00001
:10ABE000C1468800401F2000808F500001003400C3
:10ABF000C046880000FC22009080FB008100EA0033
:10AC0000CF08DE000000EB000104E0000400320089
:10AC100099C8BF000080FB000000E9004F00DE0083
:10AC200092892000014978000000E000070032000E
:10AC3000C14680002103B100C146880040ED2F00CD
:10AC4000808F500001003D00C046880011C0B30055
:10AC5000401F2000800F540003003C008040EB00A8
:10AC60000000EB000400370098C8BF000080FB0024
:10AC70000000E9004F00DE008289200001497800D1
:10AC80000000E00003003200600020000EE102003E
:10AC9000000000000A00E0000D003A000900E0009A
:10ACA00060003A005948E2005E003A00401F200070
:10ACB000800F54005B00340010C0B30059E8B700A7
:10ACC000700020000EE102000000000001003700CB
:10ACD0005968EF001008200071938000808F5000A9
:10ACE0000300340081938000808F50000A003C00F4
:10ACF000202721000008EB000080E8000008EB009E
:10AD000001C2B30080C0B300E8C50200000000002B
:10AD100001C2B300050037008040EB0080C0B300E3
:10AD2000E8C50200000000008040EB00B0C0B300A6
:10AD3000E8C502000000000058C8BF000200320051
:10AD40000040E90058E8B70032E9AB0039003200B2
:10AD5000F1F72F0020932000108860005868EF0062
:10AD600042252100A19280000009EB000004EB00C5
:10AD700010002000D2017800818F510002003400C1
:10AD800000047800830078000009EB000000E80070
:10AD9000E70F5000F7FF3A0080BB2000808F500083
:10ADA0002400340028938800202621001000E900A8
:10ADB000E20F50001F003E00080078000010A200C3
:10ADC00000F0A7000000EA000000E9004F00DE00EC
:10ADD0008000EB000004E0000500320071892000D3
:10ADE000914078008180FB008100E900CF08DE00FF
:10ADF00097E8B7000100E000030032007000200077
:10AE00000EE1020000000000E20F540009003A00C9
:10AE100060C0B30058E8B700060037008004EB00BC
:10AE200008FF3700301F2000800F5400A8FF3400B7
:10AE3000A8FF37004F05BE004F04BE000080FA0097
:10AE4000000006000C00FA00889FBE008A9FBE002A
:10AE50008C9FBE0078805700030009000018EB00AB
:10AE6000B5FE07000041EB008040780018C70200E3
:10AE7000000000005BC8EC005BE8B7008080FB00CE
:10AE8000C508DE0002C2B300F881570082F17800E5
:10AE90007F4060008101E900E781610000415100CD
:10AEA00002437800F882570086F279008100E800BA
:10AEB000E78060000041780082F27800FFEB9700A5
:10AEC0006FEB9700DFEA97004FEA9700BFE9970022
:10AED0002FE997009FE897000FE89700C8C6020087
:10AEE0000000000030FC22009080FB008100EA009E
:10AEF000CF08DE000000EB000104E0000400320097
:10AF00009CC8BF000080FB000000E9004F00DE008D
:10AF1000C3892000814978000000E000070032006A
:10AF2000E14680002103B000E1468800401F200078
:10AF3000808F500001003400E046880000FC2200B1
:10AF40009080FB008100EA00CF08DE000000EB00EB
:10AF50000104E000040032009BC8BF000080FB0039
:10AF60000000E9004F00DE00B5892000814A78002A
:10AF70000000E00007003200E14680002103B1003C
:10AF8000E146880040ED2F00808F500001003D0019
:10AF9000E0468800E84680000800E00055003500E3
:10AFA000C3918000D1918000F091800002928000D6
:10AFB000611AB9004F93DE000402410085024B0084
:10AFC000018640004FE3DE000402460085024B008C
:10AFD000EC9180006366B9004FE3DE000406460092
:10AFE00085064B0000024000CFA2DE000C064200A6
:10AFF0008D864A00D6FF2F00068BB900C1FF2F00B7
:10B00000019AB900CFA2DE00CFB0DE0004024300F7
:10B01000858248006300B900CF81DE000400400053
:10B02000858049004212DD004FA3DE00000242008D
:10B0300081024B000400460085804E006145B90046
:10B040000A01BE0084BF9F0095BF9F009A040200C2
:10B05000000000000001BE00097D20001100090071
:10B060004919D800800078002027210001085400E9
:10B070000FBA97009FBA97000400560085805E00C3
:10B080000A01BE009A040200000000000001BE0098
:10B09000110009004919D8008004780009045400FF
:10B0A000A893880080DA2F0091938000808F500051
:10B0B00001003D0090938800800F540002003D0085
:10B0C00080DA2F00A09388008025200091938000D3
:10B0D000808F50000100340090938800802520006C
:10B0E000A1938000808F500011003400A09388004D
:10B0F0000F003700209280000882B90042ED2F0037
:10B1000011000900422AD800800078002027210081
:10B1100008884000109280000882B90011000900E0
:10B12000422AD80000017800402721000808410089
:10B130001008200071938000808F500003003400BD
:10B1400081938000808F50000A003C00202721005E
:10B150000008EB000080E8000008EB0001C2B3002B
:10B1600080C0B300E8C502000000000001C2B300C7
:10B17000050037008040EB0080C0B300E8C5020046
:10B18000000000008040EB00B0C0B300E8C5020042
:10B19000000000004F06BE004F05BE004F04BE0079
:10B1A0000080FA0000000600889FBE008A9FBE0053
:10B1B000F046800080004000808040003094800095
:10B1C00000F0A7000000EA0080804000409480006A
:10B1D00000F0A7000000EA000080400051948000C9
:10B1E00001F0A7008100EA00010040004200DE00FB
:10B1F000F046880018002000ED0F500001003600D6
:10B200000004EB0011C0B300EE0F500003003E003D
:10B210008040EB000000EB00040037009FC8BF0037
:10B220000080FB000000E9004F00DE00F2892000F2
:10B23000014978000000E000050032000041EB0009
:10B2400082407800F0C0B30018C702000000000080
:10B25000F0468000ED0F500011003E005C08EC004D
:10B26000E0428800E50F500007003400EA0F50006C
:10B2700001003A005C28EF000041EB0082407800BA
:10B2800000C2B300030037000041EB0082407800A9
:10B290000240780018C702000000000005003700D7
:10B2A000A5FD07000001EB008000EB00BCC7020019
:10B2B00000000000E09480000000E0000500320083
:10B2C000C02921000008EB00500020000EE1020020
:10B2D00000000000DA918000803E2000800F5500C1
:10B2E00019003400E2918000800F510016003400F4
:10B2F000F2918000800F5100130034001292800000
:10B30000800F510003003C0022928000800F51000A
:10B310000D0034002008200072938000800F51003F
:10B320000900340082938000800F51000600340031
:10B33000202721000008EB000080E8000008EB0057
:10B34000180020004E003700C5918000803E20008C
:10B35000F4918000808F52000A003C00800F55005D
:10B3600008003C00E2918000800F510005003C0085
:10B37000800F520003003C0002928000800F5100B9
:10B380002D0034000B9280004300200011000900C2
:10B390000305D80080047800520020001100090045
:10B3A0008202D8000003780086844400E691800081
:10B3B000110009000303D8008003780007834400CC
:10B3C000110009000302D8008003780087014300C0
:10B3D000110009008205D8008003780087814100B0
:10B3E000110009000205D800000578006700200060
:10B3F000110009008702D80080027800050145008D
:10B40000A6FF2F00110009008605D80000014100A9
:10B41000B6FF2F00110009000602D800000241000B
:10B4200084804100202721000108EA000080E80014
:10B43000030852001200370013928000249280000B
:10B44000808F510002003C00800F52000800340041
:10B4500042002000110009008201D800909388006A
:10B46000110009000202D800A093880004003700F0
:10B47000202721000008EB000080E8000008EB0016
:10B480001008200071938000808F5000030034006A
:10B4900081938000808F50000D003C002027210008
:10B4A0000008EB000080E8000008EB000041EB0022
:10B4B0008240780000C2B30034C7020000000000E0
:10B4C0000041EB008240780000C2B3000800370062
:10B4D0000041EB00824078000240780034C702004F
:10B4E000000000000041EB0082407800024078003C
:10B4F00050C702000000000080DA2F009193800006
:10B50000808F500001003D009093880080DA2F006A
:10B51000A1938000808F500001003D00A09388001F
:10B520008025200091938000808F5000010034001E
:10B530009093880080252000A1938000808F500088
:10B5400001003400A0938800884078000000EB00E0
:10B550000804E000040032009EC8BF000080FB0029
:10B560000000E9004F00DE00E28920000149780078
:10B570000000E000030032004000200012E1020061
:10B58000000000000804A2000000EB000804E00036
:10B59000040032009DC8BF000080FB000000E900ED
:10B5A0004F00DE00D1892000884878000000E000CC
:10B5B000030032000080EB000EE1020000000000FA
:10B5C0004F05BE004F04BE00000006000400FA0054
:10B5D0003349AB0041003200F1BF2F00209320001F
:10B5E0001088600011862000914078000104E0007E
:10B5F0000C003A006268EF0010C0B30061E8B700C9
:10B600008043EB00074378008742780007427800C8
:10B610008741780007417800874078007F404000EC
:10B620001400370062C8BF00E1CF500014003A0098
:10B63000E24F500029003400FD4F500027003C002D
:10B6400021C0B30012862000014978000040E800C4
:10B650005EE8B70007C2B3000043EB008642780003
:10B6600006427800864178000641780087407800DD
:10B6700007407800C8C6020000000000170037002D
:10B68000E2CF500015003A005E48E30013003D0091
:10B6900071C2B300814F500010003C0030C0B300B5
:10B6A00061E8B70007C2B300074378008042EB00AF
:10B6B000054278008541780007417800874078008E
:10B6C00007407800C8C6020000000000700020009B
:10B6D0000EE10200000000006068EF0062C8BF00D9
:10B6E00031C6B300814F500002003C000040E8002A
:10B6F00062E8B70020C3B3006248E3000B003400E7
:10B700006168EF008043EB000743780087427800D0
:10B710000742780087417800074178008740780029
:10B7200007407800C8C602000000000062C8BF00E1
:10B73000E54F500015003A005FC8BF00E14F5000D0
:10B7400009003A0061C8BF00E14F50000F003A0005
:10B7500020C0B3005FE8B700000520009093880088
:10B7600000FB2F0008003700E24F500007003A00AE
:10B7700061C8BF00E14F500004003A005FE8B70025
:10B780000005200090938800A093880062C8BF0045
:10B79000FE4F500012003A0061C8BF005F48E2004F
:10B7A00008003A00E24F500006003A0010C0B30013
:10B7B0005FE8B7000005200090938800A093880000
:10B7C00007003700E24F500005003A005F68EF00C5
:10B7D000202721000008EB000080E8000008EB00B3
:10B7E00080C2B3006248E3000A003A0061C8BF00AB
:10B7F000E34F500007003A0010C0B3005FE8B70005
:10B800000105200091938800412721008008EB006A
:10B8100060E8B7001008200071938000808F50000E
:10B820000300340081938000808F50000D003C00A5
:10B83000202721000008EB000080E8000008EB0052
:10B840000041EB008240780000C2B30034C7020020
:10B85000000000000041EB008240780000C2B3000D
:10B86000080037000041EB00824078000240780079
:10B8700034C70200000000000041EB008240780065
:10B880000240780050C70200000000006048E2005B
:10B890002200320064805700D5FA07006FF9970044
:10B8A000DFF897004FF8970018C70200000000006B
:10B8B0005FF99700CFF897006FF8970050C7020024
:10B8C000000000004FF99700EFF897005FF897002D
:10B8D00034C70200000000006048EC0060E8B700D8
:10B8E000F1C7B300814F500012003A006068EF00CA
:10B8F0000041EB00824078000240780050C702000F
:10B90000000000000041EB00824078000240780017
:10B9100034C70200000000000600370006FC0700E4
:10B92000004178008040EB000140780018C7020019
:10B93000000000000080FA0000000600FEFB070087
:10B9400000417800804078000040EB0018C70200FA
:10B95000000000000040EB0001FC22001104E000A8
:10B960000D003200E38040001104E0000A003200C4
:10B97000E02621008080E8009100780010804000DF
:10B9800022002000110009000200D8006009B00068
:10B99000A046880010C0B30011FC22001104E00092
:10B9A00013003200E38040001104E0001000320078
:10B9B000E02621008080E80091007800108040009F
:10B9C00022002000110009000200D800B0468800C3
:10B9D00051092000810F500002003E00800C200021
:10B9E000B0468800A0F62F00D628B4000200370029
:10B9F0000004E0000F0032008043EB0007437800B2
:10BA00008742780007427800874178000741780034
:10BA10008740780007407800C8C602000000000098
:10BA2000202721000008EB000080E8000008EB0060
:10BA30000000060071938000A2468000828F5000B3
:10BA400002003100204723000048EB00B046800090
:10BA5000808F50000300360013C0B300214723003D
:10BA60008348780081938000828F5000020031006B
:10BA7000324723000049EB00808F5000030036005E
:10BA800011C0B3003047230001487800204723004D
:10BA900010407800314723000004E00004003A0021
:10BAA0001104E00006003A006368EF001700370059
:10BAB000E14F500002003A001104E0001200320091
:10BAC0003147230012C0B300914F110004003A0027
:10BAD0000004E00002003A0063E8EF000B003700CA
:10BAE00063C8BF004240A9000200340020C0B30078
:10BAF000050037000004E00002003200E0CFB30090
:10BB000001003700A0C0B30063E8B70063C8BF00FE
:10BB10000C003A00C012200090938800A093880087
:10BB20008043EB00074378008742780004C2B300EB
:10BB3000874178000741780087407800044078000A
:10BB400036003700E14F50000D003A00C0122000CF
:10BB500090938800402721000008EB008043EB0011
:10BB600007437800874278000742780003C2B30099
:10BB700007417800834078000740780027003700AD
:10BB8000E14F400009003A00202721000008EB00A7
:10BB9000C0122000A093880007C2B3000043EB004E
:10BBA00087427800064278000A003700E24F4000E2
:10BBB0000C003A0040ED2F0090938800C012200046
:10BBC000A09388008043EB0006C2B3008742780050
:10BBD000074278008441780004417800844078006E
:10BBE0000D003700E24F50000E003A00C012200056
:10BBF0009093880040ED2F00A09388008043EB00D5
:10BC00000743780087427800074278008741780030
:10BC100002C2B3008740780001407800C8C6040023
:10BC200000000000EA4F500004003A00C01220005B
:10BC30009093880040ED2F00A0938800000006003C
:10BC40003DFB0700004178008040EB0018C7020070
:10BC50000000000010FC22009080FB008100EA0040
:10BC6000CF08DE000000EB000104E0000400320019
:10BC7000A5C8BF000080FB000000E9004F00DE0007
:10BC8000528A2000014978000000E00002003200E2
:10BC9000A0F62F00A042880040FC22009080FB000C
:10BCA0008100EA00CF08DE000000EB000104E000A4
:10BCB00004003200A4C8BF000080FB000000E900BF
:10BCC0004F00DE00428A2000014978000000E000B9
:10BCD0000200320060092000A042880000FC22001F
:10BCE0009080FB008100EA00CF08DE000000EB003E
:10BCF0000104E00004003200A3C8BF000080FB0084
:10BD00000000E9004F00DE00328A2000014978007F
:10BD10000000E000060032005408E2000200320099
:10BD20005428EF0002003700A0F62F005228B4007C
:10BD300030FC22009080FB008100EA00CF08DE008A
:10BD40000000EB000104E00004003200A2C8BF00C4
:10BD50000080FB000000E9004F00DE00228A200086
:10BD6000014978000000E000060032005408E200BB
:10BD7000020032005428EF00020037006009200062
:10BD80005228B4008000EB0000FC22001004E00008
:10BD900004003200630040009080FB008100EA0054
:10BDA000CF08DE000000EB000104E00004003200D8
:10BDB000A1C8BF000080FB000000E9004F00DE00CA
:10BDC000128A2000014978000000E00001003200E2
:10BDD0005228EF008000EB0040FC22001004E0003D
:10BDE00004003200630050009080FB008100EA00F4
:10BDF000CF08DE000000EB000104E0000400320088
:10BE0000A0C8BF000080FB000000E9004F00DE007A
:10BE1000028A2000014978000000E00001003200A1
:10BE20005428EF00809480000000E00047003200BA
:10BE300001022000810F50003000320014003C004D
:10BE4000E60F50003A00320006003C00E40F5000BC
:10BE50002E00320039003C00E20F500039003A0059
:10BE600026003700ED0F50003400320003003C0084
:10BE7000E80F500033003A0026003700F00F500062
:10BE80002B003200F10F50002E003A001F00370047
:10BE900001052000810F50001800320008003C000E
:10BEA000E3805000810F5000180032008100E8004C
:10BEB000810F50001E0032001102200005003700E3
:10BEC00051052000810F50001000320004003C009A
:10BED000E4805000810F50001A003A000D00370036
:10BEE00061052000810F5000110032008100E80040
:10BEF000810F500013003A00100037006009200045
:10BF00005408E2000800320005003700A0F62F00B8
:10BF100008003700A0F62F005408E20002003200AB
:10BF20005428EF00070037005228B40005003700FE
:10BF300060092000A0428800020037005428EF006A
:10BF40005228EF00002921000008EB008025200086
:10BF50005208E300010034009042880080DA2F008C
:10BF60005208E30001003D00904288008025200037
:10BF70005408E30001003400A042880080DA2F005A
:10BF80005408E30001003D00A04288009142800077
:10BF9000A042800022272100010940000281E80020
:10BFA0000089500000000600001020007A74020092
:10BFB00000000000002020007A7402000000000051
:10BFC000000120007A740200000000004000200000
:10BFD0007A74020000000000100020007A74020051
:10BFE00000000000000120007A740400000000003E
:10BFF0005648EC0056E8B70041C6B300814F5000E8
:10C000002100360050C6B30056E8B70020FC2200DD
:10C010009080FB008100EA00CF08DE000000EB000A
:10C020000104E0000400320096C8BF000080FB005D
:10C030000000E9004F00DE0062892000014978001D
:10C040000000E0001000320060428000A6F9070006
:10C05000804280000000E00002003A000040210021
:10C06000140037004C08E30004003A000000EB0025
:10C0700056F907004C28EF000300370053F907007A
:10C080005008F8004C08F900D0F40200000000004D
:10C090000000E00004003A007AC302000000000043
:10C0A0000048A30006003200604280008EF90700BD
:10C0B000004020009274020000000000BAFF370028
:10C0C000604280008000EB00E70F5000E08F5800D6
:10C0D0005D003E000060010007003700540037009B
:10C0E0005400370054003700570037005300370022
:10C0F000530037005300370000FC22009080FB0003
:10C100008100EA00CF08DE000000EB000104E0003F
:10C110000400320095C8BF000080FB000000E90069
:10C120004F00DE0052892000014978000000E00045
:10C13000040032008080EB0080428000E1F80700BC
:10C140008042880010FC22009080FB008100EA0001
:10C15000CF08DE000000EB000104E0000400320024
:10C1600094C8BF000080FB000000E9004F00DE0023
:10C1700042892000014978000000E00004003200FC
:10C180008080EB0080428000CEF80700804288006B
:10C1900030FC22009080FB008100EA00CF08DE0026
:10C1A0000000EB000104E0000400320093C8BF006F
:10C1B0000080FB000000E9004F00DE003289200013
:10C1C000014978000000E000040032001100200066
:10C1D00080428000BBF807008042880040FC2200BB
:10C1E0009080FB008100EA00CF08DE000000EB0039
:10C1F0000104E0000400320092C8BF000080FB0090
:10C200000000E9004F00DE0022892000014978008B
:10C210000000E00004003200110020008042800095
:10C22000A8F807008042880080428000B7F83700F5
:10C23000D4F9370003FB3700DBFB3700E3FC3700A2
:10C24000BEFD37007EFE0700000006007042880039
:10C250000000EB00DDF807004E08E20002003200AB
:10C260005028EF00030037001000200080428800B3
:10C27000A6F80700B04620007A7404000000000011
:10C28000004020008A740200000000008000780056
:10C290000080EB000100E0000100320060428000FD
:10C2A0000000060090089000E0019000018140002D
:10C2B000630179008100E90011089800020078000C
:10C2C0000000060023002000730098007001400069
:10C2D000610029002AD3040000000000889FBE00EE
:10C2E0008A9FBE008C1F7800000678004C039000E7
:10C2F0008203E80087834300E6837B008582E900B0
:10C30000020441000803430016831100860F520007
:10C3100003003E00818540000003EB000F00370062
:10C320000C007800E7FF07000E0037004C04900077
:10C330008384430086844400110009008584D8006A
:10C3400081047800890441008984E80089844400DC
:10C35000E9357C000603E8008B85E800840F530074
:10C36000F2FF39004F0678004F05BE004F04BE00B3
:10C3700000000600889FBE008A9FBE008C1F7800C8
:10C380008005780001067800130037001B03780051
:10C390000C84E800110009008281D8008103780034
:10C3A000888343008784430085834100110009008E
:10C3B0008283D80081037800888343008783430009
:10C3C000E7347B000500E00002003D008301E90046
:10C3D000010037008301E8000500E00003003D0094
:10C3E000848F5100E9FF310002003700848F510033
:10C3F000E6FF36004F0678004F05BE004F04BE0032
:10C4000000000600889FBE008A9FBE008C9FBE0071
:10C410008E1F7800800478000304780049009000A3
:10C420000187400060057F008106E8008D86460098
:10C43000E0817E0002005500800F540003003600AA
:10C44000090078009FFF07001D0037008485E90080
:10C450000A00D1008802EA00800F51000D0031006F
:10C46000088641000201E90008014100688044009B
:10C470000C027800830141000B017800BDFF07002A
:10C4800049019000110009000B86D80001B17E001F
:10C49000080037000502E9000A02420068804400F3
:10C4A0008802780003024200828141000B0178007B
:10C4B000B0FF0700490090000804550008307F00D5
:10C4C0004F0778004F06BE004F05BE004F04BE0068
:10C4D00000000600E6874700889FBE008A9FBE00D6
:10C4E0008C9FBE008E1F78000006780081057800C2
:10C4F000F2B79F008306780005047800CC00900016
:10C500000B80450080BF9F00610778000B00E800AA
:10C510000000400000814000920478000485E9009A
:10C520008E005500810F5400030036000C00780087
:10C5300064FF0700330037008E00D100818F560062
:10C54000110031000900E00002003A0088045500A3
:10C5500006003700888454008A84440011000900D2
:10C560008A84D8008000FD008004780009097800E2
:10C570000D82E90068004600880278000802420047
:10C5800089017800070037000D0244008801470048
:10C590008301E900680046008802EA0009024200BF
:10C5A000898141000A0178008B00780071FF070043
:10C5B000FFB09700018140008002EB000B003700C4
:10C5C0008D81440085814100110009008A81D800D5
:10C5D00081017800838145008381E80083814100E7
:10C5E000E2317B008502E8000281E8004C03900004
:10C5F000888F5200F2FF39000E0444008FB8970074
:10C6000008B378004F0778004F06BE004F05BE0004
:10C610004F04BE006F00B100000006000200FA00E7
:10C62000889FBE0080047800010478000900E000C3
:10C6300003003A00000028000000640056003700A4
:10C64000000024000800E0005000320008017800DB
:10C6500002F0A7000201EA000900780000F0A7003C
:10C660000000EA006102B900E681570011000900EC
:10C6700042AAD80081097800000378005FBA9700C9
:10C680008002EB00C022DD00040020001100090040
:10C6900042AAD800000178008600780002007800E5
:10C6A0000681CF000200E0000300320003022000F8
:10C6B00002815100040037000081CF000200E00039
:10C6C00001003200700111006C03510009003B00B1
:10C6D000C2282000030020009A040200000000008D
:10C6E000440ADD004C01DE00020172000200780005
:10C6F000220037001400200005002000820178008D
:10C700008301E900030033000402420085824A00ED
:10C71000FBFF37000400500085805800680151007D
:10C720000201E900030033008180D1000080D300C2
:10C73000FBFF3700FF0160004580DE004333DD0072
:10C7400086004000018040006429290064007800D0
:10C7500002022000030351000683B9008100E800B3
:10C7600081804000648078000380B90000034300AA
:10C7700081834B0011000900423BD8000800E00013
:10C7800002003D0001002800008050000900E00088
:10C7900001003C000000EA004F04BE000080FA00E7
:10C7A000000006000000E0000C003D0002002C002C
:10C7B000820F500003003D000100280001004000EE
:10C7C0000400370011002800820F500023003200BF
:10C7D0000000EA00120020000A00370002002400D6
:10C7E000820F500003003400010028000080500038
:10C7F00003003700F1FF2700820F500017003200BE
:10C800000001EB00C780DE0000027800F407B200F0
:10C810000100E8000000400043192900630078008F
:10C820000483B9008180400000082000040050000B
:10C830006382780000A0B9000600400087804800AD
:10C84000C909DD004702DE0004827100840078001F
:10C850000200E000010032008100EA0001007800DF
:10C86000000006000100240001004000CDFF370059
:10C870000100240001003700C288DE00808F5000D4
:10C88000FDFF3C00000178000000EB0007003700CE
:10C89000808140000080D100830F510002003500EC
:10C8A0000301510001004000C288DE000100E000E9
:10C8B000F7FF3A0000000600889FBE008A9FBE0076
:10C8C0000005BE000B0178008001EB001800370066
:10C8D000430020000311B80054002000110009009B
:10C8E0004499D800000178000A0378008202E90028
:10C8F0008582420085024500020278008001EB003B
:10C9000009003700B6037800550478008884530086
:10C910004240A9000300340078BB9F00870A7800DA
:10C92000130020000402E8008B0F5200F5FF3900CD
:10C93000E10F5100E6FF3E000300E000EAFF3A008D
:10C940004F05BE004F04BE0000000600889FBE00D9
:10C950008A1F7800000478000800780051FE070064
:10C9600000057800080078004EFE0700800478007B
:10C97000080078004BFE07000A0545008984440042
:10C980008000EB0005003700480190006935790010
:10C990008100E8000A85E8008984E800808F500063
:10C9A000F9FF39004F0578004F04BE000000060073
:10C9B000889FBE008A1F7800000478000800780075
:10C9C00038FE0700800478000800780035FE070074
:10C9D000000578000800780032FE07000A054500CF
:10C9E000898444008000EB00040037004801900077
:10C9F000EA3479008100E8008984E800808F5000E3
:10CA0000FAFF39004F0578004F04BE000000060011
:10CA1000889FBE008A9FBE0000047800080078004E
:10CA200020FE070000057800080078001DFE0700C2
:10CA300080047800080078001AFE0700800578005E
:10CA40000800780017FE0700C80090008B8545009D
:10CA5000E1817D000A054500898444008000EB00E7
:10CA6000070037004801900062827C000302420008
:10CA700004317D008100E8000A85E8008984E8002F
:10CA8000808F5000F7FF39004F05BE004F04BE00F5
:10CA900000000600889FBE008A9FBE000004780048
:10CAA00008007800FFFD0700800578000800780086
:10CAB000FCFD07000005780008007800F9FD07007C
:10CAC0008004780008007800F6FD07008000EB0085
:10CAD0000001EB000E003700C80190000B824500FA
:10CAE00001024200048241008982440081824200A6
:10CAF000858241000A03450001034300868141000D
:10CB000095027800138A42000201E8008180E80063
:10CB1000800F5100F0FF39004F05BE004F04BE00EA
:10CB200000000600889FBE008A9FBE0000047800B7
:10CB300008007800DBFD0700800578000800780019
:10CB4000D8FD07000005780008007800D5FD070033
:10CB50008004780008007800D2FD07008000EB0018
:10CB60000001EB000E003700C80190000B82450069
:10CB700001024200048241008A0245008182420093
:10CB800085824100098344000103430086814100FE
:10CB900095027800138A52000201E8008180E800C3
:10CBA000800F5100F0FF39004F05BE004F04BE005A
:10CBB00000000600889FBE008A9FBE000004780027
:10CBC00008007800B7FD07008005780008007800AD
:10CBD000B4FD07000005780008007800B1FD0700EB
:10CBE0008004780008007800AEFD07008000EB00AC
:10CBF0000001EB000D003700C80190000B824500DA
:10CC00000102420009834400010343008A024500F7
:10CC10008182420063037B00E3827A0005B3B9009E
:10CC200086317A000201E8008180E800800F51001F
:10CC3000F1FF39004F05BE004F04BE0000000600A2
:10CC4000E4874700889FBE008A9FBE008C9FBE007D
:10CC50008E1F7800000478000800780091FD07001E
:10CC600080067800080078008EFD07000006780036
:10CC7000080078008BFD0700800578000800780028
:10CC800088FD0700000278008004EB000005EB003F
:10CC90001F003700C80090000C004600090040004B
:10CCA000610078000B8145000901410061017900B4
:10CCB000CF91DE00E00F5100E08F59000C003200F0
:10CCC0000D874600090747000E874000CF80DE0031
:10CCD00084BF9F00F006020000000000000F7800F3
:10CCE0000A05E8008984E8000FBA970008003700B9
:10CCF0002300200073049800700144007100290093
:10CD0000080078002AD3020000000000020037006B
:10CD1000840F5500DFFF39004F0778004F06BE0033
:10CD20004F05BE004F04BE004F00B10000000600DA
:10CD3000889FBE008A9FBE0000047800080078002B
:10CD400058FD0700800578000800780055FD0700B1
:10CD5000000578000800780052FD07008004780084
:10CD6000080078004FFD07008000EB000001EB0099
:10CD700010003700C80190008B824500818242007C
:10CD80008582410009834400010343000A024500F3
:10CD90000102420063027A00E3017B00848F5100AC
:10CDA0000100340084017800830A78000201E80061
:10CDB0008180E800800F5100EEFF39004F05BE0072
:10CDC0004F04BE0000000600889FBE008A9FBE0080
:10CDD000000478000800780032FD07008005780024
:10CDE000080078002FFD0700000578000800780093
:10CDF0002CFD0700800478000800780029FD07005A
:10CE00008000EB000001EB0010003700C80190002B
:10CE10008B82450081824200858241000983440063
:10CE2000010343000A0245000102420063027A0046
:10CE3000E3017B00848F510001003D0084017800F4
:10CE4000830A78000201E8008180E800800F510029
:10CE5000EEFF39004F05BE004F04BE000000060083
:10CE6000889FBE008A9FBE008C1F78000004780057
:10CE7000080078000BFD0700000678000800780025
:10CE800008FD0700800578000800780005FD070010
:10CE9000000578000800780002FD07008004780093
:10CEA00008007800FFFC07008000EB000002EB00A8
:10CEB00015003700480190008B81450081814100B9
:10CEC000E28279008A014500818141006283790014
:10CED0008981440081814100E2817900838F520081
:10CEE00004003C0086017800858F510001003D0060
:10CEF000850178008C0246008182420003B17A00ED
:10CF00000402E8008180E800800F5200E9FF390048
:10CF10004F0678004F05BE004F04BE00000006001B
:10CF2000889FBE008A9FBE008C1F78000004780096
:10CF300008007800DBFC0700800478000800780017
:10CF4000D8FC07008005780008007800D5FC0700B1
:10CF5000000678004805900008007800D1FC070022
:10CF6000000040006A05780008007800CDFC07004A
:10CF700001022000810F550005003C000C06460010
:10CF80008B8545000002EB006011B8000D003700F2
:10CF9000480090008984440089044000800CEB0024
:10CFA00012003700E1827D0061037E0006ABB9000C
:10CFB0000201430083814B000402E8000C86E80074
:10CFC0008B85E800C8009000800F5200F5FF390003
:10CFD000898444000A05E900030033008381D100FD
:10CFE0000281D300FBFF370082B07C004F0678003F
:10CFF0004F05BE004F04BE00000006000200FA000C
:10D00000889FBE008A9FBE00000178000200780061
:10D01000B2BF9F00A3FC0700800478003FB89700D0
:10D02000A0FC0700800578003FB897009DFC070032
:10D03000000478003FB897009AFC070000057800CC
:10D040003FB8970097FC0700800278003FB997002F
:10D050000500E000240032004202900009804400F4
:10D06000E40178006118B9008B85450003B27D00AA
:10D07000080444004202900003327C0014002000A7
:10D08000100037008901420083814100E681790068
:10D090000B034300968F510001003D00030B780005
:10D0A0004203900008034300968F510001003400B2
:10D0B000030B78004F9BDE000080410081004B0095
:10D0C0000402E80042039000850F5200EDFF390092
:10D0D0000A0545000A0443006129B800F006020071
:10D0E00000000000000C78004F05BE004F04BE0099
:10D0F0000080FA0000000600889FBE008A9FBE00E4
:10D10000000478000800780066FC070080047800BE
:10D110000800780063FC07008005780008007800AC
:10D1200060FC070000057800080078005DFC07003F
:10D130000000E000150032008B8545000A0545001F
:10D14000898444008000EB0004002800F3FF2700DE
:10D15000C802900065817C00830F510002003D00F1
:10D1600081B27D0082017800840F510003003400F9
:10D170004802900001327D00020278008100E80040
:10D180008984E800808F5000F1FF39004F05BE0010
:10D190004F04BE0000000600889FBE000004780017
:10D1A000080078003FFC0700800478000800780041
:10D1B0003CFC07008000780089844400480090000F
:10D1C00009004000BCFD07004F04BE00000006003F
:10D1D000E6874700889FBE008A9FBE008C9FBE00E6
:10D1E0008E1F780000047800080078002DFC0700EE
:10D1F00000077800080078002AFC07008006780005
:10D200000800780027FC0700000678000800780076
:10D2100024FC0700800578000800780021FC070046
:10D22000800278008004EB000005EB00240037004A
:10D23000C80090000D80460009004000610378009E
:10D240000C00460009004000610078000B81450099
:10D250000901410061017900CF91DE00E00F51002A
:10D26000E08F59000E0032000E0247000902420012
:10D270000482400000B0B90084BF9F00F5B79F0052
:10D28000F0060200000000000FBA9700000A7800C4
:10D290000A05E8008984E800FFB29700080037001B
:10D2A00023002000730498007001440071002900DD
:10D2B000080078002AD302000000000002003700B6
:10D2C000850F5500DAFF39004F0778004F06BE0082
:10D2D0004F05BE004F04BE006F00B1000000060005
:10D2E000E4874700889FBE008A9FBE008C9FBE00D7
:10D2F0008E1F78008004780009007800E9FB0700A1
:10D300000007780009007800E6FB07008006780037
:10D3100009007800E3FB07000006780009007800A8
:10D32000E0FB0700000178000004EB000005EB00C3
:10D330000F003700C90590008C004600888040002F
:10D340000D80460008004000EB8078006B007800FC
:10D3500082BF9F00B1FC07008E004700888040001C
:10D3600080B578000A05E8000884E8000FB9970046
:10D37000820F5500EFFF39004F0778004F06BE00BF
:10D380004F05BE004F04BE004F00B1000000060074
:10D39000889FBE008A9FBE008C9FBE0080047800DC
:10D3A00009007800BFFB07008006780009007800BC
:10D3B000BCFB07000005780009007800B9FB0700F6
:10D3C000000678000A0545000004EB00080037005D
:10D3D000C90590006B007D00F2FC07008D00440041
:10D3E0008180400080B578000804E8000A85E800E4
:10D3F0008C0F5400F6FF39004F06BE004F05BE00EB
:10D400004F04BE0000000600889FBE008A9FBE0039
:10D410008C9FBE008004780009007800A1FB070003
:10D4200080067800090078009EFB07000005780060
:10D43000090078009BFB0700000678000A054500FC
:10D440000004EB0008003700C90590006B007D0068
:10D4500004FD07008D0044008180400080B5780005
:10D460000804E8000A85E8008C0F5400F6FF390034
:10D470004F06BE004F05BE004F04BE000000060070
:10D48000889FBE008A9FBE008C9FBE008E1F7800C2
:10D49000000478000800780082FB0700000578008F
:10D4A000080078007FFB07008005780008007800FE
:10D4B0007CFB0700C80490008B804500E98678005B
:10D4C0008B05E8008B854500E9857D000000400064
:10D4D000690778000E007800E2FC0700000678007B
:10D4E0000E007800AFFC07008A0045000DE2B9008D
:10D4F0000B81B9000202520083825A00412BDD00E9
:10D500004F21DE000201730082B478000A05E800B2
:10D51000C80090000A0545000D81B9000BE6B9006E
:10D520000206460083864E004168DD004F61DE0042
:10D530000201700082307D004F0778004F06BE0068
:10D540004F05BE004F04BE0000000600889FBE00CD
:10D550008A9FBE008C9FBE000004780008007800FF
:10D5600050FB070080067800080078004DFB07009C
:10D5700000057800080078004AFB070000067800E4
:10D580000A0545008004EB000F003700C805900035
:10D590006B007D000A85E8000000E00005003D000A
:10D5A000C17A280008007800C69002000000000040
:10D5B00007003700AEFC07008D80440081804000EA
:10D5C00080B578008904E8008C8F5400EFFF3900A3
:10D5D0004F06BE004F05BE004F04BE00000006000F
:10D5E000889FBE008A9FBE008C9FBE00800478008A
:10D5F000090078002BFB0700000478000900780080
:10D6000028FB0700000578000900780025FB0700CB
:10D61000800578000900780022FB070000017800EF
:10D62000C90690008B854500ED837D008A01E900E5
:10D6300003824100048246000006EB000700370029
:10D640000C06E800820F560004003600080444006F
:10D65000888046008008EB004B0037005400E00053
:10D66000F7FF3A000C0278008C8141008381410071
:10D67000838146000B0037000C06E800820F56003D
:10D6800008003600080444000400E00036003200C0
:10D690000400E900870F5000330039000000D1007A
:10D6A000380037005300E000F3FF32000003EB00C6
:10D6B0008002EB008001EB000302780003003700DA
:10D6C0000402E800820F5200090031008C0442007D
:10D6D000110009008284D800810478008A84440003
:10D6E00089844400ED847C000900E000F4FF3A00E6
:10D6F00083045200858F54000600340083014200E9
:10D7000025002000110009008501D80000037800E1
:10D7100089027800820F5200050039000F0037009F
:10D720008301E800828F5100020039000B003700AE
:10D73000840178000C824100110009000282D800A7
:10D74000010278000A024200040242006D027A00DF
:10D750000400E000D8FF3A00F1FF3700080444005D
:10D76000878F520003003D0008844600008CEB00C8
:10D77000050037000C004300110009000280D800AA
:10D780008000FD0080367C004F06BE004F05BE00C5
:10D790004F04BE0000000600504B88000000060049
:10D7A00050252600514B80000088B900926123006B
:10D7B00000004100504B880000000600889FBE001A
:10D7C0008A9FBE008C1F7800000578000A00780050
:10D7D000B4FA0700800478000A007800B1FA070064
:10D7E00080057800898444000004EB0006003700BF
:10D7F0004A06900009064600E9FF0700000E78007F
:10D800000804E8008984E8008B0F5400F8FF390011
:10D810004F0678004F05BE004F04BE000000060012
:10D82000889FBE008A1F78000004780008007800F6
:10D830009CFA0700800478000800780099FA070035
:10D84000000578000800780096FA0700480090006C
:10D850000A05450089844400693578004F05780041
:10D860004F04BE0000000600889FBE008A9FBE00D5
:10D870008C9FBE00000478000800780089FA070039
:10D88000000578000800780086FA07008004780018
:10D890000800780083FA07008006400048009000E6
:10D8A000E0857E00080078007EFA07000006780018
:10D8B000080078007BFA070000027800480090001A
:10D8C00060807E000000E00003003500E3005600A9
:10D8D000810F5000030036000800780079FA070035
:10D8E000040037008C0278000A01BE000800BE0068
:10D8F0007AFA07004F06BE004F05BE004F04BE0077
:10D9000000000600889FBE008A9FBE008C9FBE005C
:10D910008E1F7800000478000800780061FA070084
:10D9200080047800080078005EFA0700000578009F
:10D93000080078005BFA070080064000480090006D
:10D94000E0857E000800780056FA0700000678009F
:10D950000800780053FA070000077800C80090001C
:10D9600009814400E10179000901E8000201410058
:10D97000E10279000C81E900E1807E000100E00015
:10D9800009003500630656008C8F500006003E00EB
:10D990008B805100810F570003003E000A054500AF
:10D9A0008003EB000F0037000800780045FA0700FD
:10D9B0000E003700C80190000B82420007024200AF
:10D9C000110009000282D80001027800048244009C
:10D9D0000482E800040242006AB279008703E8008A
:10D9E0000A85E8008E8F5300F2FF39004F07780058
:10D9F0004F06BE004F05BE004F04BE0000000600EB
:10DA0000889FBE008A9FBE008C9FBE0000047800E5
:10DA10000800780023FA07008004780008007800E6
:10DA200020FA070000057800080078001DFA0700BA
:10DA30008006400048009000E0857E0008007800E5
:10DA400018FA0700000678000800780015FA0700A9
:10DA5000800278004800900060807E000000E000B6
:10DA60000300350063005600808F55000300360028
:10DA70000800780013FA0700040037000C02780051
:10DA80000A01BE000800BE0092FA07004F06BE0061
:10DA90004F05BE004F04BE0000000600889FBE0078
:10DAA0008A9FBE008C1F7800000478000800780070
:10DAB000FCF907008004780008007800F9F90700F5
:10DAC0000006780008007800F6F90700C80090000A
:10DAD0000C06460061057E0000004000E10578006C
:10DAE00008007800EFF90700000278004800900075
:10DAF00060007E000000E00003003500630052007B
:10DB0000800F55000300360008007800EDF907008B
:10DB1000030037000A01BE000800BE0039FA070002
:10DB20004F0678004F05BE004F04BE0000000600FF
:10DB3000889FBE008A9FBE0000047800080078001D
:10DB4000D8F907008004780008007800D5F90700AC
:10DB50000005780008007800D2F9070080057800F9
:10DB600008007800CFF90700800278000B027800E7
:10DB70008001EB000A0178000800BE0055FA07009A
:10DB80004F05BE004F04BE0000000600889FBE0087
:10DB90008A9FBE000004780008007800C1F90700E1
:10DBA0008004780008007800BEF9070000057800BE
:10DBB00008007800BBF907008005780008007800AD
:10DBC000B8F907008002780048019000898044007D
:10DBD0000B027800E28178000A0178000800BE009C
:10DBE0003CFA07004F05BE004F04BE0000000600CF
:10DBF000889FBE008A9FBE008C1F780000047800BA
:10DC000008007800A7F90700800578000800780070
:10DC1000A4F907000006780008007800A1F90700C1
:10DC200000057800080078009EF90700800478005D
:10DC30008A027800090278008001EB000B0178006D
:10DC40008C00780008007800A4F907000A02780028
:10DC5000890178000001EB008B0078000800780053
:10DC6000E8F907004F0678004F05BE004F04BE00DC
:10DC700000000600889FBE008A9FBE008C9FBE00E9
:10DC8000000478000800780086F907008004780016
:10DC90000800780083F90700800678000800780003
:10DCA00080F9070000067800080078007DF9070079
:10DCB00080057800C8009000098044000080400082
:10DCC000108515008C0278000B0278008A0178001C
:10DCD000090178008D007800080078007FF90700BE
:10DCE0000C0278000A01BE000800BE00C5F907005A
:10DCF0004F06BE004F05BE004F04BE0000000600E8
:10DD0000F14380000100E0001200320084C8EC0002
:10DD100084E8B700FF4F500004003400E380600047
:10DD2000F143880000CEB30084E8B7007E08E2002B
:10DD30000800320041882000914078008100FB00FB
:10DD400001F0A7008100EA00E0C0B300E8C50200CE
:10DD500000000000F043800000F0A7000000EA008F
:10DD60000000E9004F00DE008000EB000004E0004E
:10DD700005003200E1822000914078008180FB00A4
:10DD80008100E900CF08DE002EE8B7000100E000C6
:10DD9000040032008040EB00E0C0B300E8C50200A0
:10DDA0000000000000000600881F7800F1FB220040
:10DDB000A046230065824000514178000204E00043
:10DDC0000600320010417800E3414100034878002A
:10DDD00002C2B30082CF5100010036000248780031
:10DDE0000000E800848F5000F3FF3A00C046230093
:10DDF0001004E0000B00320008022000C04623009F
:10DE00009040780008407800E8C50200000000005B
:10DE10000804E80040022000800F5400F7FF3A0099
:10DE20001C003700A0462300904078000104E00069
:10DE30000300320010C2B300E8C502000000000079
:10DE4000B0462300904078000104E0000300320057
:10DE500020C2B300E8C5020000000000D046230045
:10DE6000904078000104E0000300320000C2B300DB
:10DE7000E8C5020000000000E04623009040780062
:10DE80000104E0000300320030C2B300E8C5020024
:10DE9000000000008000EB00A04623001004E0001A
:10DEA00004003A000080E8009080FB008100E90057
:10DEB000CF08DE000000EB000104E00004003200A7
:10DEC00036C8BF000080FB000000E9004F00DE0004
:10DED00063832000814978000000E00004003200E4
:10DEE0008040EB0010C2B300E8C502000000000053
:10DEF0008000EB00B04623001004E00004003A006C
:10DF00000000E8009080FB008100E900CF08DE00FF
:10DF10000000EB000104E0000400320035C8BF003F
:10DF20000080FB000000E9004F00DE00538320006A
:10DF3000814978000000E000040032008040EB00DE
:10DF400020C2B300E8C50200000000008000EB0022
:10DF5000D04623001004E00004003A000000E9006D
:10DF60009080FB008100E900CF08DE000000EB009C
:10DF70000104E0000400320034C8BF000080FB0050
:10DF80000000E9004F00DE00438320008149780053
:10DF90000000E000040032008040EB0000C2B3004B
:10DFA000E8C50200000000008000EB00E04623000E
:10DFB0001004E00004003A000080E9009080FB00BB
:10DFC0008100E900CF08DE000000EB000104E00062
:10DFD0000400320033C8BF000080FB000000E900ED
:10DFE0004F00DE0033832000814978000000E0000C
:10DFF000040032008040EB0030C2B300E8C50200EC
:10E00000000000004F04780000000600618A200034
:10E01000914078008180FB008100E900CF08DE009C
:10E020000000EB000104E000040032003CC8BF0027
:10E030000080FB000000E9004F00DE00C2832000EA
:10E04000014978000000E000040032008040EB004D
:10E05000D0C1B300E8C5020000000000A648E200FD
:10E0600005003200A668EF0001C2B300D0C1B300C2
:10E07000E8C502000000000000000600881F7800CC
:10E080008A48EC008AE8B700EA4F500024003A00C2
:10E090008A68EF006194800050092000808F500052
:10E0A00006003C008040EB0060C2B300E8C50200FF
:10E0B0000000000001C2B3001600370080112000EC
:10E0C000808F50000600340001C2B3006E40400053
:10E0D000E8C50200000000008040EB000D003700A2
:10E0E000A0F62F00010040004500DD0022082000BE
:10E0F000110009000200D800004478008040780038
:10E1000060C2B300E8C502000000000001C2B30015
:10E1100088C0500070C2B300E8C5020000000000D3
:10E120004F04780000000600889FBE008464AB00A6
:10E130003C0032008648E2000E003A008040EB00CE
:10E1400050C0B300E8C50200000000008040EB00B2
:10E1500060C0B300E8C50200000000008040EB0092
:10E1600070C0B300E8C502000000000010C0B3009A
:10E1700086E8B700738820009341780010002000E3
:10E180000304E000010032000300FB0072C0B30092
:10E19000EA0F500004003C0022002000110009009A
:10E1A0000200D8000041E80083404100728820004E
:10E1B0000149780040C6B30080CF500012003400FF
:10E1C0008548EC0085E8B70011C0B30072882000D4
:10E1D00001497800E34F500001003A008568EF00E4
:10E1E0008548E20008003A008040EB0070C0B300B0
:10E1F000E8C50200000000008040EB0060C0B300F2
:10E20000E8C502000000000085C8BF00654040006E
:10E210007188200091407800E8C5020000000000ED
:10E22000AF003700602721008080E800910078006F
:10E2300010804000883E20000884B900A2F8200029
:10E240001100090042CCD800000478008648E200A2
:10E25000260032008668EF0050182000800F54001E
:10E260000A00360001C2B30050C0B300E8C5020086
:10E270000000000001C2B30060C0B300E8C50200A6
:10E280000000000001C2B300150037008016200016
:10E29000800F54000600360001C2B30050C0B30026
:10E2A000E8C502000000000001C2B300080037000A
:10E2B00040152000800F54000C00360001C2B3004E
:10E2C00050C0B300E8C50200000000008040EB0031
:10E2D00060C0B300E8C50200000000008040EB0011
:10E2E00070C0B300E8C502000000000011C0B30018
:10E2F00050182000800F540003003E008040EB00C7
:10E300000000EB000400370032C8BF000080FB00B3
:10E310000000E9004F00DE00228320000149780060
:10E320000000E0000C00320001C2B30050C0B30096
:10E33000E8C502000000000001C2B30060C0B300E5
:10E34000E8C502000000000001C2B30070C0B300C5
:10E35000E8C502000000000070E92F00080040003E
:10E3600011C0B300F70F5000030036008040EB00EF
:10E370000000EB000400370031C8BF000080FB0044
:10E380000000E9004F00DE00128320000149780000
:10E390000000E0000C00320001C2B30050C0B30026
:10E3A000E8C502000000000001C2B30060C0B30075
:10E3B000E8C50200000000008040EB0070C0B30020
:10E3C000E8C5020000000000B0EA2F00080040008D
:10E3D00011C0B300EE0F5000030036008040EB0088
:10E3E0000000EB000400370030C8BF000080FB00D5
:10E3F0000000E9004F00DE000283200001497800A0
:10E400000000E0000C00320001C2B30050C0B300B5
:10E41000E8C50200000000008040EB0060C0B300CF
:10E42000E8C50200000000008040EB0070C0B300AF
:10E43000E8C502000000000011C0B3004015200034
:10E44000800F5400030036008040EB000000EB001A
:10E45000040037002FC8BF000080FB000000E90067
:10E460004F00DE00F2822000014978000000E00049
:10E47000080032008040EB0060C0B300E8C5020035
:10E48000000000008040EB0070C0B300E8C502004F
:10E490000000000040152000800F540010003E00D6
:10E4A0008748EC0087E8B700E34F500004003A00CB
:10E4B00001C2B30050C0B300E8C502000000000074
:10E4C00087C8BF00E54F5000050034008040EB00D6
:10E4D00050C0B300E8C50200000000008768EF00EC
:10E4E0004F04BE000000060000FC22009080FB00EC
:10E4F0008100EA00CF08DE000000EB000104E0002C
:10E50000040032003BC8BF000080FB000000E900AF
:10E510004F00DE00B2832000014978000000E000D7
:10E5200003003200200020000EE102000000000085
:10E5300010FC22009080FB008100EA00CF08DE0082
:10E540000000EB000104E000040032003AC8BF0004
:10E550000080FB000000E9004F00DE00A2832000E5
:10E56000014978000000E000030032002000200094
:10E570000EE102000000000020FC22009080FB0061
:10E580008100EA00CF08DE000000EB000104E0009B
:10E590000400320039C8BF000080FB000000E90021
:10E5A0004F00DE0092832000014978000000E00067
:10E5B00003003200300020000EE1020000000000E5
:10E5C00030FC22009080FB008100EA00CF08DE00D2
:10E5D0000000EB000104E0000400320038C8BF0076
:10E5E0000080FB000000E9004F00DE008283200075
:10E5F000014978000000E000030032002000200004
:10E600000EE102000000000040FC22009080FB00B0
:10E610008100EA00CF08DE000000EB000104E0000A
:10E620000400320037C8BF000080FB000000E90092
:10E630004F00DE0072832000014978000000E000F6
:10E6400003003200200020000EE102000000000064
:10E6500000000600E4874700889FBE008A9FBE0036
:10E660008C9FBE008E1F7800CC3C23006B232100C2
:10E67000C23B23006E0246008B0178008C007800BC
:10E6800053007800D10F100001003D008008780091
:10E690000000E00003003200920F1000010034007F
:10E6A000000978000281E800848F5000F4FF3A00EE
:10E6B000AA3D2300C9262100E40145008900780015
:10E6C0000A00780051017800D00F110001003D00D0
:10E6D00002087800830F5000FAFF3A00AD3B230098
:10E6E0000004EB005D0078005C0710005B00100088
:10E6F00001003B000000EB00010220000181B90095
:10E70000110009004E19D80000077800A0282A003F
:10E7100060417C008E4078000240780082BF9F00FC
:10E72000E8C50200000000000FB99700E20F540096
:10E7300004003A000240E8008E407800E8C502007C
:10E74000000000000804E800E70F5400E5FF3A006D
:10E750000B292A000004EB005A01780059007800C8
:10E760000000E00001003D000000EB00010220007D
:10E770000182B90011000900422AD80080407800C7
:10E780005B407800E8C50200000000000804E800D3
:10E79000E20F5400F0FF3A004F0778004F06BE002A
:10E7A0004F05BE004F04BE004F00B1000000060040
:10E7B000889FBE0050948000F40F50003C003C0045
:10E7C00041948000309480000E630200000000003D
:10E7D00022002000110009000200D800037D200063
:10E7E00003014000F1F92000C8012000810F510011
:10E7F0001C0036000277210002024000B801200010
:10E80000810F5200170036000471220004024000FC
:10E81000A8012000810F520012003600046B230073
:10E820000402400098012000810F52000D003600C4
:10E8300088012000F5D52600850F520009003E0012
:10E84000830150006C044400818F510005003600A4
:10E8500002005000F8012000810F500001003E002E
:10E86000660444005994800009F0A7008904EA0076
:10E87000F48414008984440001003B008004EB0010
:10E88000404480000000E000030035008040EB00C1
:10E89000E8C50200000000008940780008407800C8
:10E8A000E8C5020000000000484488000700370067
:10E8B000404480000000E000030035008040EB0091
:10E8C000E8C502000000000088A8EF004F04BE0069
:10E8D00000000600670060004800DD00F18F2F0097
:10E8E000F20580008280600081007000F1058800E0
:10E8F00000000600114480000100E00002003A0020
:10E900008AC0A9009AC0A800008070001044880046
:10E91000000006008208B600000006008AC0A800B9
:10E92000000006000080EA008208B600104488005B
:10E9300001003A009AC0A900000006001000FA0089
:10E94000889FBE008A9FBE0090C8BF00E14F500064
:10E950004B023A00D0F40200000000000000E0008A
:10E9600004003A007AC30200000000000048A3003F
:10E970002700320000002100EAFF07000001EB0041
:10E980006000B800BCC70200000000008043EB003C
:10E990000743780087427800074278008741780073
:10E9A000074178008740780007407800C8C6020019
:10E9B000000000008043EB000743780087427800A6
:10E9C0000742780087417800074178008740780047
:10E9D000074078006CC702000000000020272100DB
:10E9E0000008EB000080E8000008EB007AC302009A
:10E9F000000000000058A30002003200B4C402006E
:10EA000000000000D45F0200000000003702370061
:10EA10008EC8BF00E14F500008003200E24F5000A6
:10EA2000090032000004E0000C003A000001EB0095
:10EA3000F100200000022000060037000001EB007A
:10EA40000102200002003700020220008000EB00DB
:10EA5000F0002000BCC70200000000008FC8BF000B
:10EA6000E14F40001D003A008B48EC008BE8B700F6
:10EA7000FC4F50000A003A0007C2B3000743780079
:10EA80008742780007427800874178000741780084
:10EA900087407800074078006CC702000000000043
:10EAA00080C3B3008B48E300380036008B68EF006A
:10EAB0008043EB00074378008742780007427800E4
:10EAC0008741780007417800874078000740780048
:10EAD0006CC70200000000002C0037009C540200AC
:10EAE000000000009C540200000000009C54020042
:10EAF0000000000000047800884378000843780094
:10EB000088427800084278008841780008417800FF
:10EB100088407800084078006CC7020000000000C0
:10EB20008EC8BF00E14F500008003200E24F500095
:10EB30000C0032000004E0000F003A00C545DD0083
:10EB4000C55DDE006F44B900030037006F40B900B7
:10EB5000C505DE004544DD004545DE008044EB0090
:10EB6000050037006F40B900C505DE004544DD00F3
:10EB7000C544DE000045EB000981FB008A80FB00F4
:10EB80000B80FB00BCC70200000000008FC8BF0064
:10EB9000750032004240A90003003C00E14F4000F4
:10EBA000B3013A0005003700E14F5000C9003200C0
:10EBB000E24F5000AE013A008C01370000FC220009
:10EBC0009080FB008100EA00CF08DE000000EB002F
:10EBD0000104E000040032004AC8BF000080FB00CE
:10EBE0000000E9004F00DE00A28420000149780007
:10EBF0000000E000010032008E68ED0030FC2200D1
:10EC00009080FB008100EA00CF08DE000000EB00EE
:10EC10000104E0000400320049C8BF000080FB008E
:10EC20000000E9004F00DE009284200001497800D6
:10EC30000000E000010032008E68EC0010FC2200B1
:10EC40009080FB008100EA00CF08DE000000EB00AE
:10EC50000104E0000400320048C8BF000080FB004F
:10EC60000000E9004F00DE008284200001497800A6
:10EC70000000E000010032008E68EC0040FC220041
:10EC80009080FB008100EA00CF08DE000000EB006E
:10EC90000104E0000400320047C8BF000080FB0010
:10ECA0000000E9004F00DE00728420000149780076
:10ECB0000000E000010032008E68ED008EC8BF0049
:10ECC00009003B007AC30200000000000008A30016
:10ECD0000200320020C0B3000100370010C0B300B2
:10ECE0008EE8B7000A003700E14F500004003400FE
:10ECF0007AC30200000000000008A30003003200F5
:10ED00008EC8BF00E24F5000010034008E68EF0053
:10ED100020FC22009080FB008100EA00CF08DE008A
:10ED20000000EB000104E0000400320046C8BF0010
:10ED30000080FB000000E9004F00DE00628420003C
:10ED4000014978000000E00049013200E18820001C
:10ED500091407800F28820000149780010C0B3008B
:10ED600091E8B7004201370000FC22009080FB00D0
:10ED70008100EA00CF08DE000000EB000104E000A3
:10ED80000400320045C8BF000080FB000000E9001D
:10ED90004F00DE0053842000814978000000E0002D
:10EDA000030032008D68EC00ECBD020000000000A2
:10EDB00030FC22009080FB008100EA00CF08DE00DA
:10EDC0000000EB000104E0000400320044C8BF0072
:10EDD0000080FB000000E9004F00DE0043842000BB
:10EDE000814978000000E000030032008D68ED00EA
:10EDF000ECBD0200000000008DC8BF0002003B0017
:10EE00008D68EF0004003700E84F50000200340026
:10EE100080C0B3008DE8B700D18820009140780011
:10EE20008100FB0051868900C0FF2F000088B900D7
:10EE3000E40040007A8057006A815700012878007A
:10EE40000100E00001003D000008EB00E48040000C
:10EE5000820F5000F9FF3A008FEB97002FEB9700DD
:10EE6000CFEA97006FEA97008FF197002FF1970094
:10EE7000CFF097006FF09700C8C6020000000000B6
:10EE80008000EB0020FC22001004E00005003200AE
:10EE900011892000914078008180FB008100E90009
:10EEA000CF08DE000000EB000104E00004003200A7
:10EEB00043C8BF000080FB000000E9004F00DE00F7
:10EEC00033842000814978000000E000E80032002F
:10EED000B5003700909380000000E000640032002D
:10EEE00040FC22009080FB008100EA00CF08DE0099
:10EEF0000000EB000104E0000400320042C8BF0043
:10EF00000080FB000000E9004F00DE0023842000A9
:10EF1000814978000000E000030032008C68EC00BA
:10EF2000ECBD02000000000010FC22009080FB00FD
:10EF30008100EA00CF08DE000000EB000104E000E1
:10EF40000400320041C8BF000080FB000000E9005F
:10EF50004F00DE0013842000814978000000E000AB
:10EF6000030032008C68ED00ECBD020000000000E0
:10EF7000C1882000914078000104E00018003500AD
:10EF8000FFCF50000E0034007FC150008043EB00E3
:10EF9000074378008742780007427800874178006D
:10EFA000F1C1B30007407800C8C6020000000000AD
:10EFB00020C3B3008C48E30025003400180037005C
:10EFC0008043EB00074378008742780007427800CF
:10EFD0008741780007417800074078001A00370021
:10EFE000FFCF400010003D00F7C1B30016CEB300C4
:10EFF000014353008042EB000542780085417800D0
:10F00000054178008540780005407800C8C60200B8
:10F0100000000000E0CCB3008C48E3000C003D0091
:10F020008CE8B7000A0037008143EA000043EB0098
:10F0300086427800064278008641780006417800D2
:10F040008640780006407800C8C602000000000034
:10F050008CC8BF000000FB00A10D2300031020009E
:10F0600083084000030178008180E8008008510097
:10F0700000FC22009080FB008100EA00CF08DE0047
:10F080000000EB000104E0000400320040C8BF00B3
:10F090000080FB000000E9004F00DE000284200039
:10F0A000014978000000E0000D0032002027210017
:10F0B00001F82F0010804000909388004127210024
:10F0C00002F82F009108410011E82F00810F500035
:10F0D00003003D0000E82F0090938800A093880073
:10F0E00030FC22009080FB008100EA00CF08DE00A7
:10F0F0000000EB000104E000040032003FC8BF0044
:10F100000080FB000000E9004F00DE00F3832000D8
:10F11000814978000000E0000C0032002027210027
:10F1200003082000108041009093880041272100AF
:10F1300091884100F1172000810F50000300340036
:10F140000018200090938800A09388008000EB00B6
:10F1500020FC22001004E00005003200118920008C
:10F16000914078008180FB008100E900CF08DE003B
:10F170000000EB000104E000040032003EC8BF00C4
:10F180000080FB000000E9004F00DE00E283200069
:10F19000014978000000E0003500320090938000C3
:10F1A0000000E0000C003A008FE8EF008043EB0025
:10F1B000074378008742780007427800874178004B
:10F1C000074178008740780007407800C8C60200F1
:10F1D0000000000026003700202721000008EB0077
:10F1E0000080E8000008EB00210037007AC302002D
:10F1F000000000000058A30002003A00ACC4020066
:10F20000000000008000EB0020FC22001004E00061
:10F210000500320011892000914078008180FB00B8
:10F220008100E900CF08DE000000EB000104E000EF
:10F23000040032003DC8BF000080FB000000E90070
:10F240004F00DE00D2832000014978000000E0007A
:10F25000070032007AC30200000000000058A3003B
:10F2600002003200B4C40200000000008FE8EF008A
:10F2700020FC22001004E0001C003A001A003700B5
:10F2800010FC22001004E000170032006300400070
:10F290001004E000140032009148EC0091E8B7003F
:10F2A00041C6B300814F5000100036008140E80095
:10F2B000814F500009003A0010C0B30090E8B70039
:10F2C0000040200097FD07008FE8EF005086810086
:10F2D0008DE8B700D08681008CE8B70060C6B30027
:10F2E00091E8B700010037009168EF004F05BE00BC
:10F2F0004F04BE000080FA000000060002882000D3
:10F30000124178008288AB0016003200A194800080
:10F310000100E0000B0032000080FB00810F500074
:10F32000030034004300DE00804F51000300390029
:10F330000204E000040032000240E90080E8B70067
:10F34000010037008068EF000188200091407800BC
:10F35000814F510003003200E0C1B300E8C5020054
:10F360000000000000000600E18720000000E0002F
:10F3700003003D0067006000910870000000060077
:10F380000080EA0091086000000006000200FA0018
:10F39000F0BF9F006101B900E40F5100E08F5900F8
:10F3A00010003E0002600100040037000500370035
:10F3B00006003700070037000800370011088800F2
:10F3C0000E003700610888000C00370071088800C3
:10F3D0000A003700D108880008003700E1088800DB
:10F3E000060037008F81E90042102000014D200007
:10F3F000A0152A0004FB0200000000000080FA00B3
:10F40000000006000200FA00F0BF9F00EA0F500063
:10F4100019003E00120020000010DD008241200093
:10F42000020160000D003A00000178006220B20085
:10F4300003003A000008A30015003A000E00370050
:10F44000E1806000C308DD00800880000030A1007A
:10F4500000807000800888000D003700E1806000A7
:10F46000C308DD00F00880000030A10000807000BB
:10F47000F0088800060037008F81E9004210200064
:10F48000A1462000A0152A0004FB02000000000095
:10F490000080FA00000006000200FA00F0BF9F00A2
:10F4A0006101B900EA0F5100E08F59002F003E00C2
:10F4B000026001000A003700100037001600370014
:10F4C0001C003700220037002800370027003700D3
:10F4D00026003700250037000800370015003700E8
:10F4E000E3806000C408DD00F0FC2F000401B600DA
:10F4F000008070002008880022003700E380600050
:10F50000C408DD00F0FC2F001001B6000080700080
:10F51000800888001B003700E3806000C408DD001D
:10F52000F0FC2F001201B6000080700090088800E7
:10F5300014003700E3806000C408DD00F0FC2F00F9
:10F540001E01B60000807000F00888000D00370032
:10F55000E3806000C408DD00F0FC2F002001B6004D
:10F560000080700000098800060037008F81E900E4
:10F5700042102000214A2000A0152A0004FB0200AE
:10F58000000000000080FA00000006000200FA00FF
:10F59000F0BF9F00401ADE0005002000E90F500078
:10F5A00003003200EA0F500007003A000300370062
:10F5B000620888007408880009003700D2088800B3
:10F5C000E4088800060037008F81E900421020001F
:10F5D000A14F2000A0152A0004FB0200000000003B
:10F5E0000080FA0000000600E80F5000020034001E
:10F5F0000000D0007100500000000600800078007C
:10F6000010002000E88F500001003C000000EB00DB
:10F61000000006000200FA00889FBE008A1F7800E2
:10F62000C0BF9F0000047800EC0F540006003600B5
:10F63000E881570042102000E1152000A0152A00A3
:10F6400004FB02000000000008007800E6FF07004D
:10F6500000057800A93923004250DD0000804400F5
:10F66000900078000110A1000100A00001087800BE
:10F6700008007800E1FF07000000E000040032000D
:10F680000A05E8004255DD008A8444001900A00004
:10F690004F0578004F04BE000080FA00000006000D
:10F6A000D1FF07004200DD000080E800813923001F
:10F6B0006100780061006000000006000200FA00AE
:10F6C000889FBE00D0BF9F000104780080047800AE
:10F6D000EC8F540004003600E681570042102000F1
:10F6E000E11920000B00370009007800BEFF070079
:10F6F0004200DD000080E8008139230061007800CD
:10F700000018A30006003A00E681570032102000DE
:10F71000211A2000A0152A0004FB020000000000AE
:10F720006148B900EA0F5000E08F58002A003E00FF
:10F73000006001000A0037000F0037001400370096
:10F74000190037001E003700230037002200370061
:10F750002100370020003700070037001200370073
:10F760004F44DD002008800000F0A100000074007C
:10F77000200888001C0037004F44DD00800880000E
:10F7800000F0A10000007400800888001600370017
:10F790004F44DD009008800000F0A10000007400DC
:10F7A00090088800100037004F44DD00F00880000A
:10F7B00000F0A10000007400F00888000A00370083
:10F7C0004F44DD000009800000F0A100000074003B
:10F7D0000009880004003700E6815700421020002D
:10F7E000511C2000CBFF37004F04BE000080FA0000
:10F7F000000006008000EB00B0FF37001100200081
:10F80000AEFF37000200FA00F0BF9F00CF80DE009D
:10F81000EA0F5000E08F580018003E000060010021
:10F820000A0037000C0037000D0037000F003700CA
:10F830001000370011003700100037000F003700AC
:10F840000E00370003003700070037000208880069
:10F850001000370043088800320888000D00370088
:10F86000520888000B003700B3088800A2088800FF
:10F8700008003700C2088800060037008F81E900C1
:10F8800042102000D11E2000A0152A0004FB020017
:10F89000000000000080FA00000006003800FA00B6
:10F8A000889FBE008A9FBE008C1F7800B0AF9F006B
:10F8B000C2AF9F00D3AF9F00E1AF9F006000B800D0
:10F8C0006011B800F09F9F0081A79F0092A79F0042
:10F8D000A3A79F0060FC2F000080470061172A004B
:10F8E0000700090031187800BFAC9700EC8F540076
:10F8F0000500360063FD2F008F814100421020007B
:10F90000211020000C0037000900780036FF0700A6
:10F910004200DD000080E8008139230061007800AA
:10F920000018A30007003A0063FD2F008F814100FB
:10F930003210200061102000A0152A0004FB0200F4
:10F94000000000006FAC97000800E00013003200D8
:10F95000E30F540011003200E60F54000F00320094
:10F96000E90F54000D003200E10F44001D00320089
:10F97000E20F44001B003200E30F44001900320084
:10F98000E40F440017003200C3FD2F008F814100B7
:10F9900052102000B1102000E7FF37004FA8970059
:10F9A000DFA897006011B8000005EB0006003700E3
:10F9B000A4002000050020006033B800A604020067
:10F9C000000000000A05E80069021400840F5500D9
:10F9D000F7FF3500F09F9F0081A79F0092A79F002F
:10F9E000A3A79F00E88F54007A003C008040EB0002
:10F9F0000900780083FE07006FAE97000C00E0005E
:10FA0000610035007F9C97008FA497001FA5970089
:10FA1000AFA5970006FA0200000000000002BE0039
:10FA20006033B8000440E10005C8E10006D0E10001
:10FA300007D8E100150039007F9C97008FA497003C
:10FA40001FA59700AFA5970006FA0200000000006E
:10FA50006011B80004F02F00F50F20006033B800EB
:10FA6000A6040200000000000040E10001C8E1001F
:10FA700002D0E10003D8E10004003E002AFC2F0080
:10FA80000F0545000006EB0006003700E3FB2F00E2
:10FA90008F81410012102000D1112000A6FF3700F5
:10FAA0000C06E8007F9A97008FA297001FA397008B
:10FAB000AFA39700F4AF9F0085B79F0096B79F0054
:10FAC000A7B79F0006FA0200000000000004BE0075
:10FAD0005A00BE006011B800B0B79F00C1B79F00C8
:10FAE000D2B79F00E3B79F00F4FF2F00050020006E
:10FAF0006033B800A6040200000000000802BE0047
:10FB00006033B800A6040200000000007FAA97003E
:10FB10008FB297001FB39700AFB397000020E100AA
:10FB200001A8E10002B0E10003B8E100DCFF3E0003
:10FB30007F9C97008FA497001FA59700AFA5970003
:10FB400006FA0200000000006011B8003FB2970002
:10FB5000CFB297005FB39700EFB39700A6040200FF
:10FB6000000000000203BE000002BE000800BE004C
:10FB70000A01BE00C8050200000000000205BE0028
:10FB80000004BE000C0037004FAC9700DFAC9700BC
:10FB9000E10F4400E08F5C000500360083FD2F007C
:10FBA0008F814100121020007112200062FF370087
:10FBB0000C86EA006055B8008C0078003FA89700DA
:10FBC00035FE0700880078003FA89700EFFD07008A
:10FBD0007600370011C0B3000900780009FE070065
:10FBE0006FAD97000A00E000600035007F9C970031
:10FBF0008FA497001FA59700AFA5970006FA0200F3
:10FC0000000000000002BE006033B8000440E100C4
:10FC100005C8E10006D0E10007D8E1001600390070
:10FC20007F9C97008FA497001FA59700AFA5970012
:10FC300006FA0200000000006011B80004F02F0076
:10FC4000F5FF2F00F60F200007002000A604020099
:10FC5000000000000040E10001C8E10002D0E10026
:10FC600003D8E10004003E002BFC2F008F854500E7
:10FC70000005EB0006003700E3FB2F008F814100F9
:10FC800012102000A11320002BFF37000A05E80006
:10FC90007F9897008FA097001FA19700AFA19700B2
:10FCA000B0B79F00C1B79F00D2B79F00E3B79F00D6
:10FCB00006FA0200000000005B04BE000801BE005E
:10FCC0009A040200000000000002BE006033B80089
:10FCD0003FB09700CFB097005FB19700EFB19700AA
:10FCE000C805020000000000F4FF2F00F5FF2F0000
:10FCF0006033B8000400E1000588E1000690E100EF
:10FD00000798E100E1FF3E007F9A97008FA29700DD
:10FD10001FA39700AFA39700B4B79F00C5B79F007C
:10FD2000D6B79F00E7B79F0006FA02000000000068
:10FD30000002BE006033B8003FB09700CFB097001C
:10FD40005FB19700EFB19700C80502000000000006
:10FD50000802BE006033B800C805020000000000C1
:10FD60000203BE000002BE00040037000A85EA005C
:10FD70004FAA9700DFAA97006033B8008A00780086
:10FD80003FA89700F4B79F0085BF9F0096BF9F00D4
:10FD9000A7BF9F00C0FD07007FB297008FBA9700F2
:10FDA0000401BE003FA89700F8FD07006011B800ED
:10FDB0003FA8970093FE07004F0678004F05BE004E
:10FDC0004F04BE000080FA00000006000200FA00A6
:10FDD000F0BF9F00CF80DE00EA0F5000E08F580098
:10FDE0001F003E00006001000A0037000B003700D2
:10FDF00010003700110037001700370018003700D7
:10FE000017003700160037001500370006003700CE
:10FE10000C00370000088000010037003008800027
:10FE20008000EB001400370032088000400880009A
:10FE30000600370050088000F9FF3700A008800056
:10FE4000F7FF3700A2088000B0088000800078002B
:10FE50000200780008003700C0088000F0FF37007B
:10FE60008F81E9004210200051212000A0152A00B6
:10FE700004FB0200000000000080FA000000060001
:10FE80000400FA00E0BF9F00F1BF9F00E18F500027
:10FE9000040036008F81E9006210200091222000CA
:10FEA0003E0037006FB99700CF91DE00EA0F510096
:10FEB000E08F590036003E00026001000A00370062
:10FEC00012003700190037002100370028003700E2
:10FED0002F0037002E0037002D0037002C00370090
:10FEE0000900370019003700E18060008180400080
:10FEF000200880000010A100008070002008880009
:10FF000005A1A9002800370013A1A900E180600025
:10FF100081804000800880000010A10000807000F7
:10FF20008008880011A1A9001F003700E18060004F
:10FF300081804000900880000010A10000807000C7
:10FF40009008880013A1A9001700370021A1A9007B
:10FF5000E180600081804000F00880000010A10076
:10FF600000807000F00888001FA1A9000E00370073
:10FF7000E180600081804000000980000010A10045
:10FF8000008070000009880021A1A9000600370048
:10FF9000E48157004210200011262000A0152A00FD
:10FFA00004FB0200000000000080FA0000000600D0
:10FFB0000200FA00F0BF9F006101B900EA0F510092
:10FFC000E08F59002F003E00026001000A00370058
:10FFD00010003700160037001C00370022003700E1
:10FFE000280037002700370026003700250037009B
:10FFF0000800370015003700E1806000C608DD000A
:020000040001F9
:10000000200880000060A1000080700020088800A7
:1000100022003700E1806000C608DD008008800013
:100020000060A10000807000800888001B0037007D
:10003000E1806000C608DD00900880000060A1003B
:10004000008070009008880014003700E180600094
:10005000C608DD00F00880000060A100008070008C
:10006000F00888000D003700E1806000C608DD0060
:10007000000980000060A100008070000009880075
:10008000060037008F81E90042102000412920003E
:10009000A0152A0004FB0200000000000080FA0006
:1000A000000006000400FA00889FBE008A9FBE0080
:1000B000A0BF9F0001047800B2BF9F000005780038
:1000C000EC0F550004003600EC8157004210200070
:1000D000812A200007003700BFBC97000900E90013
:1000E000E60F500006003600EA815700220020008B
:1000F000912A2000A0152A0004FB02000000000045
:100100000A00780038FD07004200DD008139230035
:1001100088307800CFD5DE00EA0F5500E08F5D0013
:1001200037003E000A6001000A0037001200370065
:100130001A0037002100370029003700300037004F
:100140002F0037002E0037002D0037001300370036
:1001500023003700E7846400CC4CDD00F0FF28006A
:10016000A400B60000807400200588008460A90007
:100170009460A80026003700E7846400CC4CDD00C2
:10018000F0FF2800A600B60000807400300588004B
:1001900084E0A90094E0A8001D003700E784640013
:1001A00080FF2F00A800B600008074004005880082
:1001B0008500A9009500A80015003700E7846400B9
:1001C000CC4CDD00F0FF2800B000B60000807400C9
:1001D000800588008760A9009760A8000C003700A0
:1001E000E784640080FF2F00B200B6000080740036
:1001F000900588008780A9009780A8000400370038
:10020000EC81570042102000D12E2000B9FF3700AA
:100210004F05BE004F04BE000080FA00000006003B
:100220000200FA00F0BF9F00CF80DE00EA0F50000E
:10023000E08F58002A003E00006001000A003700ED
:100240000F00370014003700190037001E00370078
:10025000230037002200370021003700200037003C
:100260000D00370018003700A00480004300DE00B6
:10027000610060009460A8008460A8001E00370040
:10028000A00480004700DE006100600094E0A80048
:1002900084E0A80018003700A00480004800DE00B9
:1002A000610060009500A8008500A80012003700DA
:1002B000B00480004B00DE00610060009760A80081
:1002C0008760A8000C003700B00480004C00DE00FE
:1002D000610060009780A8008780A80006003700B2
:1002E0008F81E90042102000F1332000A0152A0080
:1002F00004FB0200000000000080FA00000006007D
:100300000200FA00F0BF9F00CF80DE00EA0F50002D
:10031000E08F58001E003E00006001000A00370018
:100320000C0037000E0037001000370012003700B5
:10033000170037001600370015003700140037008B
:10034000070037000C003700200480004300DE0067
:100350000B003700200480004700DE000800370053
:10036000200480004800DE000500370030048000D3
:100370004B00DE0002003700300480004C00DE003D
:10038000610060000080FA000000060006003700EF
:100390008F81E9004210200011372000A0152A00AB
:1003A00004FB0200000000000200FA00F0BF9F0002
:1003B0006101B900EA0F5100E08F590038003E009A
:1003C000026001000A003700110037001A003700F0
:1003D0002100370028003700310037003000370097
:1003E0002F0037002E00370013003700220037009F
:1003F000200480004300DE0061006000E1806000B6
:10040000C308DD00220480000230A100070037008D
:10041000200480004700DE0061006000E180600091
:10042000C708DD00220480000270A1000281700074
:100430002204880020003700200480004800DE00ED
:1004400061006000E1806000C808DD0022048000D7
:100450000280A100F5FF3700300480004B00DE0071
:1004600061006000E1806000CB08DD0032048000A4
:1004700002B0A10007003700300480004C00DE000D
:1004800061006000E1806000CC08DD003204800083
:1004900002C0A1000281700032048800060037000B
:1004A0008F81E90042102000613B2000A0152A0046
:1004B00004FB0200000000000080FA0000000600BB
:1004C0000200FA00F0BF9F00CF80DE00EA0F50006C
:1004D000E08F58001B003E00006001000A0037005A
:1004E0000C0037000E0037001000370012003700F4
:1004F00014003700130037001200370011003700D6
:10050000070037000C0037009460A9008460A90040
:100510001200370094E0A90084E0A9000F00370022
:100520009500A9008500A9000C0037009760A9007C
:100530008760A900090037009780A9008780A9007B
:10054000060037008F81E90042102000913F200013
:10055000A0152A0004FB0200000000000080FA0041
:10056000000006000600FA00889FBE008A9FBE00B9
:100570008C9FBE00F0B79F008106780000057800D0
:10058000EC0F550004003600F281570042102000A5
:10059000210C2000100037000A00780082BF9F0065
:1005A00093BF9F0010FC0700000678004264DD0046
:1005B0000880E80081392300610078000FB99700B6
:1005C0009FB997000008A30006003A00F281570087
:1005D00022102000610C2000A0152A0004FB02005C
:1005E00000000000AB39230008844500980478001F
:1005F0000910A0000900A100090C78000A00780089
:1006000082BF9F0093BF9F00FCFB07000FB99700BC
:100610009FB997000000E000060032000C06E800D9
:100620004266DD008C8545001B00A1001820A0005B
:10063000020037000920A100090C78007FB0970064
:1006400082BF9F0093BF9F009DFF07008D00780031
:100650000FB997009FB997007FB097008FFC0700F4
:100660008000EB007FB0970005FE07008000EB00E4
:100670007FB097004EFE07004F06BE004F05BE003C
:100680004F04BE000080FA00000006000200FA00DD
:10069000F0BF9F00CF80DE00EA0F5000E08F5800CF
:1006A0001B003E00006001000A0037000B0037000D
:1006B0000C0037000D0037000E0037001400370023
:1006C0001300370012003700110037000300370015
:1006D00006003700210880000700370081088000ED
:1006E000050037009108800003003700F108800002
:1006F0000100370001098000C408DE00E3806000CB
:1007000000042000E28F500007003A000D0037007F
:100710008F81E9004210200091422000A0152A009C
:1007200004FB02000000000000102000E38F5000D6
:100730000400320080002000E18F500001003200F0
:10074000100020000080FA0000000600AA24AB0080
:100750000D003200308280001041900001C8B300CB
:10076000814F510007003A008182800011419000C2
:1007700041C8B300814F510002003A00E8C0400078
:1007800011409800AA24A9000008200050248800E5
:100790000000060000C8B30001032100914F1000C3
:1007A0002E003A00C005210001CCB30001487800BA
:1007B0003103210091407800E2CF50000800320060
:1007C000E3CF500015003200E1CF500022003A0084
:1007D00000122100D0828800200120001A0037007A
:1007E000200321001080FB0000004000E11B2100DD
:1007F000E1007800D1828800D1828000E0052100EC
:10080000A140900001487800D18280000000E800FB
:10081000B14090000148780000000600210321004B
:1008200022C0B300914F110009003E001180FB006F
:1008300000004000011C2100E1007800D182880006
:10084000D08280001080FB00F0828800000006004B
:100850000048EB00000006000048EB000000060026
:10086000800321000048EB008000E8008048EB0096
:100870000103210091407800FFC060008180FB00EF
:10088000E18F50000D003200E28F50000F00320067
:100890000100E00025003A00E18280000170A00024
:1008A000E18288001004A00011848000E18F5000D4
:1008B0001E003A001014A0001C003700E0828000E7
:1008C0000070A000E082880018003700E0828000FD
:1008D0000070A000E0828800400321001004E000C6
:1008E00006003500104078006F4060000080FB007B
:1008F00000004000A10421000500370010407800EE
:100900006F4060000080FB000000400001052100F6
:1009100061007800104090000028A300030032001E
:1009200011C0B3008003210001487800E0828000FC
:100930000078A3000800320080032100D0828800E4
:10094000E08280000000A000E082880021C0B300A7
:10095000E00521000148780000000600F1828000D7
:1009600080C0B300E78F50000B003E00F082800093
:1009700011C0B3005650E2000500320061052100AD
:1009800091407800E1CF500003003A0021C0B3004D
:100990006205210001497800F28280008080FB001E
:1009A00081005100F18288008182800080487800B7
:1009B0008103210041838800E18280000108A300B7
:1009C000070032000F003700D18280004283800090
:1009D0003159780042838800D18288000040E900C4
:1009E0000004E000F8FF3A0000000600D182800019
:1009F000428380003159780042838800D182880088
:100A00000040E9000004E000F8FF3A0000000600A2
:100A1000881F780000052100818280001104780081
:100A20004E44DE00614464001024A2000082800075
:100A3000E80F500008003A00200321001080FB005E
:100A4000B0248800000120009604E20001003A0072
:100A5000400020000082880058D0BF00E14F5000C5
:100A600011003A008103210080828000110098006B
:100A7000BAFF070061052100914078008082800064
:100A8000E2CF500002003A0041C8B3000400370032
:100A900081CCB3000804E0000100320081C8B3003B
:100AA0001140980012003700200621001004E000D9
:100AB0000E003D00E30040009181FB006400400017
:100AC0001081FB004811DD00028171000500320039
:100AD0009180FB001080FB004800DD00008070006A
:100AE00000000100200621001074A1005870EF00E2
:100AF0004F047800000006000080FB000181FB002D
:100B000000004000000141004311DD00030021000E
:100B10000301410012F0A1000104E00002003A00CC
:100B2000A104210001003700010521008230780076
:100B300012E0A1006401410012E0A00000000600E4
:100B40008430EF000001EB008000EB004007200044
:100B50003EF50200000000008284A9000001200090
:100B600000248800000006008284A8000001200004
:100B70005024880010002000208488000001EB0031
:100B80008000EB00500720003EF50400000000004C
:100B90000200FA00881F78002003210011C0B30072
:100BA00090CF10000F003A000080E900104078005C
:100BB0007F4060000B003A00E08280000070A000DF
:100BC000E08288001003210032C0B300904F110072
:100BD00003003A0010002000108488000100370054
:100BE0008230EF00200321001004E0009A003A0058
:100BF0000080E900104078007F406000E24F500024
:100C000095003A004003210010417800EF40610058
:100C10009100320010417800EF4061008180FB00BC
:100C2000E28F50008C003C00010220000282800014
:100C3000810F510088003A00E18280000170A0001D
:100C4000E18288001004E0000C00350010417800BB
:100C5000EF4061008180FB0081804000A204210000
:100C600062817800E2BF9F00104078006F40600012
:100C70000080FB00210721000B00370010417800A5
:100C8000EF4061008180FB0081804000020521006F
:100C900062817800E2BF9F00104078006F406000E2
:100CA0000080FB00E1062100614478000808A300F1
:100CB00004003A004FF897000024A100C0FF9F00F5
:100CC00003003700CFF897000124A000C1FF9F0068
:100CD000400321001004E0000600350010407800B9
:100CE0006F4060000080FB0000004000A104210074
:100CF00005003700104078006F4060000080FB0066
:100D000000004000010521006FB997008230780093
:100D10001003210031C0B30090CF100017003A003B
:100D20006FB897001000E0000F003D004003210065
:100D30001004E0000500350010407800EF4060002E
:100D40008180FB002207210004003700104078005A
:100D5000EF4060008180FB00E206210062C0780065
:100D60000014A00000F178006FB8970010419000C7
:100D700041C8B30081407100360037004FF9970039
:100D80000224A200C2FF9F00EFB89700114090001C
:100D90001100E00008003D000074A1000064A00004
:100DA0009040980022002000500020003EF50200F4
:100DB00000000000020037000064A000904098008E
:100DC0004FF897000024A200C0FF9F000818A3005E
:100DD00006003A006FB89700024028001001610039
:100DE00001002800810F510018003A004003210043
:100DF0001004E0000500350010407800EF4060006E
:100E00008180FB0022072100040037001040780099
:100E1000EF4060008180FB00E206210062C07800A4
:100E20000014A10000F17800EFB897001140900085
:100E3000B043B200904098002200200050002000F3
:100E40003EF50200000000000300370090409000D3
:100E5000B143B200114098004F0478000080FA00BE
:100E600000000600E08280000070A000E0828800A0
:100E7000AC24EF00AE24EF000000EB0001002100E5
:100E80004201DD00028140000009EB0032117800D0
:100E90000000E800EC0F5000F8FF3A009424A8008E
:100EA0004470EF009424A90068804000808288008C
:100EB000318288004182880020032100104178009F
:100EC0002104210082487800000120004250E20005
:100ED0000600320012002000210421001000200032
:100EE0003EF50200000000000002200000828800A1
:100EF000000006000003210001C6B30010C060001E
:100F00003C003A00100321001080FB008000EB0041
:100F1000EB0F5000E08F580036003E0000600100EB
:100F20001500370015003700320037001300370076
:100F300030003700060037000B003700280037006C
:100F40000B003700090037000D0037001B00370089
:100F5000E08280000070A000E08288008000200015
:100F600000828800000006000AFE3700BDFF37003F
:100F7000200421000600370039FE370004FF370047
:100F8000400321009080FB004004210000804000CD
:100F9000D0828800E08280000000A000E08288000B
:100FA00011C0B300E005210001487800E082800014
:100FB0000070A000E082880000000600E08280004F
:100FC0000070A000E0828800400321001080FB0038
:100FD00041042100220321009270780000000600E5
:100FE0000001EB008000EB00200020003EF5020035
:100FF00000000000000006009EC0A9008EA4EF00C3
:101000008AA4EF00AA24EF00AC24EF00AE24EF0086
:101010002000200030258800A824EF008644A90085
:10102000F009200080248800602488008804A8003B
:10103000000021004800DE00C02488000000EB0012
:10104000C200DD0002002100810041008008EB00A9
:10105000B11078000000E800EC0F5000F8FF3A00F3
:101060009424A8009624EF0094A4A9009424A90035
:101070000C0037008000200050248800C0052100AB
:101080000048EB00200621000048EB000000E800CB
:10109000904078000048EB000000E80090407800A5
:1010A0000048EB008A64AB00F2FF3A001000200019
:1010B000C0838800D08388007C30EF007E30EF0052
:1010C0008430EF00E2042100810421000000EB00E5
:1010D0008001EB000029EB008028EB00E4062100F2
:1010E0000372780024072100037278000000E800F2
:1010F000E30F5000F6FF3A00800021008082880054
:10110000D0002000502588000003210010808800B6
:1011100081C0B300000021000148780041C8B3003D
:101120000000E800014878004270EF004030EF0016
:10113000000006007810E20023003A0010002000B2
:10114000C08388007A10E2001F003A00D083880034
:101150008105210091407800E2CF500006003A005E
:10116000808280000048EB0081CCB3008082800048
:101170001140980000000600810521009140780090
:10118000E1CF500010003A008030EF0082C0B30081
:101190003182800082487800338280000103210080
:1011A0009101980044C8B3009441980000848800DD
:1011B0004082800002487800408280001100980040
:1011C00001C8B30011409800000006003082800082
:1011D00090407800320621001282FB000200E800F5
:1011E0009081FB00C819DD00830172000182FB00C1
:1011F000830F5200020036009280FB001080FB003B
:10120000320621001282FB000200E8009081FB0000
:10121000C819DD00830172000182FB008481510046
:101220001242780003497800C819DE0010417800A6
:10123000034878000000EB000E0037000406210090
:101240009482FB008401E8001381FB004811DD005B
:10125000028172008503210065597800944278006C
:10126000024A78004811DE00134278008249780073
:101270000000E80080CF5000F0FF3E003006210063
:101280001080FB00410621009180FB00C808DD00B2
:1012900081007000408280000D00320081C0B300E8
:1012A00001487800408280008103210011009800ED
:1012B0003182800011E8A30002003A0081CCB30023
:1012C0000100370081C8B3001140980000000600FB
:1012D00081C0B300014878004082800001032100F2
:1012E0001100980041C8B300114098005106210038
:1012F0009181FB000100E8001081FB004811DD0036
:1013000002817100050032009180FB001080FB001B
:101310004800DD0000807000000001002006210070
:101320001074A1007610E20001003A0081FF07006E
:101330000000060058D0BF00E24F500001003A0004
:10134000A2FF37005870EF008010E20009003A0059
:1013500081C0B30040828000014878004082800054
:101360000103210011009800C1C8B300114098008A
:10137000000006008030EF00000006007C30EF0027
:101380007E30EF0058D0BF00E24F500008003A0016
:1013900081C0B30040828000014878004082800014
:1013A000810321001100980081CCB30014003700A4
:1013B000610321001181FB000100E8009081FB0026
:1013C000C819DD0083017100F2828000828F510014
:1013D000050031009180FB001080FB004800DD001B
:1013E00000807000F08288005CFD0700810321000E
:1013F000808280001100980081CCB3008082800040
:10140000114098000000060094A4A900E08280002A
:101410000078A30017003A00200621001004E00025
:1014200008003D0020C0B30058F0B7007E10E20075
:1014300001003A00D1FF07007A30EF007830EF006A
:101440000000060081C0B30040828000014878009F
:10145000408280000103210011009800C1C8B30040
:1014600011409800E8C05000808280001140980030
:1014700000000600010321001104E0000A003D0005
:1014800010C0B30058F0B7007C10E20001003A0031
:10149000BAFF07007A30EF007830EF007610E200F4
:1014A0000F003A0023FF370020C0B30058F0B70008
:1014B00082C0B300408280000248780040828000F1
:1014C0001100980041C8B300114098007A30EF0035
:1014D0007830EF007610E20001003A0015FF0700B7
:1014E000000006005670EF007630EF007C30EF0011
:1014F0007E30EF008030EF005870EF0000052100D3
:1015000010017800924090000174A10011419800F0
:101510001024A20010017800924090000174A100F4
:10152000114198001024A2004182800011409000D7
:101530000074A10090409800C00521000048EB0015
:101540000000EB00F082880021062100804878002E
:101550008100E80011417800804878008100E800AF
:10156000114178008048780062FE07000001EB001E
:101570008000EB00300020003EF50200000000007B
:10158000A1FF3700D0C2B30086F0B7006CD0BF0017
:10159000B00FB2001A003A006CD0BF00C00FB2000A
:1015A0000100210001004000308288004082880054
:1015B0004850AA0002C0230010016100014023002E
:1015C000810F51000D003A00010321000101780054
:1015D000E8814000100290009458780010029000BA
:1015E0000402E80014009800838F5000F9FF3A00CD
:1015F0003082800012009800BAFF37004DFF37009C
:101600006CD0BF00B00FB200E80F500001003A00EC
:10161000FFFC070000000600889FBE008A1F7800BC
:1016200000447800814478000985FB000A38A30053
:10163000030032008040EB00084078002EFD0700D8
:101640000A28A3000300320011C0B300084078004C
:1016500029FD07000884FB0008044400A04A20007C
:1016600009707C004F0578004F04BE0000000600A2
:101670000004E0000B003A0081C0B300408280000B
:101680000148780040828000010321001100980089
:10169000C1C8B30011409800E8C0500080828000AB
:1016A0000F0037008180FB000080FB00000040003D
:1016B000008040004300DD00020021008201400064
:1016C0001342900041C8B300014272009441980057
:1016D0006400400002004000104190008140710011
:1016E00011409800000006000082FB000104E000A9
:1016F0000300320004024200050521000200370009
:1017000004024200A504210065027A008002EB0079
:101710000400E0001400320012029800034A78002E
:10172000144190000244B20012429800944190008B
:1017300082C8B30002C17100124298000080FB0011
:101740000104E00003003200000040000105210018
:101750000200370000004000A10421000100400009
:101760001024A20084027800050078000000060022
:1017700094A4AB00170032000080FB000000400082
:1017800001052100610178001203BE00040420005D
:10179000060362008003EB000689BE00E1027800C8
:1017A0001501BE000260A200828ABE000101400055
:1017B0001224A20061017800924190000344B2001B
:1017C00013419800610078009040900004C26800C6
:1017D00014409800000006009424EF008C24EF00D1
:1017E0004030EF00000006004010E20010003A0018
:1017F0009424EF008C24EF00200020003025880086
:10180000A824EF008644A900F00920008024880065
:10181000602488009EC0A800010037009404A8003E
:101820009404AB00FDFF320010002000008288000D
:1018300000000600A0009000910078008180400028
:101840001C0037000181400020029000020242008B
:10185000940278004C29DE008001EB006201510007
:10186000E0815900E90F5100E08F590011003E005E
:10187000026001000B0037000E0037000D0037003A
:1018800008003700070037000A003700090037005A
:101890000800370001003700040037000590A10060
:1018A000050A78008180E80003003700E3804000EB
:1018B000010037008100E80010019000828F500085
:1018C000E0FF390000000600E10F51000600320081
:1018D00003003900E20F510009003A00060037000A
:1018E0000100EA00000006000100780000F0A700F7
:1018F0000000EA00000006000180EA000000060087
:1019000011002000F8BC02000000000000000500EB
:10191000881F780000047800611AB800F10F5200A7
:10192000E08F5A0064003E0004600100110037009F
:10193000120037001300370014003700150037007D
:10194000160037001A0037002E0037002F0037002E
:101950003000370031003700350037003A003700DB
:101960003D00370040003700430037004600370095
:10197000490037000208DD00540037000288DE000D
:101980005200370001004100500037000280500033
:101990004E0037000190B9004C0037000200E00013
:1019A00005003200110009008200D800470037000E
:1019B0000200E0000F003A00E0A029000000E00073
:1019C000040032008000EB00080078000E9A02004C
:1019D0000000000023002000730498007001440000
:1019E00071002900080078002AD3020000000000DE
:1019F00035003700110009008200D8008000FD008A
:101A000032003700028070003000370001006900AA
:101A10002E003700010061002C0037008280680032
:101A200001F0A7008100EA008100E900040037000E
:101A30008280680001F0A7008100EA008100EA00CE
:101A40004F08DE002100370010002000828F500078
:101A50001E003C001C00370010002000828F500048
:101A60001A003D001800370010002000828F50003F
:101A7000160035001400370010002000828F50003F
:101A80001200340010003700100020000100E000B8
:101A9000040032000D0037000000EB000100E00000
:101AA0000A00320002F0A7000201EA000200EA0088
:101AB0004F00DE00050037002100200008007800FC
:101AC000F8BC0200000000000000EB004F047800AA
:101AD000000006008000EB000108980071009800EB
:101AE0002118980020019000010978003001900031
:101AF00002014100400090006C070400000000005B
:101B000020019000920178001000200009003700A9
:101B10000002400062027A00810F520004003A0085
:101B20000000E800000040006200780000000600AD
:101B30000080E800830F5000F5FF39000000050029
:101B40000600FA00889FBE008A9FBE00000478004D
:101B500008089000A800900000004000E104780010
:101B6000780090000008A30004003A0081002000E3
:101B700008007800F8BC0200000000004C48DE00BD
:101B80008000EB00EE0F5000E08F580077013E0020
:101B9000006001000E0037001100370021003700FF
:101BA00038003700550037006E0037008A003700D4
:101BB000BB003700CB003700E2003700EF003700F2
:101BC000250137003F013700440137005801370035
:101BD000780090000000A1007004980067013700B1
:101BE000C44CDD00C4CCDE00980890008100E80001
:101BF00058009000808F5000040039004100200000
:101C000008007800F8BC020000000000E800900026
:101C1000180890000000E800100C98000000400038
:101C200032003700980890008100E80058009000CA
:101C3000808F500004003900410020000800780027
:101C4000F8BC020000000000680190001808900035
:101C50000000E800100C9800000040008808900088
:101C60008100E800A801900081804000E3807800B6
:101C700001317800080890000080E800000C98000E
:101C80003E013700F0FF2000808464009808900037
:101C90008100E80058009000808F50000400390057
:101CA0004100200008007800F8BC0200000000009D
:101CB00038009000808F540004003900610020003B
:101CC00008007800F8BC020000000000E800900066
:101CD000180890000000E800100C98000000400078
:101CE0004801900089844400E2847C0089307800B7
:101CF000080890000000E800E0FF3700F0FF200037
:101D000080846400180890000000E00004003D009A
:101D10005100200008007800F8BC0200000000001C
:101D200038009000808F54000400390061002000CA
:101D300008007800F8BC02000000000018089000BD
:101D4000C800900089844400E80190000001400030
:101D50006301790082B07C000000E900100C98005B
:101D6000E3FF3700180890000000E00004003D0089
:101D70005100200008007800F8BC020000000000BC
:101D8000880990000300E800A800900000004000CF
:101D90006101780098089000818040006800900000
:101DA0008100400011007800820F500003003900CC
:101DB00093BF9F00A2BF9F001E003700F2FF2000CC
:101DC0008284640009004000480190000000400047
:101DD000E2087800A7FF3700180890000000E00034
:101DE00004003C005100200008007800F8BC02000C
:101DF00000000000080990000200E800A800900020
:101E000000004000E1007800E80190001808900010
:101E10000002E9000402420063027A000000400070
:101E200063007800810F50001300390092BF9F00BB
:101E3000A1BF9F00B0BF9F00200020007004980049
:101E4000630020006E8157006100290008007800BF
:101E50002AD3020000000000E0A029000000E000FA
:101E6000C60032008000EB00080078000E9A0200E5
:101E700000000000C1003700F1FF200081846400F1
:101E800009004000C8009000000040008430780045
:101E9000180890000080E900100C980075FF3700CA
:101EA000180890000000E00004003D0051002000F0
:101EB00008007800F8BC020000000000090178006A
:101EC000F20FB20018089000E800900000004000F7
:101ED000E1007800080078007BFE07009808900079
:101EE00014003700180890000000E00004003C00D7
:101EF0005100200008007800F8BC0200000000003B
:101F00006800900098089000018140008100E9007D
:101F1000818040008981FB0060017900E0807800C9
:101F2000080078007AFE0700980890008100E90018
:101F3000110C9800680190008180400000B1780089
:101F40006BFF3700C44CDD00C4CCDE008808900075
:101F50008180440018009000808F500004003900F8
:101F60007100200008007800F8BC020000000000AA
:101F700008089000890440006B00370018089000A2
:101F80000000E00004003C00510020000800780040
:101F9000F8BC020000000000680090009808900063
:101FA000018140008100E900818040008981FB00BF
:101FB00060017900E08078000800780054FE070096
:101FC000980890008180E900110C98008808900022
:101FD0000000E000050032000930B2002A002000B5
:101FE00002302000828F540006003A002801900041
:101FF0008101E80083814100628579000000E000F2
:1020000005003200818040002800900081004000DF
:102010001190A00003003700818040008100410042
:102020001190A100880890008100450018009000E0
:10203000808F5000040039007100200008007800F3
:10204000F8BC020000000000080890000A054000EB
:102050000A0C98004900370028009000880890007A
:102060000101E80002014100E00579008180E800FB
:10207000818040006085780040202000800F55005E
:1020800004003600A100200008007800F8BC02001F
:10209000000000008B854500480190000B014100C5
:1020A000F1FF2000818064008A014500080078006B
:1020B0002AD30200000000000808900063004000DE
:1020C000EEFE3700F1FF20008180640008007800F8
:1020D0007ABB02000000000005FF3700F0FF20007F
:1020E00080846400980890008100E8005800900007
:1020F000808F500004003900410020000800780063
:10210000F8BC020000000000E800900018089000F1
:102110000000E800100C9800000040000080400023
:10212000880890000108E800090C980013003700A7
:10213000180890000000E00004003D00510020005D
:1021400008007800F8BC02000000000018089000A9
:102150006801900080004000E2807800010C980047
:102160000000E900100C9800040037003100200046
:1021700008007800F8BC0200000000004F05BE0017
:102180004F04BE000080FA00000006000000FA00C4
:10219000889FBE008A9FBE008C9FBE00000478000E
:1021A000810578000F0578000B00780060070200B9
:1021B00000000000800678006386460065804600C7
:1021C0000000A100808747008A047800E0A0290071
:1021D0000000E000040032008B0078000800780066
:1021E0000E9A0200000000002000200070049800F9
:1021F00008089000800C7800AD449800638044008B
:102200000D0178008B0078005207020000000000EA
:102210008C017800090178009100290008007800FD
:102220002AD30200000000008A0778004F06BE0093
:102230004F05BE004F04BE000080FA0000000600FB
:10224000A0199000000178008000EB000A00370020
:10225000A20A90000281E800000A9000848F5200D8
:1022600004003A00F00090000110A00071009800F6
:10227000100005008100E800838F5000F4FF390052
:1022800000000500889FBE000004BE00780090009A
:102290000020A000700498000900E0000D0032004A
:1022A000030037000800780025FE07008904E900D4
:1022B0007800900065006000E50F500009003A00CA
:1022C0000900E000F7FF3A00060037000800780038
:1022D0001BFE07007800900065006000E50F5000CD
:1022E000FAFF3200780090000020A10070049800EE
:1022F0004F04BE0000000600889FBE000004BE0020
:1023000018009000808F54000400390091002000D4
:1023100008007800F8BC020000000000A818900037
:102320000040EB00EF8F500006003E006A80400046
:1023300000004000093478008100E800211C98006A
:1023400010C0B3004F04BE0000000600201A900029
:10235000800178000001EB0012003700A30A900012
:102360008381E800818F52000D003A008401E9006A
:1023700023189800EA0041008180400001004000DD
:10238000040037000201E8000080E80090007800B7
:1023900071B89F00830F5100FAFF3900100005004B
:1023A0000201E800840F5100ECFF39000000050035
:1023B0008000EB0021189800000006000400FA00DD
:1023C00080089000E1BF9F00F0009000F1BF9F00E7
:1023D0004300200064815700A10029002AD3020095
:1023E000000000000080FA0000000600889FBE0088
:1023F0000004BE00780090000020A0007004980047
:102400000900E0001B0032000700370008007800D8
:102410008BFF07000000E0000E003A000800780083
:10242000C7FD07008904E90078009000650060009E
:10243000E50F500013003A000900E000F3FF3A00F6
:1024400010003700080078007DFF07000000E00062
:1024500006003200780090000010A0007004980080
:1024600008007800D5FF0700090037000800780051
:10247000B3FD07007800900065006000E50F500094
:10248000F0FF3200780090000020A1007004980056
:102490004F04BE0000000600F00190000001EB00B8
:1024A0000308A300090032000318A30007003A0044
:1024B000201990000200E00002003200CBFF07006C
:1024C000010037006FFF07001200200002007800B3
:1024D00000000600889FBE00000478000800780015
:1024E00087FD0700800478000900E0001300320037
:1024F000780090000008A30006003200700144003C
:102500002300200081002900080078002AD302005F
:1025100000000000090C98000080EB00100C9800EF
:10252000780090000000A000700498000018A3003C
:102530000200320008007800A0FF070009007800C0
:102540004F04BE00000006000600FA00889FBE008F
:102550008A9FBE000004780000002A00808F50008F
:1025600004003A0040002000920F1000AC003E0032
:10257000A800370010012A00808F500006003A00A2
:102580005000200090BF9F00230020006E81570064
:10259000C1002900650037000300E000A000320000
:1025A00012007800980F50009D003A000285E80064
:1025B0008305E900F2FF2500F3FF2F0002804000B1
:1025C000E0804900EF0F5000E08F580094003E007B
:1025D000006001000F003700210037003000370095
:1025E0003B00370040003700450037003B00370014
:1025F00045003700510037005400370056003700BF
:1026000064003700770037007A0037007D0037001C
:10261000800037009A0478008B05E9008980450026
:1026200018009000808F50000400360071002000D8
:1026300008007800F8BC0200000000008984440013
:102640000000EB00040037000000E800A800900044
:10265000DAB07C008984E8008B0F5000FAFF390063
:1026600020002000700498000800780071FC07002A
:10267000C0112C000000E0000300320008007800C8
:102680001CC10200000000008080EB000800780000
:1026900090FF07000000E00061003A000F003700E3
:1026A000780090000010A1007004980008007800E5
:1026B00042FF0700C0B229000000E00058003200CD
:1026C000080078002C9B0200000000005400370036
:1026D000780090000010A0007004980008007800B6
:1026E00036FF07004E003700780090000008A30076
:1026F0004B0032000800780011FD0700F7FF37009B
:1027000020002000F4FF37009A007800A1BF9F004E
:1027100008007800F8FE07000080FB00B0BF9F00B3
:10272000430020006C815700B100290008007800A8
:102730002AD3020000000000390037009A00780018
:102740000800780001FF0700350037000800780016
:1027500017FF0700320037009A0478001A0590002E
:102760008900450038009000808F5000040036003A
:102770006100200008007800F8BC020000000000A2
:102780000A0178000800BE0058D3020000000000D3
:10279000230037009A0478008B05E9008980450002
:1027A00038009000808F5000040036006100200047
:1027B00008007800F8BC0200000000008984440092
:1027C0000000EB00040037000000E800C8009000A3
:1027D000DAB07C008984E8008B0F5000FAFF3900E2
:1027E0000F003700080078008ABB020000000000DC
:1027F0000B003700080078004EBB0200000000000C
:1028000007003700080078006EBB020000000000DF
:102810000300370008007800ACD30200000000007D
:102820004F05BE004F04BE000080FA000000060005
:10283000920078000100E00005003500B0FC0700C0
:1028400000F0A7000000EA008001E9001000370056
:1028500013002000F4FF2900848F50000D00360083
:10286000120190008001EB000402E800848F500008
:102870000800320071024200848F500005003200CF
:102880009001690003F0A7008301EA008301EA00D8
:10289000CF19DE000300780000000600627E2400ED
:1028A000F10F200012C86000124190001240980001
:1028B000827E2400928160002340980012419000A3
:1028C00032409800A27E240092806000414098002F
:1028D0001241900052409800917F2400914078006E
:1028E00061409800A17F24009140780071409800D9
:1028F000B17F24009140780001489800C17F2400F6
:102900009140780011489800C17E240091407800E1
:1029100021489800D17E24009140780031489800E9
:10292000E17E24009140780041489800F17E240027
:102930009140780051489800017F24009140780030
:1029400061489800117F24009140780071489800F8
:10295000417F24009140780001509800517F24006D
:102960009140780011509800317F24009140780008
:1029700021509800717F24009140780031509800D8
:10298000817F2400914078004150980000000600AB
:10299000889FBE008A9FBE000004BE000A4020003F
:1029A0000B0020000005450081854D000A0037001E
:1029B0000800BE007CCB020000000000F2FF2F00E8
:1029C000F30F2000820F5000838F580007003A0059
:1029D00062044400E0844C008A0F54008B8F5C003A
:1029E000F3FF39000000EB00010037001000200069
:1029F0004F05BE004F04BE00000006000001EB00C2
:102A0000110221000001200026F902000000000050
:102A100081012000607E240032F9020000000000E5
:102A20006AF9020000000000E17F24001100680044
:102A300000F0A7000000EA000000E9004F00DE00FF
:102A4000000006002E00FA0023FD2F008F814100B8
:102A5000D2022000BCCB0200000000009FA897001B
:102A60006380680000F0A7000000EA000000E900B1
:102A70004F00DE000080FA00000006001600FA0099
:102A8000889FBE008A9FBE000005BE007E044000F5
:102A9000E08448000A003700FE8157005201200000
:102AA0000800BE00BCCB0200000000000FE8970049
:102AB0000008A3000A003A006E044400E0844C00C1
:102AC00000402000010020000A0040008B804800E8
:102AD000800F5400818F5C00EFFF39006044B80024
:102AE0000800BE004F05BE004F04BE000080FA0083
:102AF000000006001600FA00881F78008A9FBE00BA
:102B00008C9FBE00000478000206BE008801780099
:102B1000D20220000C00BE00BCCB0200000000006E
:102B2000086890000040E800006C98007E054600B0
:102B3000E0854E00CA00370003FE2F008F81410060
:102B4000520120000A00BE00BCCB020000000000C1
:102B5000C86090006FE0970000C07000406498006B
:102B6000D86090007FE0970000C07000506498002B
:102B7000E86090000FE8970000C070006064980063
:102B8000F86090001FE8970000C070007064980023
:102B9000CFF097008180FB00286190000281FB004C
:102BA000386090004800DD000000710000804000A7
:102BB000206498004800DE0030649800BFF0970061
:102BC0008180FB00086190000281FB00186090008A
:102BD0004800DD00000071000080400000649800A3
:102BE0004800DE0010649800AFF097008180FB0081
:102BF000685990000281FB00785890004800DD0081
:102C00000000710000804000605C98004800DE0019
:102C1000705C98009FF097008180FB0048599000FD
:102C20000281FB00585890004800DD000000710050
:102C300000804000405C98004800DE00505C980036
:102C40008FF097008180FB00285990000281FB00E3
:102C5000385890004800DD000000710000804000FE
:102C6000205C98004800DE00305C9800FFE8970088
:102C70008180FB00085990000281FB0018589000E9
:102C80004800DD000000710000804000005C9800FA
:102C90004800DE00105C9800EFE897008180FB00A0
:102CA000685190000281FB00785090004800DD00E0
:102CB0000000710000804000605498004800DE0071
:102CC00070549800DFE897008180FB004851900025
:102CD0000281FB00585090004800DD0000007100A8
:102CE00000804000405498004800DE005054980096
:102CF000CFE897008180FB00285190000281FB0003
:102D0000385090004800DD00000071000080400055
:102D1000205498004800DE0030549800BFE8970027
:102D20008180FB00085190000281FB001850900048
:102D30004800DD0000007100008040000054980051
:102D40004800DE0010549800484990000281FB00C2
:102D5000D8499000C819DD0003007100684990004F
:102D60000281FB00F8499000C819DD008300710062
:102D70002FB1970000004100E0804800404C9800CF
:102D80004801DE00524C9800614C98004808DE0073
:102D9000704C9800084990000281FB00984990000F
:102DA000C819DD0003007100284990000281FB0072
:102DB000B8499000C819DD00830071001FB1970069
:102DC00000004100E0804800004C98004801DE000F
:102DD000124C9800214C98004808DE00304C9800B6
:102DE000484190000281FB00D8419000C819DD00E5
:102DF00003007100684190000281FB00F8419000DF
:102E0000C819DD00830071000FB197000000410078
:102E1000E0804800404498004801DE005244980099
:102E2000614498004808DE0070449800AFE89700BD
:102E30008180FB00284190000281FB003840900017
:102E40004800DD0000007100008040002044980030
:102E50004800DE00304498006E054500E0854D00D6
:102E600000402000010020000C0040008D80480040
:102E7000800F5500818F5D002FFF39004F06BE0087
:102E80004F05BE004F0478000080FA0000000600E5
:102E90004F03B000889FBE008A1F78008E1F780005
:102EA0000004BE00E00F5100E08F590006003A0018
:102EB0000F0078006003B100150009000018EB0056
:102EC0000058EB0003003700A0FC2F000F0040006B
:102ED00008FF070030002000D0A79F000800BE00B8
:102EE000ABFE07000000E000030032000800BE0057
:102EF0001ACC0200000000000005EB00A1FC2F002E
:102F00008F8040000A804000B0407800E1C79F00F9
:102F10006EFC2F000F074700306F780010407800DC
:102F2000104798003FA19700CFA197000800BE006E
:102F300054CC02000000000062044400E0844C0015
:102F400063054500D0022000800F5500EBFF3A00DA
:102F50004F0778004F0578004F04BE004F03B100C3
:102F60000000060000C0230011002000B5FE07008D
:102F70000000E00014003A000000240011002000CE
:102F8000B0FE07006011B8000000E0000800320049
:102F90000000240011002000B8FE0700E00F5000E0
:102FA000E08F580028003A0002002400130020009F
:102FB00000C0230011002000B5FF0700E0C123007E
:102FC000110020000000060000C0230011002000B6
:102FD000AAFE0700E00F5000E08F58001A003A00E8
:102FE000000024001100200096FE07000000E00011
:102FF00008003A0002C02300130020000000240053
:1030000011002000A2FF0700E001240011002000B1
:1030100000000600000024001100200097FE0700B9
:10302000E00F5000E08F580007003A000200240033
:103030001300200000C023001100200094FF0700AF
:10304000E0C123001100200000000600FC874700BB
:10305000881F78008A9FBE008C9FBE008E1F78005C
:103060000004EB00B1938000F0282000808F500016
:103070002F003400BBFF07000006BE00E0FD2F005C
:103080000F00400005FE07000C05BE00E1FD2F000B
:103090008F80400008804000B0407800A1DF9F0092
:1030A000AEFD2F000F074700306F7800104078000A
:1030B000104798005FA99700EFA997000A00BE008B
:1030C00054CC02000000000062054500E0854D0080
:1030D00063044400F50F5400ECFF3A006E00460014
:1030E000E0804E000200240013002000820F5000F8
:1030F000838F580005003A0002C02300130020000F
:1031000063FF0700180020000900370018002000A6
:103110000440240015002000840F5000858F5800C3
:1031200003003A0000C023001100200058FF0700F0
:10313000080078004F0778004F06BE004F05BE001C
:103140004F047800CF01B10000000600303F82003C
:10315000E10F400002003200617E24008008E80098
:1031600040610200000000000000E00006003D0099
:10317000707F240090407800E1CF40000A003200C8
:103180000148E80008003700E8004000627E2400A3
:10319000E2C07800E1CF4000030032008140E80047
:1031A00068014100017178008464AB000F003200B7
:1031B000D0F40200000000000000E0000600320031
:1031C000403F8200E10F400008003200817E240071
:1031D0008008E80000000600503F8200E10F400038
:1031E00002003200A17E24008008E80000000600F2
:1031F0000080FB00C300DE00927F240002814000BB
:10320000C308DD0001005000110020000008DD00AF
:10321000124970000000060061052000810F500077
:103220000B0039008100E800810F500004003600D7
:10323000F0804000810F500005003A000200370086
:1032400070C0B300EAFF370000C1B300E8FF070019
:103250000000060021062000810F500011003E00F2
:103260008180E900810F50001D003100F103200032
:10327000810F500007003E00E6805000810F500093
:1032800015003100A002B100E40F50001C003E0008
:103290000F0037000005B100E50F500018003E0098
:1032A0000D00370051062000810F500004003E0041
:1032B0008100E900810F50000D0031000A00370045
:1032C00061062000810F50000D003A000A0037000F
:1032D000F0C0B3000700370080C0B300050037001E
:1032E000E0C0B3000300370090C0B3000100370016
:1032F00010C1B300BEFF370000C1B300BCFF070020
:10330000000006008000EB004002B1000180B10027
:10331000EF0F5000E08F58001F003E0000600100DA
:103320000F0037000E0037000D0037000E00370089
:103330000F0037000E0037000D003700080037007F
:103340000D0037000E0037000D0037000E0037006B
:103350000D0037000C0037000F0037000C0037005D
:10336000A0C0B30009003700D0C0B3000700370089
:10337000C0C0B3000500370020C1B3000300370010
:10338000B0C0B3000100370030C1B30098FF370070
:1033900070C1B30096FF070000000600724980006C
:1033A0008349800061004100E08049007049880045
:1033B0008149880002302A0023002000820F50003B
:1033C000838F580007003A002E29EF003029EF00C4
:1033D000807F240090407800E1CF4000010032005F
:1033E0000148E800000006000001EB001102210086
:1033F0000001200026F902000000000081012000E9
:10340000607E240032F90200000000006AF9020028
:1034100000000000F03F8A000000060020C0B3005A
:1034200073FF37002C09EC006049880001A62E00CC
:10343000810F500002003A002C29EF0043FF0700E3
:1034400000000600889FBE008A1F780040F120001F
:10345000B1788000910078004A0020008004EB00E1
:1034600018002000908F500032003600770037009F
:103470008800440081004000E0FF2F001100500050
:103480008000EB00F00F5000E08F580022003E005B
:1034900000600100100037000F0037000E003700F9
:1034A0000D0037000C0037000B0037000C00370010
:1034B000190037000C0037000B0037000C003700F4
:1034C00015003700100037000B0037000C003700E4
:1034D0000F0037000E003700F0C0B3000D003700BA
:1034E00080C0B3000B003700E0C0B3000900370014
:1034F00000C1B3000700370010C1B300050037005A
:1035000070C0B3000300370040C1B30001003700B2
:1035100050C1B30036FF0700B078800060007D0026
:10352000808F540001003100800478000884E80096
:1035300064054500B0788000900F5400CCFF39003E
:103540003F003700B1788000080044006100780037
:103550004C01DE008001EB00ED0F5100E08F5900BF
:1035600036003E00026001000D00370033003700D6
:103570001D0037000D003700100037001300370022
:10358000160037002D0037002C00370018003700D8
:10359000150037001A003700250037001E003700DD
:1035A000890F54002500390028003700F1FF200062
:1035B0000100600027FF070020003700F1FF200016
:1035C0000100600014FF07001C003700F1FF20001D
:1035D000010060001FFF070003003700F1FF20001B
:1035E000010060000CFF07000884E80014003700A9
:1035F0004400DD004480DE00080040000800370081
:103600000800E800000040006100780011FF07009A
:10361000630444000A003700F1FF2000010060004D
:10362000808F5400050031008004780003003700CB
:10363000F1FF20000100600032FF07000804E800ED
:1036400040F12000900F5400BEFF39004F05780074
:103650004F04BE0000000600D07E24009040780099
:10366000E1CF4000010032000148E80075FF37005B
:10367000E2FC07000000E00003003A00607E240046
:103680000C0009000018EB004027AB0003003200DB
:1036900010C0B300D6FE07004027A900807F240099
:1036A0001004E00004003A00313F8200005A20007C
:1036B000808F50000600360064FE07000000E00026
:1036C00003003200607E24000C0009000018EB00AB
:1036D000C07E240090407800E1CF4000010032001D
:1036E0000148E800000006001C00FA00881F78006E
:1036F0008A9FBE000004780058019000E801900005
:1037000008007800D04F0200000000000AC023002B
:103710001B0020000A00BE007CCB0200000000005D
:1037200080B79F0091B79F00E3FD2F008F8141007C
:103730003200200001FE2F008F804000080078003A
:103740005E4D0200000000007FA89700E30F5000CC
:1037500025003A0062054500E0854D000040240048
:1037600011002000800F5500818F5D00E9FF3A00B5
:103770007C80570049FC0700E3FD2F008F8141004A
:1037800052012000FC805700080078005E4D0200C6
:1037900000000000607E24000C0009000018EB000F
:1037A00000C023001100200079FC07000000E000A9
:1037B0000400320000C02300110020001ACC0200D7
:1037C00000000000000024001100200070FC070031
:1037D0000000E0000400320000002400110020007E
:1037E0001ACC0200000000004F05BE004F04780014
:1037F0000080FA000000060090089000E0019000B0
:1038000001814000630179008100E90011089800FE
:1038100002007800000006000003BE0053002000F4
:103820000002EB0002712200110009000283D8009F
:1038300001037800800278000500E00004003A00EF
:103840000400E00002003A00E10F510003003A00DA
:1038500000C3B30080DB420014002000A50020005C
:10386000110009000581D800000178008301E900FA
:10387000EDFF3A000700780000000600E6FF0700B1
:10388000E1C2B3000148780071C7B3000168780055
:10389000F6C0500001687800F5C04000016878006B
:1038A0008040EB001140980000000600889FBE0099
:1038B0008A1F78008004780049049000090078008D
:1038C000CDFF070000004000680478004905900023
:1038D00009007800C8FF070000004000EA007800F7
:1038E000EF0F5400080032000800E0000600350029
:1038F00070022000800F540003003C000840780054
:10390000E8C50200000000004F0578004F04BE002B
:10391000000006000E00FA00881F7800F0805700B3
:10392000050009008018EB008058EB0001C7B300C8
:1039300081F79F0040049000AFFF070000004000A7
:10394000680478001000200092740200000000005B
:103950006CE00200000000000000EB00E10F4400FA
:1039600004003200EF80570008007800C3FF070012
:1039700070805700F4E00200000000004F0478005F
:103980000080FA00000006000E00FA00881F780090
:10399000F0805700050009008018EB008058EB000C
:1039A00021C7B30081F79F004004900092FF0700F9
:1039B0000000400068047800E10F440003003A0072
:1039C00070B3020000000000090037001000200062
:1039D0009274020000000000EF8057000800780099
:1039E000A6FF07007080570014B30200000000001B
:1039F0004F0478000080FA00000006000E00FA0074
:103A0000881F7800F0805700050009008018EB003F
:103A10008058EB0021C7B30081F79F00400490005D
:103A200075FF0700000040006804780010002000C7
:103A300092740200000000006CE002000000000030
:103A40000000EB00E10F440004003200EF8057005B
:103A50000800780089FF070070805700F4E002003A
:103A6000000000004F0478000080FA00000006000B
:103A7000F0874700889FBE008A1F78008E1F78005D
:103A80000004780076805700050009000018EB005C
:103A90000058EB007687570020C7B300005F78001E
:103AA000C80490000800780053FF070000004000A1
:103AB00069057800080078004FFF0700800478004F
:103AC0008E0078000A0078006CFF070089844400AB
:103AD00048009000890440007680570096B30200A9
:103AE00000000000800C78004F0778004F05780038
:103AF0004F04BE000F01B100000006000E00FA00E6
:103B0000881F7800F0805700050009008018EB003E
:103B10008058EB0031C7B30081F79F00400490004C
:103B200035FF070000004000680478001000200006
:103B300092740200000000006CE00200000000002F
:103B4000080078000EE10200000000000000E00024
:103B500006003200EF8057000800780047FF07009A
:103B600070805700F4E00200000000004F0478006D
:103B70000080FA0000000600E4874700889FBE002E
:103B80008A9FBE008C9FBE008E1F78008000780048
:103B9000410490000100780081BF9F0016FF0700DC
:103BA00000004000E80478008FB8970041049000BE
:103BB0000100780010FF0700000040006804780052
:103BC0008FB8970041059000010078000AFF0700B8
:103BD000000040006A0578008FB89700C10590008A
:103BE0000100780004FF070000004000EB057800AA
:103BF0008FB897004106900001007800FEFE070094
:103C0000000040006C0678008FB89700C106900055
:103C100001007800F8FE070000004000ED06780083
:103C20008FB897004107900001007800F2FE07006E
:103C3000000040006E0778008FB8970041019000A7
:103C40000100780082BF9F00EBFE070000004000EB
:103C50000FB99700E20378000010200087BF9F0093
:103C600092740200000000008FBB97000E437800A2
:103C70008D4278000C4278008B4178000A41780030
:103C80008840780009407800C8C6020000000000A3
:103C90004F0778004F06BE004F05BE004F04BE0020
:103CA0004F00B10000000600889FBE008A9FBE0042
:103CB000000578004A0490000A007800CEFE070054
:103CC0000000400068047800CA0490000A007800F0
:103CD000C9FE070000004000E9047800CA05900012
:103CE0000A007800C4FE0700000040006B01780065
:103CF000894078000840780018C7020000000000E2
:103D00004F05BE004F04BE0000000600889FBE00A5
:103D10008A9FBE00000578004A0490000A007800DF
:103D2000B5FE07000000400068047800CA04900057
:103D30000A007800B0FE070000004000E9047800A7
:103D4000CA0590000A007800ABFE070000004000A2
:103D50006B017800894078000840780034C7020081
:103D6000000000004F05BE004F04BE00000006002A
:103D7000889FBE008A9FBE00000578004A0490001C
:103D80000A0078009CFE07000000400068047800EC
:103D9000CA0490000A00780097FE07000000400067
:103DA000E9047800CA0590000A00780092FE070036
:103DB000000040006B0178008940780008407800DE
:103DC00050C70200000000004F05BE004F04BE00B7
:103DD00000000600889FBE008A9FBE008C1F7800EE
:103DE00000047800C80490000800780082FE0700F4
:103DF00000004000E9057800C80490000800780041
:103E00007DFE07000000400069057800C8049000AE
:103E10000800780078FE070000004000E904780000
:103E2000480690000800780073FE0700000040007C
:103E30006C04780020002000927402000000000052
:103E40008B40780000C2B300E8C50200000000000B
:103E50008A40780030C2B300E8C5020000000000CC
:103E60008940780010C2B300E8C5020000000000DD
:103E70008840780020C2B300E8C5020000000000BE
:103E80004F0678004F05BE004F04BE00000006003C
:103E9000E4874700889FBE008A9FBE008C9FBE00BB
:103EA0008E1F7800800078004104900001007800A7
:103EB00081BF9F0050FE070000004000E80478002A
:103EC0008FB8970041049000010078004AFE070077
:103ED00000004000680478008FB89700410590000A
:103EE0000100780044FE0700000040006A057800E9
:103EF0008FB89700C1059000010078003EFE0700D2
:103F000000004000EB0578008FB897004106900054
:103F10000100780038FE0700000040006C067800C1
:103F20008FB89700C10690000100780032FE0700AC
:103F300000004000ED0678008FB897004107900020
:103F4000010078002CFE0700000040006E0778009A
:103F50008FB89700410190000100780082BF9F0058
:103F600025FE0700000040000FB99700E20378002B
:103F70004000200087BF9F009274020000000000F4
:103F80008FBB97000E4378008D4278000C4278007A
:103F90008B4178000A417800884078000940780019
:103FA0006CC70200000000004F0778004F06BE00FB
:103FB0004F05BE004F04BE004F00B10000000600D8
:103FC000889FBE008A1F780000047800C804900013
:103FD0000800780008FE070000004000E9047800AF
:103FE000480590000800780003FE0700000040002C
:103FF0006A04780040002000927402000000000073
:104000008940780060C1B300E8C5020000000000EC
:104010008840780070C1B300E8C5020000000000CD
:104020004F0578004F04BE0000000600881F78008E
:1040300040049000F0FD0700000040006804780094
:104040000004200092740200000000008840780004
:10405000D0C1B300E8C50200000000004F047800A2
:1040600000000600881F780040049000E2FD070071
:1040700000004000680478000001200092740200F3
:104080000000000088407800E0C1B300E8C50200ED
:10409000000000004F04780000000600889FBE006A
:1040A0008A1F780000047800C80490000800780097
:1040B000D1FD070000004000E904780048059000A9
:1040C00008007800CCFD0700000040006A0478007A
:1040D0000020200092740200000000008940780057
:1040E00060C2B300E8C5020000000000884078000C
:1040F00070C2B300E8C50200000000004F05780060
:104100004F04BE0000000600889FBE008A1F780092
:10411000800478004904900009007800B6FD07008B
:10412000000040006804780049059000090078000C
:10413000B1FD070000004000EA04780010002000F4
:1041400092740200000000006CE002000000000019
:104150000800BE002EE10200000000004F057800BC
:104160004F04BE0000000600889FBE0000047800D7
:10417000C8049000080078009FFD07000000400080
:1041800000804400000178008000EB00030820005C
:1041900032824100F30F2000830F520005003600E9
:1041A000E1B1290008007800C6900200000000007C
:1041B000060037008100E800E3082000838F5000EC
:1041C000F2FF3A00E0F60200000000004F04BE00DB
:1041D00000000600881F78004004900086FD07005C
:1041E00000004000680078000000E000030032009A
:1041F0008CB10200000000000200370096B10200FE
:10420000000000004F047800000006000E00FA00D5
:10421000889FBE008A1F780000047800C8049000C0
:104220000800780074FD0700000040006905780070
:104230000800780070FD0700800478007480570043
:10424000050009000018EB000058EB0050C7B30050
:10425000C0EF9F00E10F450008003A000000EB00AE
:10426000C4B40200000000004800900089844400AB
:1042700089044000800CEB0014003700F3805700E5
:104280000A00780064FD0700E1C2B300014878002D
:1042900041C6B30001687800E3C0500001687800AF
:1042A000F3C04000016878008040EB0011409800A6
:1042B00089844400480090008904400074805700BD
:1042C000C4B4020000000000800C78004F057800A4
:1042D0004F04BE000080FA0000000600889FBE0068
:1042E0008A9FBE0080047800C9059000090078000C
:1042F00041FD070000057800090078003EFD070039
:1043000000047800090078003BFD07000804440021
:10431000C900900008844000800040000A05450064
:104320000A80450098B5020000000000000CD10092
:104330004F05BE004F04BE0000000600889FBE006F
:104340008A9FBE0080047800C905900009007800AB
:1043500029FD0700000578000900780026FD070008
:10436000000478000900780023FD070008044400D9
:10437000C900900008844000800040000A05450004
:104380000A80450052B5020000000000000CD10078
:104390004F05BE004F04BE0000000600889FBE000F
:1043A0008A1F780080047800490490000900780092
:1043B00011FD070000004000680578000900780042
:1043C0000DFD070000004000490490000004440077
:1043D0006150B900000040008180480012B5020021
:1043E00000000000000C78004F0578004F04BE006C
:1043F00000000600881F780040049000FEFC0700C3
:10440000000040006800780090C302000000000037
:10441000D0C40200000000004F0478000000060035
:10442000881F7800980E2000803E20004AFA020083
:10443000000000000804E900FBFF3A004F04780088
:104440000000060001C2B30080C0B300E8C502004E
:1044500000000000F2FF07008040EB0080C0B300C6
:10446000E8C502000000000001C2B30090C0B30024
:10447000E8C5020000000000E9FF07008040EB00F3
:1044800090C0B300E8C502000000000001C2B30004
:10449000A0C0B300E8C5020000000000E0FF070074
:1044A0008040EB00A0C0B300E8C50200000000009F
:1044B00001C2B300B0C0B300E8C5020000000000B4
:1044C000D7FF07008040EB00B0C0B300E8C5020092
:1044D0000000000001C2B300C0C0B300E8C5020084
:1044E00000000000CEFF07008040EB00C0C0B3001A
:1044F000E8C502000000000001C2B300D0C0B30054
:10450000E8C5020000000000C5FF07008040EB0086
:10451000D0C0B300E8C502000000000001C2B30033
:1045200020C0B300E8C5020000000000BCFF070087
:104530008040EB0020C0B300E8C50200000000008E
:1045400001C2B30030C0B300E8C5020000000000A3
:10455000B3FF07008040EB0030C0B300E8C50200A5
:104560000000000001C2B30040C0B300E8C5020073
:1045700000000000AAFF07008040EB0040C0B3002D
:10458000E8C504000000000001C2B30020C2B3006F
:10459000E8C5020000000000A1FF07008040EB001A
:1045A00020C2B300E8C502000000000001C2B30051
:1045B00001407800E8C502000000000098FF0700F5
:1045C0008040EB0000C2B300E8C50200000000001C
:1045D00001C2B30030C2B300E8C502000000000011
:1045E0008FFF07008040EB0030C2B300E8C5020037
:1045F0000000000001C2B30010C2B300E8C5020011
:104600000000000086FF07008040EB0010C2B300EE
:10461000E8C504000000000001C2B300C0C1B3003F
:10462000E8C50200000000007DFF07008040EB00AD
:10463000C0C1B300E8C502000000000001C2B30021
:1046400040C2B300E8C502000000000074FF07008C
:104650008040EB0040C2B300E8C50200000000004B
:1046600001C2B30050C2B300E8C502000000000060
:104670006BFF07008040EB0050C2B300E8C50200AA
:104680000000000001C2B300F0C1B300E8C50200A1
:104690000000000062FF07008040EB00F0C1B300A3
:1046A000E8C502000000000001C2B30080C1B300F1
:1046B000E8C502000000000059FF07008040EB0041
:1046C00080C1B300E8C502000000000001C2B300D1
:1046D00090C1B300E8C502000000000050FF0700D1
:1046E0008040EB0090C1B300E8C50200000000006C
:1046F00001C2B300A0C1B300E8C502000000000081
:1047000047FF07008040EB00A0C1B300E8C50200EE
:104710000000000001C2B300B0C1B300E8C5020050
:10472000000000003EFF07008040EB00B0C1B30076
:10473000E8C504000000000001C2B30000C1B300DE
:10474000E8C502000000000035FF07008040EB00D4
:1047500000C1B300E8C502000000000001C2B300C0
:1047600010C1B300E8C50200000000002CFF0700E4
:104770008040EB0010C1B300E8C50200000000005B
:1047800001C2B30040C1B300E8C502000000000050
:1047900023FF07008040EB0040C1B300E8C50200E2
:1047A0000000000001C2B30050C1B300E8C5020020
:1047B000000000001AFF07008040EB0050C1B3006A
:1047C000E8C502000000000001C2B30020C1B30030
:1047D000E8C502000000000011FF07008040EB0068
:1047E00020C1B300E8C502000000000001C2B30010
:1047F00030C1B300E8C502000000000008FF070058
:104800008040EB0030C1B300E8C5040000000000A8
:104810008040EB0050C0B300E8C50200000000007B
:10482000C5FF070001C2B300D0C1B300E8C5020054
:1048300000000000FAFE07008040EB00D0C1B3008A
:10484000E8C502000000000001C2B300E0C1B300EF
:10485000E8C5020000000000F1FE07008040EB0008
:10486000E0C1B300E8C502000000000001C2B300CF
:1048700050C0B300E8C5020000000000E8FE0700D9
:104880008040EB0050C0B300E8C50200000000000B
:1048900001C2B30060C0B300E8C502000000000020
:1048A000DFFE07008040EB0060C0B300E8C50200F7
:1048B0000000000001C2B30070C0B300E8C50200F0
:1048C00000000000D6FE07008040EB0070C0B3007F
:1048D000E8C50200000000004FFF07002AFF0700A4
:1048E00001C2B30060C2B300E8C5020000000000CE
:1048F000CBFE07008040EB0060C2B300E8C50200B9
:104900000000000001C2B30070C2B300E8C502009D
:1049100000000000C2FE07008040EB0070C2B30040
:10492000E8C502000000000001C2B3000040EB0037
:10493000E8C5020000000000B9FE07008040EB005F
:1049400001407800E8C502000000000001C2B30089
:10495000E0C0B300E8C5020000000000B0FE0700A0
:104960008040EB00E0C0B300E8C50200000000009A
:1049700001C2B30010C0B300E8C50200000000008F
:10498000A7FE07008040EB0010C0B300E8C502009E
:104990000000000001C2B30060C1B300E8C502001E
:1049A000000000009EFE07008040EB0060C1B300E5
:1049B000E8C502000000000001C2B30070C1B300EE
:1049C000E8C502000000000095FE07008040EB00F3
:1049D00070C1B300E8C502000000000099FE370076
:1049E0008BFF070001C2B30020C0B300E8C502007E
:1049F0000000000001C2B30000C1B300E8C502001E
:104A00000000000001C2B30010C1B300E8C50200FD
:104A10000000000001C2B30040C1B300E8C50200BD
:104A20000000000001C2B30020C1B300E8C50200CD
:104A30000000000001C2B30030C1B300E8C50200AD
:104A40000000000001C2B3000040EB00E8C5020016
:104A50000000000001C2B30010C0B300E8C50200AE
:104A60000000000001C2B300E0C1B300E8C50200CD
:104A70000000000001C2B30070C2B300E8C502002C
:104A80000000000001C2B30080C1B300E8C502000D
:104A90000000000001C2B30090C1B300E8C50200ED
:104AA0000000000001C2B300A0C1B300E8C50200CD
:104AB0000000000001C2B300B0C1B300E8C50200AD
:104AC0000000000001C2B300C0C1B300E8C502008D
:104AD0000000000001C2B30040C2B300E8C50200FC
:104AE0000000000001C2B30050C2B300E8C50200DC
:104AF0000000000001C2B300F0C1B300E8C502002D
:104B00000000000001C2B300D0C1B300E8C502003C
:104B10000000000001C2B30060C1B300E8C502009C
:104B20000000000001C2B30070C1B300E8C502007C
:104B30000000000001C2B30080C0B300E8C502005D
:104B40000000000001C2B300D0C0B300E8C50200FD
:104B50000000000001C2B300E0C0B300E8C50200DD
:104B600000000000008020007A74020000000000B5
:104B70001000200094E8040000000000C02821007C
:104B800072F32F0090004100A0122000808F50008F
:104B900005003E003809A8008040EB00634050004B
:104BA000E8C5020000000000602721008080E800C6
:104BB0009100780010804000813E20000182B90001
